:100000000C94012B0C94062E0C94312E0C945C2E27
:100010000C94872E0C94B22E0C94DD2E0C94082F89
:100020000C94332F0C94322B0C94322B0C94322BD7
:100030000C94322B0C94322B0C94322B0C94322BCC
:100040000C94322B0C941CBE0C94322B0C94322B3F
:100050000C94322B0C94322B0C94FAB00C94342B5D
:100060000C94322B0C942F9D0C94DB9D0C94322B12
:100070000C94322B0C94322B0C94322B0C94322B8C
:100080000C94322B0C94322B0C94322B0C94322B7C
:100090000C94322B0C94322B0C94322B0C94322B6C
:1000A0000C94322B0C94322B0C94322B0C94322B5C
:1000B0000C94322B0C94322B0C94322B0C94322B4C
:1000C0000C94322B0C94322B0C94322B0C94322B3C
:1000D0000C94322B0C94322B0C94322B0C94322B2C
:1000E0000C94322B7C2C812C862C902C9A2C132D4A
:1000F000A42CAC2CB42CBE2CC82CD22CE12CEB2C78
:10010000132DF52CFF2C092D372D3A2D292D2D2DB2
:10011000332D712D3E2D422D482D4C2D502D562D19
:100120005A2D5E2D712D642D682D6C2D326012605C
:10013000186015601B601E6021602D6024603F60A8
:1001400027602A606A9A689A8C9A899A879ABE9AD6
:10015000BB9AB99A179BE59AE29AE09A629D689DCC
:10016000799D849D8C9DA19D909DA19D949D989D20
:10017000A19D9E9D084AD73B3BCE016E84BCBFFD2E
:10018000C12F3D6C74319ABD56833DDA3D00C77F67
:1001900011BED9E4BB4C3E916BAAAABE0000008000
:1001A0003F05A84CCDB2D44EB93836A9020C50B98F
:1001B000918688083CA6AAAA2ABE000000803F00BB
:1001C0000D940C180D94553B0D944C2C0D940D4032
:1001D0004E414E494E495459494E46CDCCCC3D0A2C
:1001E000D7233C17B7D13877CC2B329595E6241F0F
:1001F000B14F0A000020410000C84200401C4620C8
:10020000BCBE4CCA1B0E5AAEC59D7400000A0B0240
:10021000090C0D0E08070304010000000000000097
:1002200000000000000000000000000000000000CE
:10023000000000000000001211100000000000008B
:1002400000000000000000000000000000000000AE
:1002500000010210202008081020401020408002D9
:1002600001020108040201010204081020408080FC
:100270004020100804020180040201804020100880
:100280000402010804020101020408102040800158
:100290000204081020408005050505070508080828
:1002A00008020202020A0A08080404040401010107
:1002B000010101010103030303030303030407070F
:1002C000070C0C0C0C0C0C0C0C02020202060606AD
:1002D00006060606060B0B0B0B0B0B0B0B00002088
:1002E000002300260029002C002F0032000001000E
:1002F0000003010601090100002200250028002B4F
:10030000002E003100340002010000050108010B3D
:100310000100002100240027002A002D00300033B6
:100320000001010000040107010A0101060D00FEA1
:1003300009016602D620FFFE0BFE0AFE0D006022B8
:100340001969808080808080800080183363A0A03D
:10035000A00357675050F850F85050025969207860
:10036000A0A0702828F02002596948A85010204009
:1003700050A89002586840A0A040A0989068281308
:1003800063808080113B6B20404080808080804073
:100390004020113B6B8040402020202020404080A6
:1003A00006556520A870A8200455652020F8202057
:1003B000113363604080065161F811336340E040BF
:1003C00002596908081010204040808002596920B5
:1003D00050888888888850200259692060A0202091
:1003E000202020F80259697088880810204080F881
:1003F000025969F8081020700808887002596910BD
:100400001030505090F81010025969F88080B0C830
:100410000808887002596970888080F08888887020
:10042000025969F8081010202040404002596970B4
:100430008888887088888870025969708888887868
:100440000808887011386840E040000040E0401122
:10045000386840E040000060408002596908102080
:10046000408040201008045464F80000F8025969E4
:100470008040201008102040800259697088880848
:10048000102020002002596970888898A8A8B080A0
:10049000780259692050888888F8888888025969C4
:1004A000F048484870484848F00259697088808090
:1004B0008080808870025969F04848484848484818
:1004C000F0025969F8808080F0808080F8025969D4
:1004D000F8808080F08080808002596970888080F8
:1004E000809888887002596988888888F888888800
:1004F00088123969E040404040404040E00259697C
:10050000381010101010109060025969888890A05F
:10051000C0A0908888025969808080808080808017
:10052000F80259698888D8A8A888888888025969F3
:1005300088C8C8A8A8989888880259697088888847
:100540008888888870025969F0888888F08080805F
:1005500080015A6A70888888888888A8700802593B
:1005600069F0888888F0A09088880259697088802E
:10057000807008088870025969F820202020202007
:10058000202002596988888888888888887002595C
:100590006988888888505050202002596988888846
:1005A00088A8A8A8A850025969888850502050509F
:1005B00088880259698888505020202020200259BC
:1005C00069F808101020404080F8113B6BE08080F3
:1005D00080808080808080E0025969808040402057
:1005E00010100808113B6BE0202020202020202044
:1005F00020E0085363205088015161F82A2262806C
:100600004002566670087888986802596980808030
:10061000F088888888F0025666708880808870022A
:10062000596908080878888888887802566670882A
:10063000F880887002596930484040F0404040409E
:1006400000586870888888780888700259698080A6
:1006500080B0C8888888881238684000C040404010
:1006600040E0004A6A1000301010101090906002B4
:10067000596980808090A0C0A09088123969C040DC
:10068000404040404040E0025666D0A8A8A8A88854
:10069000025666B0C888888888025666708888883E
:1006A0008870005868F0888888F0808080005868DA
:1006B0007888888878080808025666B0C8808080E4
:1006C000800256667088601088700258684040F05A
:1006D00040404048300256668888888898680256AC
:1006E000668888885050200256668888A8A8A85036
:1006F000025666885020205088005868888888985C
:1007000068088870025666F810204080F8015B6B1C
:100710001820202020C02020202018221969808045
:1007200080808080808080015B6BC020202020182A
:1007300020202020C008536348A890FFFFFFFFFF40
:10074000FFFFFFFFFFFFFFFFFFFFFFFFFFFFFFFFB9
:10075000FFFFFFFFFFFFFFFFFFFFFFFF0D00602216
:1007600019698000808080808080800358682070B4
:10077000A8A0A0A8702002596930484040E040403D
:1007800048B003566688705050708802596988884E
:100790005050F820F8202022196980808080008045
:1007A000808080124A6A60908060909060109060B3
:1007B0001A3262A0A00359697088A8D8C8D8A8883E
:1007C00070045767700878887800F80356662850D8
:1007D000A0A05028045363F80808163161E00359BB
:1007E000697088E8D8D8E8D888700A5161F8174449
:1007F00064609090600357672020F8202000F8077D
:10080000356540A02040E007356540A04020C02A63
:10081000226240800058688888888898E880800232
:10082000596978E8E8E8E868282828262161C02086
:100830002262408007356540C04040E00457677041
:100840008888887000F8035666A050282850A002B7
:100850005A6A40C04040E00818283808025A6A40E6
:10086000C04040E01028081038025A6A40A04020DA
:10087000A0481828380802596920002020408088A4
:100880008870025A6A40200020508888F8888802C0
:100890005A6A10200020508888F88888025A6A30E6
:1008A000480020508888F88888025A6A285000201A
:1008B000508888F88888025A6A50500020508888EA
:1008C000F88888025A6A20502020508888F8888842
:1008D00002596958A0A0A0B0E0A0A0B8005B6B705E
:1008E00088808080808088702040025A6A40200082
:1008F000F88080F08080F8025A6A102000F880802A
:10090000F08080F8025A6A304800F88080F08080D9
:10091000F8025A6A505000F88080F08080F8123A4D
:100920006A804000E04040404040E0123A6A204087
:1009300000E04040404040E0124A6A609000E040E1
:1009400040404040E0123A6AA0A000E040404040F1
:1009500040E0025969F0484848E8484848F0025ADF
:100960006A2850008888C8A8988888025A6A402057
:100970000070888888888870025A6A102000708801
:100980008888888870025A6A304800708888888809
:100990008870025A6A285000708888888888700297
:1009A0005A6A505000708888888888700355658816
:1009B00050205088015B6B08709898A8A8A8C8C8F8
:1009C0007080025A6A40200088888888888870026F
:1009D0005A6A10200088888888888870025A6A308D
:1009E000480088888888888870025A6A5050008831
:1009F000888888888870025A6A1020008888502069
:100A000020202002596980F0888888F08080800248
:100A10005969609090A0A0908888B00259694020E0
:100A2000007008788898680259691020007008786A
:100A30008898680259693048007008788898680278
:100A40005969285000700878889868025969505090
:100A500000700878889868025A6A30483000700838
:100A600078889868025666702870A0A85000586868
:100A7000708880808870204002596940200070880A
:100A8000F88088700259691020007088F88088709A
:100A90000259693048007088F8808870025969509E
:100AA00050007088F8808870123969804000C0401A
:100AB000404040E0123969204000C040404040E0E2
:100AC000124969609000C040404040E0123969A07E
:100AD000A000C040404040E0025A6A5020601070C0
:100AE0008888888870025969285000B0C88888882A
:100AF0008802596940200070888888887002596986
:100B00001020007088888888700259693048007009
:100B10008888888870025969285000708888888879
:100B20007002596950500070888888887003576730
:100B3000202000F8002020015868087098A8A8C854
:100B40007080025969402000888888889868025916
:100B500069102000888888889868025969304800A0
:100B600088888888986802596950500088888888E1
:100B70009868005B6B1020008888889868088870E7
:100B8000005A6A8080B0C88888C8B08080005B6BDB
:100B9000505000888888986808887001050700FE12
:100BA0000500FB01F220FFFE05FE05FE02004002EB
:100BB00015258080800080053242A0A00255655036
:100BC000F850F8500146562070C030E020025565BC
:100BD0009010204048025565608068906805122298
:100BE000808002253540808080400225358040404D
:100BF0004080043343A040A003334340E04001223F
:100C0000324080043141E002112180025565081014
:100C10002040800245556090909060022535C0408C
:100C2000404040024555E0106080F0024555E0101C
:100C30006010E00245552060A0F020024555F0808C
:100C4000E010E00245556080E09060024555F010EC
:100C5000204040024555609060906002455560908C
:100C600070106003132380008002142480008080B1
:100C70000235452040804020033343E000E0023548
:100C8000458040204080024555E0106000400255FC
:100C9000657088B8A870024555609090F090024544
:100CA00055E090E090E0023545608080806002452C
:100CB00055E0909090E0023545E080E080E002351C
:100CC00045E080E080800245557080B0907002451C
:100CD000559090F09090023545E0404040E002454C
:100CE00055301010906002455590A0C0A09002357C
:100CF0004580808080E002556588D8A888880245B4
:100D00005590D0B09090024555609090906002450B
:100D100055E09090E08001465660909090601002FF
:100D20004555E09090E09002455570806010E002DB
:100D30003545E0404040400245559090909060021B
:100D400045559090A0A04002556588A8A8A85002DB
:100D500045559090609090024555909070106002BB
:100D60003545E0204080E0022535C0808080C0020B
:100D700055658040201008022535C0404040C00520
:100D8000324240A0024151F00522328040024454D8
:100D90007090907002455580E09090E0023444607D
:100DA000808060024555107090907002445460B08D
:100DB000C0600235452040E04040004656709090AB
:100DC00070106002455580E09090900215258000DB
:100DD00080808000273740004040404080024555D9
:100DE0008090A0E09002152580808080800254646D
:100DF000F0A8A8A8024454E0909090024454609057
:100E00009060004656E09090E080800046567090DA
:100E100090701010023444A0C0808002445470C00E
:100E200030E002354540E04040200244549090902C
:100E3000700244549090A040025464A8A8505002FC
:100E40003444A04040A0004656909090701060023C
:100E50004454F02040F00235456040804060021567
:100E6000258080808080023545C0402040C00542FA
:100E70005250A0FFFFFFFFFFFFFFFFFFFFFFFFFF3D
:100E8000FFFFFFFFFFFFFFFFFFFFFFFFFFFFFFFF72
:100E9000FFFFFFFF020040FFFFFFFFFFFFFFFFFF1D
:100EA000FFFFFFFFFFFFFFFFFFFFFFFFFFFFFFFF52
:100EB000FFFFFFFFFFFFFFFFFFFFFFFFFFFFFFFF42
:100EC000FFFFFFFFFFFFFFFFFFFFFFFFFFFFFFFF32
:100ED000FFFFFFFFFFFFFFFFFFFFFFFFFFFFFFFF22
:100EE000FFFFFFFFFFFFFFFFFFFFFFFFFFFFFFFF12
:100EF000FFFFFFFFFFFF01050800FF06012102358C
:100F000020FFFF07FF06FF09005022165680808051
:100F1000800080153353A0A0A00257575050F850BE
:100F2000F850500257572070A07028702013355584
:100F300080A040A02002475740A0A040A0A050257C
:100F40001353808080122656408080808040122675
:100F5000568040404040800245559060F0609002CD
:100F600055552020F8202011335360408004415112
:100F7000F011335340E0400246561010204080806C
:100F800012365640A0A0A0A04012365640C04040A5
:100F900040E00246566090106080F0024656F02015
:100FA000601090600246562060A0F0202002465655
:100FB000F080E01090600246566080E09090600201
:100FC0004656F010202040400246566090609090B7
:100FD00060024656609090701060122555C0C000A7
:100FE000C0C0113656606000604080123656204006
:100FF00080804020034353F000F01236568040209A
:1010000020408012365640A0204000400158583001
:101010004898A8A8904030024656609090F0909072
:10102000024656E090E09090E00246566090808044
:101030009060024656E090909090E0024656F08014
:10104000E08080F0024656F080E0808080024656C4
:10105000609080B090600246569090F09090901210
:101060003656E040404040E002465670202020A026
:101070004002465690A0C0A0A090024656808080B4
:101080008080F002465690F0F09090900246569084
:10109000D0F0B0B0900246566090909090600246BA
:1010A00056E09090E08080014757609090D0B0600B
:1010B00010024656E09090E09090024656609040B4
:1010C000209060123656E040404040400246569024
:1010D000909090906002465690909090606002468A
:1010E00056909090F0F090024656909060609090EC
:1010F000025656888850202020024656F010204084
:1011000080F0123656E080808080E0024656808073
:1011100040201010123656E020202020E0163252D7
:1011200040A0014151F01622528040024454709078
:1011300090700246568080E09090E01234546080B7
:10114000806002465610107090907002445460B057
:10115000C060024656205040E04040014555609036
:101160007010600246568080E09090901236564093
:1011700000C04040E01137572000202020A040024E
:101180004656808090E09090123656C040404040D5
:10119000E0025454D0A8A8A8024454E090909002D1
:1011A000445460909060014555E090E08080014596
:1011B000557090701010024454A0D08080123454A6
:1011C00060C020C00246564040E0405020024454D7
:1011D00090909070123454A0A0A04002545488A85B
:1011E000A8500244549060609001455590907090D2
:1011F00060024454F02040F0024757304020C020A5
:101200004030221656808080808080024757C02060
:1012100040304020C006425250A0FFFFFFFFFFFFBA
:10122000FFFFFFFFFFFFFFFFFFFFFFFFFFFFFFFFCE
:10123000FFFFFFFFFFFFFFFFFFFFFF090050221628
:10124000568000808080800146562070A0A07020CB
:101250000246562050E04050A0025555887050700C
:10126000880256568850F820F82022175780808030
:10127000008080800247577080E0907010E0173146
:1012800051A002565670A8C8C8A87014355560A061
:101290006000E003435350A050123353E020201469
:1012A0003151E002565670E8D8E8D870173151E055
:1012B00015335340A04012355540E04000E014354E
:1012C0005540A02040E0143555C020C020C0162253
:1012D000524080014555909090E08002565678E843
:1012E000E868282824115180112252408014355575
:1012F00040C04040E014355540A04000E003435357
:10130000A050A0024757808080A060F0200247577D
:101310008080A0D010207002475780408060A0F0ED
:101320002012365640004080A040024757402060BF
:1013300090F0909002475720406090F090900247C4
:101340005760906090F0909002475750A06090F0E6
:10135000909002475790006090F09090024757603D
:10136000906090F0909002465670A0A0F0A0B0015E
:101370004757609080809060400247574020F0803F
:10138000E080F00247572040F080E080F0024757AD
:101390006090F080E080F00247579000F080E0809D
:1013A000F01237578040E0404040E012375720406D
:1013B000E0404040E012375740A0E0404040E0129B
:1013C0003757A000E0404040E00256567048E848D9
:1013D000487002475750A090D0B0909002475740B5
:1013E00020609090906002475720406090909060FD
:1013F0000247576090609090906002475750A060FD
:1014000090909060024757900060909090601233E7
:1014100053A040A002465670B0B0D0D0E00247576B
:10142000402090909090600247572040909090907C
:1014300060024757609090909090600247579000EC
:1014400090909090600257571020885020202002E2
:10145000465680E09090E0800246566090A0A090B2
:10146000A0024757402000709090700247572040DC
:10147000007090907002475720500070909070025A
:10148000475750A0007090907002465650007090E0
:10149000907002475760906070909070025454F0C2
:1014A00068B0781135556080806040024757402011
:1014B0000060B0C06002475720400060B0C06002CA
:1014C000475760900060B0C060024656500060B060
:1014D000C060123757804000C04040E012375720AC
:1014E0004000C04040E012375740A000C04040E0FC
:1014F000123656A000C04040E0024757A040A0105E
:1015000070906002475750A000E0909090024757BB
:10151000402000609090600247572040006090900B
:10152000600247576090006090906002475750A05B
:101530000060909060024656900060909060123576
:10154000554000E0004002445470B0D0E0024757DC
:10155000402000909090700247572040009090905B
:10156000700247576090009090907002465690002D
:1015700090909070014858204000909070906001C9
:1015800047578080E090E08080014757900090901E
:10159000709060202020200020202020202020008B
:1015A00025753A2530327500253032753A253032AE
:1015B000750025756420253032753A253032750066
:1015C0003FFFF03800703186302387102787902F37
:1015D00087D02F03D02030102078102078102030B2
:1015E000102F03D02F87D027879023871031863084
:1015F0003800703FFFF03FFFF038007030FC3020C3
:10160000FC102078102030102C00D02E31D02F7BF1
:10161000D02F7BD02E31D02C00D02030102078104D
:1016200020FC1030FC303800703FFFF00410400206
:1016300008200208200410400820801041001041BA
:10164000000820800410400000001FFFF81FFFF872
:101650001FFFF81FFFF81FE020102010201010209F
:1016600010202010201030300840048003001FE0BC
:101670003FF03FF03FF01FE01FE03FF03FF03FF052
:101680000FC0078003004572723A207574663820D7
:10169000666F6E74206E6F7420696E697469616C18
:1016A000697A65642E004572723A20757466382036
:1016B000666F6E74206E6F7420696E697469616CF8
:1016C000697A65642E004572723A20757466382016
:1016D000666F6E74206E6F7420696E697469616CD8
:1016E000697A65642E00506C65617365207265735C
:1016F0006574005052494E5445522048414C54455F
:1017000044007F80FFC0FFC0FFC07F807F80FFC09C
:10171000FFC0FFC03F001E000C00FFFFFF0E000EC9
:10172000000E000E000E000E000E000E007FC03FE7
:10173000801F000E00040004000E001F003F807F89
:10174000C00E000E000E000E000E000E000E000E69
:101750000000FE0003FF800783C00E01C00E00E002
:101760001C00E07F00E03E00E01C00E00800E0001C
:1017700000E00001C00E01C00F078007FF0001FC60
:101780000001FC0007FF000F07800E01C00001C030
:101790000000E00800E01C00E03E00E07F00E01CEC
:1017A00000E00E00E00E01C00783C003FF8000FED2
:1017B0000000060C00FE07022603BC017FFE08FEA7
:1017C00008FE05080806000040F0C88888987810D0
:1017D000050808060000C0F88888888888F805058C
:1017E000050600012030F83020050808060000201A
:1017F00070F820202020E00509090600FF2070A8CD
:10180000A8B888887020050606060001E08CEA8CDE
:101810008A0A0509090600FFF8A88888888888A828
:10182000F8050A0A0600FE205050505088A8A888E3
:101830007003030306000340A040FFFFFFFFFFFF0C
:10184000FFFFFFFFFFFFFFFFFFFFFFFFFFFFFFFFA8
:101850000000000605FF0107070602008080808067
:10186000800080030303060105A0A0A0050606066C
:10187000000050F85050F8500509090600FF20708C
:10188000A8A07028A87020050707060000C8C81087
:101890002040989805070706000040A0A040A890A7
:1018A000680103030602058080800309090601FF21
:1018B0002040408080804040200309090601FF80CD
:1018C000404020202040408005070706000020A857
:1018D000702070A8200505050600012020F82020B2
:1018E0000203030601FFC04080050101060003F862
:1018F000020202060100C0C005070706000008102A
:101900001020404080050707060000708898A8C88E
:10191000887003070706010040C040404040E005D2
:101920000707060000708808102040F80507070622
:101930000000F8081030088870050707060000103E
:10194000305090F81010050707060000F880F008E6
:10195000088870050707060000304080F08888700E
:10196000050707060000F8081010202020050707CB
:1019700006000070888870888870050707060000D8
:1019800070888878081060020505060100C0C00054
:10199000C0C00206060601FFC0C000C040800305AB
:1019A000050601012040804020050303060002F8DF
:1019B00000F8030505060101804020408005070767
:1019C0000600007088102020002005070706000090
:1019D0007088B8A8B880700507070600007088886E
:1019E000F8888888050707060000F04848704848CE
:1019F000F005070706000070888080808870050762
:101A000007060000F04848484848F0050707060068
:101A100000F88080F08080F8050707060000F88055
:101A200080F080808005070706000070888080981D
:101A30008870050707060000888888F8888888036A
:101A40000707060100E04040404040E00507070668
:101A5000000038101010109060050707060000887D
:101A600090A0C0A0908805070706000080808080B5
:101A70008080F805070706000088D8A8888888882D
:101A80000507070600008888C8A898888805070702
:101A9000060000708888888888700507070600009F
:101AA000F08888F08080800507070600007088882D
:101AB00088A89068050707060000F08888F0A090C5
:101AC0008805070706000070888070088870050781
:101AD00007060000F8202020202020050707060028
:101AE000008888888888887005070706000088882D
:101AF000888850502005070706000088888888A835
:101B0000A8500507070600008888502050888805DF
:101B100007070600008888502020202005070706B8
:101B20000000F80810204080F80309090601FFE0D2
:101B300080808080808080E005070706000080406C
:101B400040201010080309090601FFE02020202092
:101B5000202020E005030306000520508805010130
:101B60000600FEF803030306010580402005050575
:101B70000600007008788878050707060000808056
:101B8000F0888888F0050505060000708080887060
:101B90000507070600000808788888887805050585
:101BA0000600007088F080700507070600003048C6
:101BB00040E04040400507070600FE7088888878AE
:101BC00008700507070600008080F0888888880371
:101BD00007070601004000C0404040E00409090634
:101BE00001FE10003010101010906005070706006D
:101BF0000080808890E09088030707060100C040BD
:101C000040404040E0050505060000D0A8A8A8A86F
:101C1000050505060000B0C888888805050506008A
:101C20000070888888700507070600FEF08888889D
:101C3000F080800507070600FE7888888878080805
:101C4000050505060000B0C8808080050505060072
:101C50000078807008F00507070600002020F820B3
:101C60002020180505050600008888889868050565
:101C700005060000888888502005050506000088B4
:101C800088A8A85005050506000088502050880542
:101C900007070600FE888888502040800505050655
:101CA0000000F8102040F80309090601FF20404019
:101CB0004080404040200109090602FF808080806A
:101CC00080808080800309090601FF804040402019
:101CD0004040408005030306000248A890FF1FFF14
:101CE000FFFFFFFFFF600000000001FF4000000059
:101CF0000000FF8000000000007F83CF00000C3058
:101D00003F87FF80000C301F867980000C000F8C0D
:101D100030C7838C30E78C30CFC7CC31F38C30DCCC
:101D2000ECEC33B98C30D86C6C33198C30D06C0C33
:101D300033198C30D86C0C33198C30DC6C0E3B1999
:101D40008C30CF7C079F198C30C77C038F194000E3
:101D50000000000002600000000000061FFFFFFFFF
:101D6000FFFFF8000000000000000000000000007D
:101D70000000000000000000000000000000000063
:101D80000000000000000C000000000000000C003B
:101D9000000000000000120000000000000023000E
:101DA00000000000000021000000000000004C8046
:101DB0000000000000005E80000000000000924073
:101DC000000000000000A1400000000000012120F0
:101DD0000000000000027F900000000000020010E0
:101DE000000000000007FFF80000000000040008E9
:101DF00000000000000800040000000000080006C9
:101E000000000000001000020000000000301E0171
:101E10000000000000207F81000000000041FFE082
:101E2000800000000043FCF08000000000873B7849
:101E300040000000018EDBFC60000000010FEBCCD5
:101E400020000000021FEDB610000000021FDEB6E9
:101E5000100000000439CD7F080000000436E0FFC8
:101E600008000000087EC0BB84000000187F005DF1
:101E700086000000107FC0ED82000000203CC0738F
:101E800001000000203B337F01000000701BE77E53
:101E900003800000C81DEEDE04C00000880FDEDCF9
:101EA00004400001240FDF3C092000012607DBF875
:101EB000192000027203E7F0139000025101FFE0C5
:101EC0002290000489007F802448000904801E00BD
:101ED0004824000BFE400000DFF40010004000002A
:101EE0008002001FFFFFFFFFFFFE00000000000058
:101EF00000000000000000000000000000000000E2
:101F00000000001022103C3C0E1F00102210042282
:101F10001104001022100822110400102210083CA5
:101F2000110400102210102211040010221020228F
:101F30001104001E1C1E3C3C0E04000000000000AA
:101F40000000000000000000000000000000000091
:101F50000000000000000000000000000000000081
:101F60000000000000000000000000000000000071
:101F70000000000000000000000000000000000061
:101F80000000000000000000000000000000000051
:101F90000000000000000000000000000000000041
:101FA0000000060900FE06018902FE20FFFE07FE72
:101FB00006FE0000000600070106060602008080FB
:101FC00080800080030303060103A0A0A00507078B
:101FD0000600FF5050F850F850500509090600FE61
:101FE0002070A8A07028A870200608080600FF40EE
:101FF000A84810204854080507070600FF60909085
:10200000609890680103030602038080800207073E
:102010000602FF408080808080400207070602FFA2
:10202000804040404040800505050600008850F88B
:1020300050880505050600002020F8202002040431
:102040000602FEC0404080050101060002F80202BF
:1020500002060200C0C0040606060100101020405F
:102060008080040606060100609090909060030650
:102070000606010040C0404040E00406060601009C
:102080006090102040F0040606060100F020601069
:1020900010E005060606000010305090F810040607
:1020A00006060100F080E01010E0040606060100BC
:1020B0006080E0909060040606060100F010102099
:1020C000404004060606010060906090906004069F
:1020D000060601006090907010600205050602007F
:1020E000C0C000C0C00207070602FEC0C000C0405A
:1020F0004080050505060000186080601805030390
:10210000060001F800F8050505060000C03008309B
:10211000C0040707060100609010604000400506FB
:10212000060600007090A8B0807005060606000044
:10213000205088F88888050606060000F088F08898
:1021400088F0040606060100609080809060040616
:1021500006060100E090909090E00406060601005B
:10216000F080E08080F0040606060100F080E08048
:102170008080040606060100609080B0906004062E
:10218000060601009090F09090900306060601006C
:10219000E040404040E00506060600003810101000
:1021A000906004060606010090A0C0A0909004066E
:1021B000060601008080808080F00506060600008B
:1021C00088D8A8A8888804060606010090D0B09098
:1021D00090900506060600007088888888700406BE
:1021E00006060100E09090E080800407070601FFEA
:1021F000609090D0B06010040606060100E0909058
:10220000E090900406060601006090402090600572
:102210000606060000F820202020200406060601FD
:1022200000909090909060040606060100909090B7
:10223000F060600506060600008888A8A8D8880512
:102240000606060000885020205088050606060075
:1022500000888850202020040606060100F0102087
:102260004080F0030606060100E080808080E004E4
:1022700006060601008080402010100306060601B5
:1022800000E020202020E005030306000320508802
:102290000501010600FEF802020206020480400465
:1022A0000404060100709090700406060601008088
:1022B00080E09090E00404040601007080807004C7
:1022C00006060601001010709090700404040601C8
:1022D0000060B0C070040606060100205040E040D7
:1022E000400406060601FE60909070106004060629
:1022F0000601008080E090909003060606010040F1
:1023000000C04040E00308080601FE2000602020D5
:1023100020A0400406060601008080A0C0A0900313
:102320000606060100C040404040E00504040600E7
:1023300000D0A8A888040404060100E0909090044E
:102340000404060100609090600406060601FEE0A9
:102350009090E080800406060601FE709090701058
:1023600010040404060100A0D080800404040601C7
:102370000070C030E00406060601004040E0405016
:1023800020040404060100909090700404040601E7
:10239000009090606005040406000088A8A850041E
:1023A0000404060100906060900406060601FE9099
:1023B0009090709060040404060100F02040F00347
:1023C0000707060100204040804040200107070623
:1023D00002FF8080808080808003070706010080E4
:1023E00040402040408004020206010350A0FFFF4D
:1023F000FFFFFFFFFFFFFFFFFFFFFFFFFFFFFFFFED
:10240000FFFFFFFFFFFFFFFFFFFFFFFFFFFFFF00DB
:10241000000006000701060606020080008080809A
:10242000800406060601FF2070A0A07020050707A3
:102430000600FF304840F04040F805050506000062
:10244000A8508850A80506060600008850F820F815
:10245000200107070602FF8080800080808004073B
:10246000070601FF708060906010E0030101060123
:1024700005A0060707060000788494A494847803D6
:10248000050506010160A06000E0050505060000E5
:102490002850A05028040303060100F01010040186
:1024A00001060102F00607070600007884B4A4A420
:1024B0008478040101060105F004030306010260AB
:1024C00090600507070600FF2020F8202000F80391
:1024D000050506010140A02040E0030505060101B5
:1024E000C0204020C002020206020440800405050C
:1024F0000601FF9090B0D08005060606000078E83F
:10250000E868282801010106020280020202060290
:10251000FE408003050506010140C04040E0030580
:102520000506010140A04000E0050505060000A0E9
:10253000502850A00508080600FF40C040507030E9
:1025400078100508080600FF40C0405068081038A1
:102550000508080600FFC0204030F030781004075E
:102560000706010020002060809060050707060034
:1025700000402020507088880507070600001020C2
:1025800020507088880507070600002050205070F2
:1025900088880507070600002850205070888805A5
:1025A00007070600005000205070888805070706BE
:1025B000000020502050708888050606060000782C
:1025C000A0F0A0A0B80408080601FE6090808090EA
:1025D0006020400407070601004020F080E080F002
:1025E0000407070601002040F080E080F0040707A0
:1025F0000601002050F080E080F00407070601008B
:102600005000F080E080F00307070601008040E002
:10261000404040E00307070601002040E040404002
:10262000E003070706010040A0E0404040E0030748
:1026300007060100A000E0404040E0050606060055
:10264000007048E848487004070706010050A09051
:10265000D0B0909004070706010040206090909051
:102660006004070706010020406090909060040716
:102670000706010020506090909060040707060153
:102680000050A06090909060040707060100500081
:1026900060909090600505050600008850205088E5
:1026A0000408080601FF1070B0B0D0D0E080040725
:1026B00007060100402090909090600407070601F3
:1026C0000020409090909060040707060100205081
:1026D0009090909060040707060100500090909041
:1026E0009060050707060000102088502020200475
:1026F000060606010080E09090E0800406060601D0
:10270000006090A0A090A0040707060100402000F0
:1027100070909070040707060100204000709090B0
:1027200070040707060100205000709090700407A5
:102730000706010050A00070909070040606060184
:102740000050007090907004070706010020502090
:102750007090907005040406000070A8B07804061C
:10276000060601FE70808070204004070706010005
:1027700040200060B0C07004070706010020400040
:1027800060B0C07004070706010020500060B0C0B0
:1027900070040606060100500060B0C07003070711
:1027A000060100804000C04040E00307070601002A
:1027B000204000C04040E003070706010040A000A1
:1027C000C04040E0030606060100A000C04040E013
:1027D000040707060100306010709090600407073E
:1027E00006010050A000E090909004070706010049
:1027F0004020006090906004070706010020400020
:1028000060909060040707060100205000609090DF
:102810006004070706010050A00060909060040665
:102820000606010050006090906005050506000056
:102830002000F8002004040406010070B0D0E00479
:1028400007070601004020009090907004070706DB
:1028500001002040009090907004070706010020BE
:102860005000909090700406060601005000909071
:1028700090700409090601FE20400090909070902D
:10288000600408080601FE8080E09090E0808004EB
:1028900008080601FE5000909090709060536E34CE
:1028A0006B3300496E7661646572730042726963CE
:1028B0006B6F7574004D61696E005072696E7420A3
:1028C00066726F6D205344005072696E7420667298
:1028D0006F6D20534400022E2E004D61696E005032
:1028E00072696E740043616E63656C00537461724B
:1028F00074207072696E7420003F00536D6F6F74A6
:1029000068696E6700536D6F6F7468696E67005A0F
:10291000005A005900590058005800436F72726500
:102920006374696F6E00436F7272656374696F6E72
:10293000004D61696E0046696C616D656E740042A0
:1029400061636B6C6173680053746570732F6D6D98
:10295000004A65726B00416363656C6572617469FE
:102960006F6E0056656C6F6369747900436F6E66B5
:10297000696775726174696F6E0045737465707311
:102980002F6D6D004573746570732F6D6D005A73F4
:10299000746570732F6D6D005A73746570732F6D4D
:1029A0006D005973746570732F6D6D005973746584
:1029B00070732F6D6D005873746570732F6D6D009B
:1029C0005873746570732F6D6D00416476616E632A
:1029D00065642053657474696E67730056652D6A6B
:1029E00065726B0056652D6A65726B00567A2D6AAA
:1029F00065726B00567A2D6A65726B0056792D6A86
:102A000065726B0056792D6A65726B0056782D6A77
:102A100065726B0056782D6A65726B004164766151
:102A20006E6365642053657474696E677300416DED
:102A30006178204500416D6178204500416D6178E5
:102A4000205A00416D6178205A00416D617820590B
:102A500000416D6178205900416D61782058004136
:102A60006D6178205800412D74726176656C00416B
:102A70002D74726176656C00412D726574726163AC
:102A80007400412D72657472616374004163636503
:102A90006C00416363656C00416476616E636564DC
:102AA0002053657474696E677300565472617620A2
:102AB0006D696E005654726176206D696E00566DB8
:102AC000696E00566D696E00566D6178204500563E
:102AD0006D6178204500566D6178205A00566D6111
:102AE00078205A00566D6178205900566D61782023
:102AF0005900566D6178205800566D617820580055
:102B0000416476616E6365642053657474696E67B1
:102B100073004C6F6164206D6D004C6F6164206DBB
:102B20006D00556E6C6F6164206D6D00556E6C6F3D
:102B30006164206D6D00416476616E6365204B00B9
:102B4000416476616E6365204B00416476616E631B
:102B500065642053657474696E67730044697361BA
:102B6000626C65207374657070657273004D3834E3
:102B7000004175746F20686F6D6500473238004CF6
:102B80006576656C2058206178697300004D6F761A
:102B9000652061786973004D61696E0045787472D3
:102BA0007564657220004D6F7665205A004D6F7612
:102BB000652059004D6F76652058004D6F76656D24
:102BC000656E7400457874727564657220004D6F8F
:102BD000766520302E3032356D6D004D6F76652074
:102BE000302E316D6D004D6F766520316D6D004D6D
:102BF0006F76652031306D6D004D6F7665206178A0
:102C0000697300486F74656E6420746F6F20636F22
:102C10006C6400457874727564657220004D6F763F
:102C200065205A004D6F76652059004D6F766520FE
:102C300058004D6F7665205A004D6F76652059001B
:102C40004D6F76652058005761697420666F720079
:102C500066696C616D656E742070757267650000E1
:102C6000506C6561736520776169742E00507265E0
:102C7000737320627574746F6E00746F2072657365
:102C8000756D65207072696E740057616974206695
:102C90006F720066696C616D656E74206C6F616443
:102CA00000496E736572742066696C616D656E743F
:102CB00000616E6420707265737320627574746F46
:102CC0006E00746F20636F6E74696E75650050726C
:102CD00065737320627574746F6E00746F2068651D
:102CE0006174206E6F7A7A6C65004E6F7A7A6C65CB
:102CF0002068656174696E6700506C65617365205A
:102D0000776169742E2E2E005761697420666F7288
:102D10000066696C616D656E7420756E6C6F6164C0
:102D2000005761697420666F720066696C616D6539
:102D30006E74206368616E676500746F20737461E0
:102D40007274005061726B696E672E2E2E0043689C
:102D5000616E67696E672046696C616D656E7400AF
:102D6000554E4C4F41442046494C414D454E540030
:102D70004C4F41442046494C414D454E5400202083
:102D80004E6F7A7A6C653A20002000456E642066AA
:102D9000696C616D656E74206368616E6765005073
:102DA00075726765206D6F726500004368616E67BC
:102DB000652066696C616D656E7400556E6C6F613F
:102DC000642066696C616D656E74004C6F6164208F
:102DD00066696C616D656E74004D3630302042302E
:102DE00020542564004D373032203B2564004D3798
:102DF000303220542564004D373031205425640092
:102E00005072656865617420437573746F6D00500E
:102E100072656865617420437573746F6D005072DC
:102E20006568656174204142530050726568656150
:102E30007420504C41004261636B004E6F2053443C
:102E40002063617264005072696E742066726F6DE7
:102E5000205344004368616E6765205344206361DA
:102E60007264004D32310041626F75742050726996
:102E70006E746572004368616E67652066696C6197
:102E80006D656E74004368616E67652066696C618C
:102E90006D656E74004D36303020423000436F6EE9
:102EA00066696775726174696F6E0054656D7065EF
:102EB000726174757265004D6F76656D656E740034
:102EC000526573756D65207072696E740054756E0D
:102ED000650053746F70207072696E740050617574
:102EE0007365207072696E7400496E666F2073633B
:102EF0007265656E0053746F70004261636B0053BE
:102F0000746F70207072696E74003F0050726F624F
:102F100065205A204F66667365740042616279735A
:102F2000746570205900426162797374657020582D
:102F300000466C6F7700466C6F770046616E2073B9
:102F40007065656420310046616E2073706565644C
:102F500020310042656400426564004E6F7A7A6CED
:102F600065004E6F7A7A6C65005370656564005336
:102F700070656564004D61696E00426162797374C9
:102F80006570205900426162797374657020580041
:102F900047616D6573004669726D77617265205691
:102FA000657273696F6E004D61696E00436F6F6C7F
:102FB000646F776E0046616E2073706565642031C2
:102FC0000046616E2073706565642031004265645F
:102FD00000426564004E6F7A7A6C65004E6F7A7AB3
:102FE0006C65004D61696E006F6F6F0000001FC05F
:102FF0007FF0DDD8FFF87FF044402480000031806E
:10300000000024804440107CFEFEFE04000E000EF2
:10301000007FC0FFE0FFE0FFE0FFE006000F001FC1
:103020008036C03FC009001680294006000F001FEF
:103030008036C03FC0168020401080104008801F9E
:10304000C037607FF05FD050500D80104048905FD7
:10305000D077707FF01FC0104020200F007FE0FF6E
:10306000F0E670FFF0198036C0C0300F007FE0FF3F
:10307000F0E670FFF0198036C0198047414D4520B9
:103080004F56455200526573746F726520666169D0
:103090006C73616665004C6F61642073657474695C
:1030A0006E67730053746F72652073657474696E14
:1030B00067730050726F6265205A204F66667365B1
:1030C0007400416476616E6365642053657474694D
:1030D0006E6773004D61696E0050726F6265205AB1
:1030E000204F6666736574004D6F76696E672E2E8D
:1030F0002E004D3234004D323520500A4D3234000E
:103100005072696E742070617573656400506175EA
:103110007365207072696E74005072696E742061FC
:10312000626F72746564004C756C7A426F742054DF
:10313000415A20362072656164792E005072696EA2
:1031400074696E672E2E2E005072696E7420706145
:103150007573656400436172642072656D6F766596
:1031600064004361726420696E7365727465640003
:103170004D313137004D33310043616E6E6F742035
:10318000656E746572207375626469723A20002EF0
:103190000A006F70656E206661696C65642C20465C
:1031A000696C653A20006175746F25632E67006550
:1031B00072726F722077726974696E6720746F2003
:1031C00066696C650A004E6F742053442070726902
:1031D0006E74696E670A005344207072696E746978
:1031E0006E67206279746520002E0A0044656C6564
:1031F00074696F6E206661696C65642C2046696C29
:10320000653A200046696C652064656C6574656488
:103210003A0057726974696E6720746F2066696C32
:10322000653A20002E0A006F70656E206661696C39
:1032300065642C2046696C653A20002E0A006F7088
:10324000656E206661696C65642C2046696C653A20
:10325000200046696C652073656C65637465640A5B
:10326000002053697A653A200046696C65206F70CA
:10327000656E65643A20002066696C653A200066D8
:103280007265736800646F696E67004E6F77200027
:10329000454E4420535542524F5554494E450A001D
:1032A0002220706F73002220706172656E743A2262
:1032B00000535542524F5554494E452043414C4CC2
:1032C000207461726765743A2200747279696E675E
:1032D00020746F2063616C6C207375622D67636F5F
:1032E00064652066696C6573207769746820746F03
:1032F0006F206D616E79206C6576656C732E204D44
:103300004158206C6576656C2069733A310A004D2E
:103310003234004D323320257300534420636172F0
:1033200064206F6B0A006F70656E526F6F74206659
:1033300061696C65640A00766F6C756D652E696EE7
:103340006974206661696C65640A00534420696E83
:103350006974206661696C0A00286E6F2066696C6A
:1033600065290043616E6E6F74206F70656E207307
:10337000756264697220007C3C3E5E2B3D3F2F5B92
:103380005D3B2C2A225C004F4646004F4E00656391
:10339000686F3A004572726F723A004572726F72CE
:1033A0002077726974696E6720746F2045455052AA
:1033B0004F4D210A00507265737320627574746FEB
:1033C0006E20286F72204D3130382920746F2068AC
:1033D000656174206E6F7A7A6C650A00507265734D
:1033E0007320627574746F6E20286F72204D3130B7
:1033F000382920746F20726573756D650A00496EF7
:10340000736572742066696C616D656E7420616E9F
:103410006420707265737320627574746F6E2028F7
:103420006F72204D313038290A004D3630303A2045
:10343000546F6F20636F6C6400486F74656E642016
:10344000746F6F20636F6C640A00486F74656E64FC
:1034500020746F6F20636F6C640A00496E7365722D
:10346000742066696C616D656E7420616E64207095
:103470007265737320627574746F6E20286F72208A
:103480004D313038290A0063616E63656C007265E6
:1034900073756D656400726573756D650070617537
:1034A00073656400706F7765726F6666002F2F61B9
:1034B0006374696F6E3A0020573A0020573A00480B
:1034C0006F74656E6420436F6F6C696E672E2E2E6D
:1034D00000486F74656E642048656174696E672E7C
:1034E0002E2E00202F002042403A0020403A004D6E
:1034F000383420582059205A204500546865726D90
:10350000616C2052756E6177617900486F74656EE9
:103510006420544845524D414C2052554E4157412C
:10352000590042454420544845524D414C20525583
:103530004E4157415900202D20496E76616C6964D7
:10354000206578747275646572206E756D6265723F
:1035500020210A0048656174696E67206661696CA4
:103560006564004265642068656174696E67206601
:1035700061696C656400546865726D616C20527598
:103580006E617761790042454420544845524D416F
:103590004C2052554E415741590048656174696E3F
:1035A00067206661696C656400486F74656E6420AD
:1035B00048656174696E67206661696C6564005472
:1035C0006865726D616C2052756E61776179004833
:1035D0006F74656E6420544845524D414C205255DD
:1035E0004E41574159004D494E54454D502074723B
:1035F0006967676572656400486F74656E6420452D
:1036000072723A204D494E54454D50004572723AFF
:10361000204D494E54454D5020424544004D41589F
:1036200054454D502074726967676572656400483F
:103630006F74656E64204572723A204D415854454E
:103640004D50004572723A204D415854454D50201E
:1036500042454400626564002C2073797374656D83
:103660002073746F707065642120486561746572A1
:103670005F49443A200023646566696E65204445CD
:103680004641554C545F004B6420004B6920004B71
:103690007020000062656400504944204175746FD9
:1036A00074756E652066696E697368656421205063
:1036B000757420746865206C617374204B702C20C5
:1036C0004B6920616E64204B6420636F6E7374617C
:1036D0006E74732066726F6D2062656C6F772069FF
:1036E0006E746F20436F6E66696775726174696F7F
:1036F0006E2E680A00504944204175746F74756ECF
:1037000065206661696C6564212074696D656F75FB
:10371000740A00546865726D616C2052756E617731
:10372000617900486F74656E6420544845524D417C
:103730004C2052554E41574159004245442054486F
:1037400045524D414C2052554E4157415900486514
:103750006174696E67206661696C656400486F74A6
:10376000656E642048656174696E67206661696C86
:103770006564004265642068656174696E672066EF
:1037800061696C656400504944204175746F7475BB
:103790006E65206661696C6564212054656D706595
:1037A00072617475726520746F6F20686967680A4A
:1037B00000204B643A2000204B693A2000204B70D7
:1037C0003A20000A20436C617373696320504944B6
:1037D000200A002054753A2000204B753A20002022
:1037E0006D61783A2000206D696E3A200020643ABD
:1037F000200020626961733A2000504944204175DD
:10380000746F74756E652073746172740A00504928
:1038100044204175746F74756E65206661696C65CE
:1038200064212054656D70657261747572652074D1
:103830006F6F20686967680A001000AD0330016A85
:103840000150022B0170030A019004F500B005E558
:1038500000D006D800F007CE001009C500300ABE1F
:1038600000500BB700700CB100900DAB00B00EA66D
:1038700000D00FA200F0109D001012990030139597
:10388000005014920070158E0090168B00B01787B0
:1038900000D0188400F0198100101B7E00301C7BC2
:1038A00000501D7900701E7600901F7300B02070CC
:1038B00000D0216E00F0226B0010246900302566D4
:1038C00000502663007027610090285E00B0295CDC
:1038D00000D02A5900F02B5600102D5400302E51E4
:1038E00000502F4E0070304B0090314800B03245F0
:1038F00000D0334200F0343E0010363B0030373702
:10390000005038330070392E00903A2900B03B2324
:1039100000D03C1B00F03D1100103F0100F03F00C3
:10392000001000C90210012C014001220170011891
:1039300001B0010E01F00104015002FA00B002F0E2
:10394000003003E600D003DC009004D2007005C80C
:1039500000A006BE000008B400B009AA00D00BA069
:1039600000600E960060118C00001582002019780E
:1039700000C01D6E00A0226400B0275A00902C5099
:103980000000314600E0343C0010383200903A2804
:1039900000603C1E00A03D1400803E0A00203F0055
:1039A000006F70656E0054524947474552454400C8
:1039B0003A20007A5F70726F6265007A5F6D696E9F
:1039C00000795F6D617800795F6D696E00785F6D79
:1039D000617800785F6D696E005265706F7274690E
:1039E0006E6720656E6473746F7020737461747594
:1039F000730A00456E6473746F707320256320250D
:103A0000632025632025630020503A00205A3A00A5
:103A100020593A0020583A00656E6473746F7073D1
:103A2000206869743A2000486F6D696E672066618E
:103A3000696C656400496E76616C696420657874B0
:103A400072756465720A0045313A200045303A20AB
:103A5000005A3A2000593A20004D53312C4D533230
:103A60002C4D53332050696E730A583A20004D692B
:103A700063726F737465707320756E617661696CC3
:103A800061626C650A00205A3A0020593A002043CE
:103A90006F756E7420583A00C23100001C26000079
:103AA000F4190000D80F0000EB080000C00400006B
:103AB000750200004001000024F4D43050C38E2071
:103AC000C2A24017828B7011127A910D816CD90AB3
:103AD000A861E108C7586607615143061E4B5D05A2
:103AE000C145A7041A411104093D980371393103F6
:103AF0004036DB0265339102D4305402802E1D0221
:103B0000632CEE01752AC501B028A00110278101A0
:103B10008F2564012B244B01E0223401AC211F01CD
:103B20008D200D01801FFC00841EED00971DDF001D
:103B3000B81CD200E61BC600201BBC00641AB200F1
:103B4000B219A8000A19A0006A189900D1179100AB
:103B500040178B00B516840031167E00B31579002E
:103B60003A157300C7146F0058146A00EE1366000C
:103B70008813630025135E00C7125B006C125700A8
:103B800015125400C111510070114F0021114B004A
:103B9000D61049008D104700461044000210420024
:103BA000C00F4000800F3E00420F3C00060F3B005C
:103BB000CB0E3800930E37005C0E3500270E340014
:103BC000F30D3200C10D3100900D3000600D2E005C
:103BD000320D2D00050D2C00D90C2B00AE0C290048
:103BE000850C29005C0C2700350C27000E0C2600E4
:103BF000E80B2400C40B2400A00B23007D0B230042
:103C00005A0B2100390B2100180B2000F80A1F0065
:103C1000D90A1E00BB0A1E009D0A1D00800A1D0055
:103C2000630A1C00470A1B002C0A1B00110A1A0019
:103C3000F7091A00DD091900C4091900AB091900B8
:103C4000920917007B091800630917004C09160038
:103C500036091600200916000A091500F508150096
:103C6000E0081400CC081400B8081400A4081400DC
:103C7000900813007D0812006B081300580812000A
:103C80004608120034081100230811001208110020
:103C900001081100F0071000E0071000D007100025
:103CA000C0071000B0070F00A107100091070E0019
:103CB00083070F0074070F0065070E0057070E00FB
:103CC00049070E003B070D002E070E0020070D00D0
:103CD00013070D0006070D00F9060C00ED060D0098
:103CE000E0060C00D4060C00C8060C00BC060C0054
:103CF000B0060C00A4060B0099060C008D060B0004
:103D000082060B0077060B006C060B0061060A00AA
:103D100057060B004C060A0042060A0038060A0045
:103D20002E060A0024060A001A060A0010060900D8
:103D300007060A00FD050900F4050900EB05090066
:103D4000E2050900D9050900D0050900C7050900E9
:103D5000BE050900B5050800AD050800A505090068
:103D60009C050800940508008C05080084050800DF
:103D70007C050800740508006C050700650508004F
:103D80005D050700560508004E05070047050700BA
:103D90004005080038050700310507002A0507001F
:103DA000230507001C050600160507000F05070080
:103DB0000805060002050700FB040600F5040700DD
:103DC000EE040600E8040600E2040700DB04060037
:103DD000D5040600CF040600C9040600C30406008B
:103DE000BD040600B7040600B1040500AC040600DB
:103DF000A6040600A00405009B0406009504050027
:103E0000900406008A04050085040500800406006D
:103E10007A04050075040500700405006B040500B4
:103E200066040500610405005C04050057040500F4
:103E3000520405004D040500480405004304050034
:103E40003E0404003A040500350405003004040073
:103E50002C04050027040400230405001E040400AC
:103E60001A04040016040500110404000D040400E3
:103E7000090405000404040000040400FC03040019
:103E8000F8030400F4030400F0030400EC0304004E
:103E9000E8030400E4030400E0030400DC0304007E
:103EA000D8030400D4030400D0030400CC030400AE
:103EB000C8030300C503030024F404D9201BC40C69
:103EC0005C0E9804C4095F0265077101F405F900EE
:103ED000FB04B30048048700C10369005803550080
:103EE00003034500BE023A008402310053022A0057
:103EF0002902250004022000E4011C00C801190069
:103F0000AF01170098011400840113007101100023
:103F10006101100051010E0043010D0036010B003C
:103F20002B010B0020010B00150109000C010900F9
:103F300003010800FB000800F3000800EB00070085
:103F4000E4000600DE000600D8000600D2000600ED
:103F5000CC000500C7000500C2000500BD0004003C
:103F6000B9000400B5000400B1000400AD00040075
:103F7000A9000400A5000300A20003009F000400A4
:103F80009B000300980003009500020093000300CB
:103F9000900003008D0002008B00030088000200E7
:103FA0008600020084000300810002007F000200FE
:103FB0007D0002007B000200790002007700010012
:103FC000760002007400020072000100710002001D
:103FD0006F0002006D0001006C0002006A00010029
:103FE0006900020067000100660001006500010031
:103FF0006400020062000100610001006000010035
:104000005F0002005D0001005C0001005B00010038
:104010005A0001005900010058000100570001003A
:10402000560001005500010054000100530000003B
:104030005300010052000100510001005000010036
:104040004F0001004E0000004E0001004D00010035
:104050004C0001004B0000004B0001004A00010031
:10406000490001004800000048000100470001002D
:104070004600000046000100450000004500010028
:104080004400010043000000430001004200000022
:104090004200010041000000410001004000010019
:1040A0003F0000003F0001003E0000003E00010014
:1040B0003D0000003D0001003C0000003C0000000D
:1040C0003C0001003B0000003B0001003A00000002
:1040D0003A000100390000003900010038000000FA
:1040E00038000000380001003700000037000100F0
:1040F00036000000360000003600010035000000E8
:1041000035000000350001003400000034000000DC
:1041100034000100330000003300000033000100D0
:1041200032000000320000003200010031000000C7
:1041300031000000310001003000000030000000BC
:10414000300001002F0000002F0000002F000000B1
:104150002F0001002E0000002E0000002E000100A4
:104160002D0000002D0000002D0000002D0001009A
:104170002C0000002C0000002C0000002C0001008E
:104180002B0000002B0000002B0000002B00010082
:104190002A0000002A0000002A0000002A00010076
:1041A000290000002900000029000000290000006B
:1041B000290001002800000028000000280000005D
:1041C0002800000028000100270000002700000050
:1041D0002700000027000000270001002600000043
:1041E0002600000026000000260000002600010036
:1041F000250000002500000025000000250000002B
:10420000250000002500010024000000240000001B
:10421000240000002400000024000100230000000E
:104220002300000023000000230000002300000002
:1042300023000000230001002200000022000000F3
:1042400022000000220000002200000022000100E5
:1042500021000000210000002100000021000000DA
:1042600021000000210000002100010020000000CA
:1042700020000000200000002000000020000000BE
:104280002000000020000000200001001F000000AE
:104290001F0000001F0000001F0000001F000000A2
:1042A0001F0000001F0001001E0000001E00000093
:1042B0001E0000001E00000020204D36303320007C
:1042C0003A0A0020286D6D2900205300205A002052
:1042D000590020580020204D3432352046004261DC
:1042E000636B6C61736820636F6D70656E7361746E
:1042F000696F6E3A0A002055004C0046696C616D8A
:10430000656E74206C6F61642F756E6C6F616420D4
:104310006C656E677468733A0A0020204D3930303E
:10432000204B004C696E65617220416476616E635A
:10433000653A0A0020204D383531205A005A2D5058
:10434000726F6265204F66667365740020440020BA
:10435000490020204D3330342050002044002049B3
:104360000020204D333031205000504944207365E7
:104370007474696E67733A0A002046002042002078
:10438000480020204D3134352053004D6174657252
:1043900069616C2068656174757020706172616D0F
:1043A00065746572733A0A0020204D343230205310
:1043B000004175746F20426564204C6576656C69B8
:1043C0006E673A0A00204500205A00205900205804
:1043D0000020540020530020204D32303520420070
:1043E00020453C6D61785F655F6A65726B3E0020B9
:1043F000583C6D61785F785F6A65726B3E20593C0E
:104400006D61785F795F6A65726B3E205A3C6D61C1
:10441000785F7A5F6A65726B3E00416476616E63B5
:1044200065643A20423C6D696E5F7365676D656EC9
:10443000745F74696D655F75733E20533C6D696E82
:104440005F66656564726174653E20543C6D696E9B
:104450005F74726176656C5F6665656472617465D0
:104460003E0020540020520020204D323034205095
:1044700000416363656C65726174696F6E202875B5
:104480006E6974732F7332293A20503C7072696ED2
:10449000745F616363656C3E20523C726574726147
:1044A00063745F616363656C3E20543C7472617633
:1044B000656C5F616363656C3E0A00204500205AAD
:1044C0000020590020204D3230312058004D6178B5
:1044D000696D756D20416363656C65726174696FA8
:1044E0006E2028756E6974732F7332293A0A002082
:1044F0004500205A0020590020204D3230332058EA
:10450000004D6178696D756D2066656564726174D2
:1045100065732028756E6974732F73293A0A0053E6
:10452000746570732070657220756E69743A0A0044
:1045300020204D3134392043203B20556E6974735F
:1045400020696E2043656C736975730A00202047EB
:104550003231202020203B20556E69747320696E13
:10456000206D6D0048617264636F6465642044650A
:104570006661756C742053657474696E6773204C42
:104580006F616465640A002823000028230000642A
:10459000000000282300000000964300009643001E
:1045A0000040400000C8410000C9420000C942006C
:1045B00000C84400804F44454550524F4D20496E3D
:1045C000697469616C697A65640A00290A0020626D
:1045D000797465733B2063726320002073746F727B
:1045E00065642073657474696E6773207265747294
:1045F0006965766564202800202863616C63756CAA
:104600006174656429210A0020213D200045455040
:10461000524F4D20435243206D69736D617463683E
:10462000202D202873746F7265642920002053693F
:104630007A653A2000496E6465783A2000204D6121
:10464000726C696E3D563638290A00454550524F06
:104650004D2076657273696F6E206D69736D61743C
:1046600063682028454550524F4D3D00290A0020DF
:1046700062797465733B20637263200053657474C0
:10468000696E67732053746F7265642028000A0096
:104690003B20454550524F4D20496E6465783A2085
:1046A000005570646174696E67207A6F6666736521
:1046B0007420696E20454550524F4D3A20004545C3
:1046C00050524F4D206461746173697A6520657240
:1046D000726F722E0A004175746F6C6576656C207E
:1046E0006661696C65640A004175746F6C65766516
:1046F0006C206661696C6564005761726E696E67F3
:104700003A20486F6D696E672042756D702044696C
:104710007669736F72203C20310A00020204486FF0
:104720006D65202573257325732066697273740087
:104730002066697273740A00486F6D6520002074EA
:104740006F6F206C6F6E6720657874727573696F18
:104750006E2070726576656E7465640A0020636F02
:104760006C6420657874727573696F6E2070726501
:1047700076656E7465640A0020453A00205A3A0056
:1047800020593A00583A00000048420000484200D0
:10479000004040FF01FF0000A0400000A0400000DA
:1047A000004000809D430000A143000087430000BB
:1047B000D8C10000974300000000000090430000B3
:1047C0009743000087430000D8C10000A0C100004B
:1047D000000020746F6F206C6F6E672065787472B4
:1047E0007573696F6E2070726576656E7465640AA4
:1047F0000020636F6C6420657874727573696F6EE6
:104800002070726576656E7465640A0062757379EE
:104810003A2070617573656420666F7220696E70EE
:1048200075740A00627573793A20706175736564F6
:1048300020666F7220757365720A00627573793A2B
:104840002070726F63657373696E670A004D313152
:10485000372050726F62652073756363657373668A
:10486000756C0A0020496E76616C69642065787405
:1048700072756465722000205A3A200020593A204F
:104880000042656420583A200050726F6265205AD9
:10489000204F66667365743A20003F5A206F757426
:1048A000206F662072616E676520282D3220746F3C
:1048B0002035290A004D31343520533C696E64653A
:1048C000783E206F7574206F662072616E67652078
:1048D00028302D31290A00436C69636B20746F20E6
:1048E000726573756D652E2E2E00220A00556E6B53
:1048F0006E6F776E20636F6D6D616E643A2022007B
:10490000454550524F4D204F4B0A004E6F206D6F62
:1049100076652E004543484F00494E464F004552AC
:10492000524F52530044525952554E00434F4D4D31
:10493000554E49434154494F4E006F666600144935
:1049400019491E4925492C4944454255473A004CCE
:10495000756C7A426F742054415A2036204F464677
:104960002E00205A00205900580020204D61783A2E
:104970002000205A00205900580020204D696E3A2E
:104980002000536F667420656E6473746F70733AA1
:1049900020002569730025696D202569730025694C
:1049A000682025696D2025697300256964202569C3
:1049B000682025696D20256973002569792025699E
:1049C00064202569682025696D202569730050726F
:1049D000696E742074696D653A20004D3131332061
:1049E00053002F2F20004361703A004348414D424D
:1049F00045525F54454D5045524154555245004D26
:104A00004F54494F4E5F4D4F444553005448455213
:104A10004D414C5F50524F54454354494F4E004115
:104A200055544F5245504F52545F53445F53544175
:104A30005455530050524F4D50545F535550504FA2
:104A4000525400454D455247454E43595F504152DF
:104A500053455200434153455F4C494748545F42D8
:104A600052494748544E45535300544F47474C45CD
:104A70005F4C494748545300534F465457415245A1
:104A80005F504F574552004255494C445F50455284
:104A900043454E54004C4556454C494E475F4441B2
:104AA0005441005A5F50524F4245004155544F4CBB
:104AB0004556454C005052494E545F4A4F420050B3
:104AC000524F4752455353004155544F5245504F52
:104AD00052545F54454D5000564F4C554D4554521D
:104AE000494300454550524F4D0042494E415259AD
:104AF0005F46494C455F5452414E53464552005320
:104B0000455249414C5F584F4E5F584F464600460C
:104B100049524D574152455F4E414D453A4D6172A4
:104B20006C696E20204649524D574152455F5645AB
:104B30005253494F4E3A322E302E302E31343520DA
:104B400045585452554445525F545950453A466C65
:104B50006578797374727564657220534F5552434A
:104B6000455F434F44455F55524C3A6874747073C7
:104B70003A2F2F636F64652E616C6570686F626A8F
:104B8000656374732E636F6D2F64696666757369F0
:104B90006F6E2F4D41524C494E2050524F544F434F
:104BA0004F4C5F56455253494F4E3A312E30204DAF
:104BB000414348494E455F545950453A4C756C7ACB
:104BC000426F742054415A2036204558545255445F
:104BD00045525F434F554E543A3120555549443A5A
:104BE00038343566303033632D616562642D346549
:104BF00035332D613662392D376430393834666487
:104C0000653630390A002020536D6F6F7468696E05
:104C10006720286D6D293A20202020202020202088
:104C20002020202020202020530020204261636B80
:104C30006C6173682044697374616E636520286DCC
:104C40006D293A20202020202020200020284631D5
:104C50002E30203D2066756C6C2C2046302E302086
:104C60003D206E6F6E65290A002020436F727265C9
:104C70006374696F6E20416D6F756E742F46616449
:104C8000652D6F75743A20202020204600616374E2
:104C90006976653A0A00696E004261636B6C617304
:104CA0006820436F7272656374696F6E2000486F8D
:104CB0006D652058592066697273740A00486F6DDB
:104CC0006520585920666972737400426564204CEF
:104CD0006576656C696E6720004661696C65642065
:104CE000746F20656E61626C6520426564204C655E
:104CF00076656C696E670A00426564204C6576656E
:104D00006C20436F7272656374696F6E204D6174BD
:104D10007269783A000A0A426564204C6576656CCF
:104D200020436F7272656374696F6E204D61747297
:104D300069783A00202B000A436F727265637465CC
:104D40006420426564204865696768742076732E24
:104D50002042656420546F706F6C6F67793A0A0067
:104D6000202B000A426564204865696768742054F6
:104D70006F706F6772617068793A0A2020202B2D5E
:104D80002D2D204241434B202D2D2B0A2020207C0D
:104D900020202020202020202020207C0A204C20A1
:104DA0007C20202020282B29202020207C20520A13
:104DB0002045207C20202020202020202020207C16
:104DC00020490A2046207C20282D29204E20282BEF
:104DD00029207C20470A2054207C202020202020CD
:104DE00020202020207C20480A2020207C202020F9
:104DF00020282D29202020207C20540A2020207CBF
:104E000020202020202020202020207C0A2020205C
:104E10004F2D2D2046524F4E54202D2D2B0A202849
:104E2000302C30290A003474682070726F6265205B
:104E3000706F696E742C2064697374616E63652091
:104E400066726F6D20706C616E653A200020284498
:104E5000525952554E2900473239204175746F20FE
:104E6000426564204C6576656C696E67003F20285A
:104E70004C2C522C462C4229206F7574206F6620D2
:104E8000626F756E64732E0A003F50726F62652008
:104E9000706F696E74732028592920697320696DB9
:104EA000706C61757369626C652028322D32292E11
:104EB0000A003F50726F626520706F696E747320D4
:104EC00028582920697320696D706C617573696257
:104ED0006C652028322D32292E0A003F285629657C
:104EE00072626F7365206C6576656C2069732069EA
:104EF0006D706C61757369626C652028302D342982
:104F00002E0A0043757272656E742066696C653A8C
:104F10002000456E642066696C65206C6973740AB4
:104F200000426567696E2066696C65206C69737400
:104F30000A00416476616E6365204B3D003F4B2063
:104F400076616C7565206F7574206F662072616E76
:104F500067652028302D3130292E0A004D31313738
:104F600020486F7420456E642048656174696E67DF
:104F70002E2E2E0A4D31303420533137302054300C
:104F80000A473238204F310A473120593235205AEA
:104F900031302046353030300A4D313137205265BE
:104FA000776970696E67206E6F7A7A6C650A543023
:104FB0000A473120582D31372059323520463530B7
:104FC00030300A4D31303920523137302054300AD8
:104FD0004731205A310A473120582D313720593274
:104FE000352046343030300A473120582D313720B3
:104FF0005939352046343030300A473120582D3168
:1050000037205932352046343030300A4731205865
:105010002D3137205939352046343030300A473168
:1050200020582D3137205932352046343030300A5F
:10503000473120582D31372059393520463430300A
:10504000300A473120582D31372059323520463427
:105050003030300A473120582D313720593935202A
:1050600046343030300A473120582D3137205932FC
:10507000352046343030300A473120582D31372022
:105080005939352046343030300A473120582D31D7
:1050900037205932352046343030300A47312058D5
:1050A0002D3137205939352046343030300A4731D8
:1050B000205A31350A4D3130362053323535200AE9
:1050C00047302058302059300A4D31303920523184
:1050D00036302054300A4D3130370A00473238001C
:1050E00020466C6F773A200020643A0020693A002D
:1050F00020703A00204500205A00205900204D39E8
:105100003220580043290A0061626C656420286DD2
:10511000696E2074656D70200064697300656E00AF
:10512000436F6C6420657874727564657320617276
:10513000652000205400205200416363656C657255
:105140006174696F6E3A205000496E76616C6964D3
:105150002065787472756465720A0020643A0020D4
:10516000693A0020703A00536C6565702E2E2E004F
:1051700047322F47332062616420706172616D6530
:10518000746572730A0050726F6265205A204F6610
:10519000667365743A2000446F6E652073617669AA
:1051A0006E672066696C652E0A0053442072656143
:1051B00064206572726F720A00446F6E65207072AF
:1051C000696E74696E672066696C650A004D3239D4
:1051D0000053544F505045442E20005072696E7455
:1051E00065722073746F70706564206475652074D7
:1051F0006F206572726F72732E2046697820746812
:1052000065206572726F7220616E6420757365200F
:105210004D39393920746F20726573746172742E40
:10522000202854656D7065726174757265206973AC
:105230002072657365742E20536574206974206133
:10524000667465722072657374617274696E672921
:105250000A004E6F20436865636B73756D20776934
:105260007468206C696E65206E756D6265722C20A5
:105270004C617374204C696E653A20004E6F204378
:105280006865636B73756D2077697468206C696EEF
:1052900065206E756D6265722C204C617374204CB4
:1052A000696E653A2000636865636B73756D206D88
:1052B00069736D617463682C204C617374204C6950
:1052C0006E653A20004C696E65204E756D626572A0
:1052D000206973206E6F74204C617374204C696E6A
:1052E00065204E756D6265722B312C204C61737494
:1052F000204C696E653A20004D31313000526573A3
:10530000656E643A20002042002050006F6B00223E
:105310000A00656E7175657565696E6720220050BB
:105320004944204175746F74756E65206661696CBF
:1053300065642120426164206578747275646572C9
:10534000206E756D6265720A0042656420636F6F3E
:105350006C696E672E2E2E0042656420686561744C
:10536000696E672E2E2E006F6B004739310A473069
:10537000205A313520463630300A4739300A473016
:1053800020583137302059323930204633303030D0
:105390000A4D313137205072696E742061626F722C
:1053A0007465642E002020506C616E6E65724275CB
:1053B0006666657242797465733A200020467265AC
:1053C00065204D656D6F72793A2000436F6D70698D
:1053D0006C65643A204A756C2031362032303139A0
:1053E0000A00207C20417574686F723A2028416C55
:1053F000657068204F626A6563747320496E632E1E
:105400002C204C756C7A426F742047697420526569
:10541000706F7369746F7279290A0000204C617390
:105420007420557064617465643A2000322E302E09
:10543000302E3134350A004D61726C696E00205394
:105440006F6674776172652052657365740A002017
:105450005761746368646F672052657365740A00EE
:105460002042726F776E206F757420526573657479
:105470000A002045787465726E616C205265736510
:10548000740A00506F77657255700A007374617208
:10549000740A004B494C4C45442E20005072696EF2
:1054A0007465722068616C7465642E206B696C6C25
:1054B00028292063616C6C6564210A004B494C4CBF
:1054C0002063617573656420627920746F6F206D4D
:1054D00075636820696E6163746976652074696DAF
:1054E00065202D2063757272656E7420636F6D6D1B
:1054F000616E643A20004730205A31300A47313219
:105500000A4D31303920523136300A4D3131372091
:1055100050726F62696E67206265640070726F62BC
:10552000655F726577697065004175746F6C65764B
:10553000656C206661696C6564004D3131372042CD
:105540006564206C6576656C696E67206661696C60
:1055500065642E0A4730205A31300A4730204530E2
:105560000A4D3330302050323520533838300A4D10
:10557000333030205035302053300A4D3330302016
:1055800050323520533838300A4D333030205035C2
:10559000302053300A4D33303020503235205338CC
:1055A00038300A47342053310070726F62655F668D
:1055B00061696C65640050726F7465637465642022
:1055C00050696E0A0025301D0C18282924311C0B47
:1055D000174527232F1B0A444316222B1A41420347
:1055E0003809FF360308060202000100C743FE80A7
:1055F000218BC0A05DBBB8F8E000E400E200E6004B
:10560000418B11241FBECFEFD1E2DEBFCDBF00E042
:105610000CBF14E0A0E0B2E0E2E7F9E902E00BBF62
:1056200002C007900D92A431B107D9F727E1A4E198
:10563000B4E001C01D92A535B207E1F71AE2C0E05F
:10564000DBE200E006C021970109802FFE010F94E4
:105650007344C63FD10780E00807A9F70E94AA3724
:105660000D94A74C0C9400001F920F920FB60F924E
:1056700011242F933F938F939F93AF93BF93809168
:10568000150490911604A0911704B091180430915C
:10569000140423E0230F2D3720F40196A11DB11D22
:1056A00005C026E8230F0296A11DB11D2093140406
:1056B0008093150490931604A0931704B0931804D4
:1056C0008091190490911A04A0911B04B0911C04BC
:1056D0000196A11DB11D8093190490931A04A09303
:1056E0001B04B0931C04BF91AF919F918F913F9188
:1056F0002F910F900FBE0F901F9018952FB7F89411
:10570000609115047091160480911704909118040B
:105710002FBF08953FB7F8948091190490911A040F
:10572000A0911B04B0911C0426B5A89B05C02F3F77
:1057300019F00196A11DB11D3FBFBA2FA92F982FB7
:105740008827820F911DA11DB11DBC01CD0142E032
:10575000660F771F881F991F4A95D1F708958F927A
:105760009F92AF92BF92CF92DF92EF92FF926B0126
:105770007C01D0DF4B015C01C114D104E104F104D0
:10578000F1F09CD3C7DFDC01CB0188199909AA0984
:10579000BB09883E9340A105B10570F321E0C21A10
:1057A000D108E108F10888EE880E83E0981EA11C5C
:1057B000B11CC114D104E104F10421F7DDCFFF9045
:1057C000EF90DF90CF90BF90AF909F908F90089513
:1057D0008230910538F0880F991F880F991F05971F
:1057E0000197F1F70895789484B5826084BD84B5FB
:1057F000816084BD85B5826085BD85B5816085BDCC
:10580000EEE6F0E0808181608083E1E8F0E01082E4
:10581000808182608083808181608083E0E8F0E025
:10582000808181608083E1EBF0E08081846080830F
:10583000E0EBF0E0808181608083E1E9F0E080814D
:1058400082608083808181608083E0E9F0E08081F4
:1058500081608083E1EAF0E08081826080838081E2
:1058600081608083E0EAF0E0808181608083E1E212
:10587000F1E0808182608083808181608083E0E2CA
:10588000F1E0808181608083EAE7F0E080818460DC
:105890008083808182608083808181608083808139
:1058A000806880831092C10008951F93CF93DF9387
:1058B000182FEB0161E016D1209711F460E004C0CD
:1058C000CF3FD10531F461E0812FDF91CF911F915E
:1058D00045C1E12FF0E0E55FFD4FE4914E2F50E030
:1058E000FA013197E231F10508F09DC08827EE58A2
:1058F000FF4F8F4F0D94734484B5806884BDC7BD3E
:1059000097C084B5806284BDC8BD92C0809180007C
:10591000806880938000D0938900C093880088C0FD
:1059200080918000806280938000D0938B00C09330
:105930008A007EC080918000886080938000D09330
:105940008D00C0938C0074C08091B00080688093FB
:10595000B000C093B3006CC08091B00080628093AF
:10596000B000C093B40064C08091900080688093C0
:105970009000D0939900C09398005AC080919000F5
:10598000806280939000D0939B00C0939A0050C097
:1059900080919000886080939000D0939D00C09388
:1059A0009C0046C08091A00080688093A0008091F8
:1059B000A0008F7B8093A000D093A900C093A80083
:1059C00037C08091A00080628093A000D093AB008C
:1059D000C093AA002DC08091A00088608093A00091
:1059E000D093AD00C093AC0023C0809120018068AB
:1059F00080932001D0932901C093280119C0809180
:105A00002001806280932001D0932B01C0932A0152
:105A10000FC080912001886080932001D0932D01D8
:105A2000C0932C0105C0C038D1050CF04CCF46CF37
:105A3000DF91CF911F91089590E0FC013197E23101
:105A4000F10508F04EC08827EC57FF4F8F4F0D949B
:105A50007344809180008F7703C0809180008F7D98
:105A600080938000089580918000877FF9CF84B56E
:105A70008F7702C084B58F7D84BD08958091B0007A
:105A80008F7703C08091B0008F7D8093B000089520
:105A9000809190008F7707C0809190008F7D03C028
:105AA00080919000877F8093900008958091A0005E
:105AB0008F7707C08091A0008F7D03C08091A000E8
:105AC000877F8093A0000895809120018F7707C081
:105AD000809120018F7D03C080912001877F80937A
:105AE00020010895CF93DF9390E0FC01EF5AFD4F22
:105AF0002491FC01E956FD4F8491882361F190E0E7
:105B0000880F991FFC01EF5EFC4FC591D491FC01F9
:105B1000E950FD4FA591B491611109C09FB7F89468
:105B20008881209582238883EC912E230BC06230DC
:105B300061F49FB7F8943881822F809583238883FE
:105B4000EC912E2B2C939FBF06C08FB7F894E88161
:105B50002E2B28838FBFDF91CF9108951F93CF9372
:105B6000DF93282F30E0F901E55FFD4F8491F901C3
:105B7000EF5AFD4FD491F901E956FD4FC491CC2362
:105B8000C1F0162F811158DFEC2FF0E0EE0FFF1F50
:105B9000E950FD4FA591B4918FB7F894111105C04C
:105BA0009C91ED2FE095E92302C0EC91ED2BEC9355
:105BB0008FBFDF91CF911F910895CF93DF93282F4F
:105BC00030E0F901E55FFD4F8491F901EF5AFD4F97
:105BD000D491F901E956FD4FC491CC2389F081118C
:105BE0002BDFEC2FF0E0EE0FFF1FE352FD4FA591EE
:105BF000B491EC91ED2381E090E021F480E002C0CB
:105C000080E090E0DF91CF91089508951F920F9268
:105C10000FB60F9211240BB60F922F933F934F9311
:105C20005F936F937F938F939F93AF93BF93EF9304
:105C3000FF93E0910802F09109021995FF91EF910D
:105C4000BF91AF919F918F917F916F915F914F9194
:105C50003F912F910F900BBE0F900FBE0F901F9092
:105C600018951F920F920FB60F9211240BB60F9238
:105C70002F933F934F935F936F937F938F939F9354
:105C8000AF93BF93EF93FF93E0910A02F0910B0261
:105C90001995FF91EF91BF91AF919F918F917F9156
:105CA0006F915F914F913F912F910F900BBE0F908D
:105CB0000FBE0F901F9018951F920F920FB60F9264
:105CC00011240BB60F922F933F934F935F936F93D3
:105CD0007F938F939F93AF93BF93EF93FF93E09145
:105CE0000C02F0910D021995FF91EF91BF91AF91C8
:105CF0009F918F917F916F915F914F913F912F91E4
:105D00000F900BBE0F900FBE0F901F9018951F9213
:105D10000F920FB60F9211240BB60F922F933F9351
:105D20004F935F936F937F938F939F93AF93BF93A3
:105D3000EF93FF93E0910E02F0910F021995FF91FE
:105D4000EF91BF91AF919F918F917F916F915F91F3
:105D50004F913F912F910F900BBE0F900FBE0F9060
:105D60001F9018951F920F920FB60F9211240BB629
:105D70000F922F933F934F935F936F937F938F93E4
:105D80009F93AF93BF93EF93FF93E0910402F09141
:105D900005021995FF91EF91BF91AF919F918F915E
:105DA0007F916F915F914F913F912F910F900BBE1B
:105DB0000F900FBE0F901F9018951F920F920FB665
:105DC0000F9211240BB60F922F933F934F935F9333
:105DD0006F937F938F939F93AF93BF93EF93FF93B3
:105DE000E0910602F09107021995FF91EF91BF91A2
:105DF000AF919F918F917F916F915F914F913F9163
:105E00002F910F900BBE0F900FBE0F901F90189503
:105E10001F920F920FB60F9211240BB60F922F9371
:105E20003F934F935F936F937F938F939F93AF9322
:105E3000BF93EF93FF93E0911002F0911102199537
:105E4000FF91EF91BF91AF919F918F917F916F9152
:105E50005F914F913F912F910F900BBE0F900FBE0E
:105E60000F901F9018951F920F920FB60F9211244A
:105E70000BB60F922F933F934F935F936F937F9344
:105E80008F939F93AF93BF93EF93FF93E091120291
:105E9000F09113021995FF91EF91BF91AF919F91EE
:105EA0008F917F916F915F914F913F912F910F90C3
:105EB0000BBE0F900FBE0F901F90189508951F9363
:105EC000CF93DF93EC011D821C821F821E821986F4
:105ED00081E0888782E28A871F861E86FE01B3964C
:105EE000CE01C1962FEF2193E817F907E1F711E0F2
:105EF00018A3CE0122D61F8B188E198E80E48A8FAC
:105F00001B8E8EE693E39AAB89ABDF91CF911F9105
:105F10000895DB01ED91FC911994EF92FF921F938C
:105F2000CF93DF931F921F92CDB7DEB77C01DC01C8
:105F3000D196ED91FC91D29782E069837A8319958D
:105F400020E030E04AE069817A81C701E2DF182F62
:105F5000D701D196ED91FC91D29783E01995D701A5
:105F6000D196ED91FC91D29780E01995812F0F90F9
:105F70000F90DF91CF911F91FF90EF9008950F93B5
:105F80001F93CF93DF93EC018B01E9A9FAA982E07B
:105F90001995E9A9FAA981E0199520E030E044E1DA
:105FA000B801CE01B6DF9E012D5C3F4F47E1B8013D
:105FB000CE01AFDFE9A9FAA980E0DF91CF911F916F
:105FC0000F911994EF92FF921F93CF93DF93EC01FF
:105FD0007B01E9A9FAA982E01995E9A9FAA981E06A
:105FE000199520E030E045E1B701CE0192DF182F8E
:105FF000882339F09E012D5C3F4F47E1B701CE0168
:1060000088DFE9A9FAA980E01995812FDF91CF9166
:106010001F91FF90EF900895FC01448F258F9C0104
:10602000245E3F4F42E375CFCF93DF931F92CDB7EE
:10603000DEB79E012F5F3F4F46E46BDF89810F90F3
:10604000DF91CF910895CF93DF931F92CDB7DEB745
:106050009E012F5F3F4F47E45CDF89810F90DF9106
:10606000CF91089520E030E048E453CFCF93DF9301
:10607000EC016A817B81D8DF88836A817B81CE01D4
:10608000E2DF89836A817B81CE01ECDF8B879E0111
:106090002D5C3F4F6A817B8147E1CE01DF91CF913B
:1060A00038CFCF93DF93EC016A817B8136DF882381
:1060B00019F0CE01DBDF81E0DF91CF9108958F925F
:1060C0009F92AF92BF92CF92EF920F93CF93DF93B5
:1060D0001F921F92CDB7DEB74C015B012A83498323
:1060E000EEDEF401B382A282498147A32A8120A770
:1060F00005A3E4A2C3A2C4010F900F90DF91CF913A
:106100000F91EF90CF90BF90AF909F908F90C9CF9D
:10611000FC016281738133CFCF93DF93EC01EE8575
:10612000FF85309709F019956A817B81CE01DF9157
:10613000CF9148CF362F242FFC0162817381432FEA
:106140006BCF0F93FC0182819381648F458F278FE2
:10615000068F9F01245E3F4F4BE3BC01CF010F919F
:10616000D8CEFC0160A30895BF92CF92DF92EF9248
:10617000FF920F931F93CF93DF936C01D62FB42E12
:10618000C22F7801CC2369F0F701049120E04B2D58
:106190006D2FC601D6DFFFEFEF1AFF0AC150D85F9F
:1061A000F1CFDF91CF911F910F91FF90EF90DF9092
:1061B000CF90BF9008958F929F92AF92BF92CF924F
:1061C000DF92EF92FF920F931F93CF93DF935C01C7
:1061D000C62EC42FD22ED02F220F220F220F1ED058
:1061E000882379F0DC0F8D2C912CCD1751F087018D
:1061F0002D2D4C2F6C2DC501B7DFE80CF91CCF5F9E
:10620000F4CFDF91CF911F910F91FF90EF90DF902E
:10621000CF90BF90AF909F908F9008950F93FC0107
:106220000150040F84A996A9941718F0081728F4B0
:1062300002C0081750F0041740F42150260F83A91C
:1062400095A9961720F4281720F480E007C0281796
:1062500020F481E0261710F0F8CF81E00F91089527
:1062600081E008952EE93FE0009729F0F901319788
:10627000F1F70197F9CF0895FC01128280818150D6
:10628000838314820895FC0180819281980F928308
:106290002181921760F494819F5F94839381890F89
:1062A000821710F08FEF820F838381E0089580E0E2
:1062B0000895FC0191E08381861708F490E031E0B5
:1062C000461708F030E0832F892B21E052814517D3
:1062D00008F420E02823832F8923822B0895DC01F2
:1062E000FB01108212968C911297818315968C91E6
:1062F00015978150828313968C9183830895FB01B7
:1063000041812381213029F0233031F468EF640F7B
:1063100004C0642F485F01C0642FCBCFDC01159609
:106320002C9115971696ED91FC911797CF01820F3E
:10633000911D820F911D1192E817F907E1F7089559
:10634000FC01A681B7818281481B8581483018F005
:10635000A80FB11D4770382F369536953695562FB4
:10636000577080E890E002C0959587955A95E2F7BE
:10637000439F402D1124669566956695E62FF0E0C3
:10638000E40FF11DEA0FFB1F3081222311F0832B54
:1063900002C08095832380830895FB014181DC0145
:1063A00012962C911297421760F013962C91139726
:1063B000241738F0608115962C91621710F424810F
:1063C000BFCF0895CF92DF92FF920F931F93CF9389
:1063D000DF936C01EB01FA809B81913051F030F03A
:1063E000923049F0933051F41FEF09C010E001E002
:1063F00007C011E004C010E00FEF02C010E000E0A1
:10640000F7FE03C0BE01C601C8DF9881900F9883D4
:106410009981910F9983FF0C99F7DF91CF911F918B
:106420000F91FF90DF90CF9008950F931F93CF931C
:10643000DF938901FB01C281D3814233D9F058F443
:106440004531E1F0473109F1443141F5CE0166DFD4
:10645000CE0112DF23C04634E1F04734E1F04B3384
:10646000E9F4B901CE014BDF8823C1F0B801CE01B8
:10647000A9DF14C0B901CE0190DF10C0CE0103DF47
:10648000882369F0CE014ADF09C0B901CE0127DFB8
:1064900005C08D8101C08981F801808381E0DF9191
:1064A000CF911F910F910895CF92DF92EF92FF92BB
:1064B0000F931F93CF93DF937C01D62FD42EC22F3F
:1064C000122FC62EC20E6C2D611B183038F00FEF44
:1064D00020E04D2DC70135DE1850F5CF6C2F687FB9
:1064E0006D0F2C2F277071F097E029272F5F2770F1
:1064F0000FEF10E001C0000F2A95EAF720E04D2DC4
:10650000C7011FDEDF91CF911F910F91FF90EF9098
:10651000DF90CF900895CF92DF92EF92FF920F938A
:106520001F93CF93DF937C01D62ED42FC22F122F2F
:10653000C42EC20E4C2D411B183038F00FEF21E055
:106540006D2DC701FEDD1850F5CF4C2F487F4D0F44
:106550002C2F277071F097E029272F5F27700FEFFE
:1065600010E001C0000F2A95EAF721E06D2DC70168
:10657000E8DDDF91CF911F910F91FF90EF90DF90B9
:10658000CF900895EF92FF920F931F93CF93DF93D5
:10659000EC01162FF42EE22E01E040DE882359F0A4
:1065A0002E2D4F2D612FCE01DF91CF911F910F9195
:1065B000FF90EF9079CFDF91CF911F910F91FF90D6
:1065C000EF900895EF92FF920F931F93CF93DF9375
:1065D000EC01162FF42EE22E022F21E01FDE88237D
:1065E00059F02E2D4F2D612FCE01DF91CF911F91AC
:1065F0000F91FF90EF908FCFDF91CF911F910F916F
:10660000FF90EF900895DF92EF92FF920F931F9308
:10661000CF93DF937C01162FC42FD22ED02FFEDD17
:106620008823F9F02D2D4C2F612FC7013DDF2D2F31
:106630004C2F612FC7016FDF6FEF6D0D610F2D2F95
:106640004C2FC70168DF4FEF4D0F4C0F2D2D612FE1
:10665000C701DF91CF911F910F91FF90EF90DF90D5
:1066600023CFDF91CF911F910F91FF90EF90DF909B
:106670000895EF92FF920F931F93CF93DF937C01C6
:10668000D62F122FC42F040F212F4C2F6D2FC7018F
:106690000BDFCF5F0C13F8CFDF91CF911F910F91DC
:1066A000FF90EF900895DF92EF92FF920F931F9368
:1066B000CF93DF93EC01162FF42EE22EAFDD88236B
:1066C00029F02E2D4F2D612FCE01D3DFDF91CF91F9
:1066D0001F910F91FF90EF90DF9008950895FC01B6
:1066E000E60FF11D849190E0982F88273196E49170
:1066F0008E0F911D0895FC0184910895FCDF88237D
:1067000021F0823011F083E0089586E0089580E062
:106710000895FC018081089566E0E1CF68E0DFCF55
:106720000A96FC01849108950B96FC0184910895CA
:10673000DC011496ED91FC911597319684910895A2
:10674000BF92CF92DF92EF92FF920F931F93CF935E
:10675000DF938C01E62EDC011496CD91DC91159728
:10676000CE01C9DFF82EF80184819581C7DFC82EDC
:10677000F1E0FF1203C02FE0B22E02C0BB24BA9496
:10678000D80114968D919C911597CADFF82EF801C7
:1067900084819581C9DFD82ED80114968D919C9162
:1067A0001597BCDFB0E6BE1538F4009729F0C80F86
:1067B000D91F91E6F92E0FC0F80184819581ACDFD5
:1067C000F0E4FE1538F4009729F0C80FD91F81E4D2
:1067D000F82E01C06196DE1490F4D80150961C92F8
:1067E000509753961C92539754961C9254975196D7
:1067F0001C92519752961C9280E090E066C0DF1484
:1068000060F38C2D90E0FE0124912F3F11F421962E
:1068100057C0FE104CC0D80114968D919C911597CD
:106820006ADF9E012F5F3F4FFE01882311F0823007
:10683000E1F48491D80153968C935397F9012491F4
:1068400054962C935497FE013396E4915096EC9312
:106850005097FE013496E4915196EC935197FE01C6
:106860003596E4915296EC9320C08491982F9F70B6
:106870009250D80152969C93529782958F70519660
:106880008C935197F9012491822F8F7054968C9399
:10689000549722952F7053962C935397FE0132965E
:1068A000E491E295EF705096EC93CE010EC0FE019C
:1068B0003296E491EB219C012E0F311DC20FD31FA4
:1068C000FD1409F48ACFF3949ECFDF91CF911F91ED
:1068D0000F91FF90EF90DF90CF90BF9008954F926F
:1068E0005F926F927F929F92AF92BF92CF92DF9210
:1068F000EF92FF920F931F93CF93DF931F92CDB729
:10690000DEB72C01C62E942E622F1ADF7C01892B54
:1069100009F43AC0F20184819581F0DEB82EF201CB
:10692000138904898189C80E8289981AD92CD01AB2
:10693000212F4D2D6C2DC20171DC882311F1EB0C40
:10694000F11C195F169516951695612E712CD914A8
:10695000C1F03C2D57018A2D8E19811770F4F50175
:10696000049120E04D2D632FC2013983EADBFFEF54
:10697000AF1ABF0A3981385FEECFE60CF71CD3940B
:10698000E6CFF201808901C080E00F90DF91CF91C6
:106990001F910F91FF90EF90DF90CF90BF90AF903D
:1069A0009F907F906F905F904F9008950F931F93EB
:1069B000CF93DF9300D0CDB7DEB78C01DC015596C5
:1069C000ED91FC9156972B834A83698319954A81EF
:1069D000480F2B816981C8010F900F900F90DF91B4
:1069E000CF911F910F917BCFAF92BF92DF92EF9229
:1069F000FF920F931F93CF93DF931F921F92CDB7F8
:106A0000DEB77C01D62E042FDC015596ED91FC916A
:106A1000569729833A831995080F2981A22E3A8126
:106A2000B32E10E0F50121915F01222339F0402FB0
:106A30006D2DC70154DFD80E180FF4CF812F0F90A2
:106A40000F90DF91CF911F910F91FF90EF90DF900A
:106A5000BF90AF900895DF92EF92FF920F931F9334
:106A6000CF93DF937C01D62FD42E8901DC0155967C
:106A7000ED91FC9156971995D80EC0E0F80124913C
:106A8000222349F04D2D6D2FC70129DFD80FC80FE4
:106A90000F5F1F4FF3CF8C2FDF91CF911F910F917D
:106AA000FF90EF90DF900895DC0114962D913C91BA
:106AB00015972115310509F43FC057968C915797CA
:106AC000F901811108C03596E4915896EC935897D6
:106AD000F9013C9611C0813041F43F96E4915896FB
:106AE000EC935897F901709607C03D96E49158963B
:106AF000EC935897F9013E96E4915996EC93599787
:106B000058968C915897082E000C990B59962C91F9
:106B10005997821B910927FD93955A962C915A9764
:106B2000203441F0829FC001112426E0969587957C
:106B30002A95E1F75B968C93089527E833E3FC01EF
:106B4000368B258B0895CF92DF92EF92FF920F93B1
:106B50001F93CF93DF938C017B016A01CB01FA0174
:106B60001995D82F882311F1682FC801E9DDF801A4
:106B7000C189C195FFEFEF1AFF0AC701F601199508
:106B8000F801882351F08089C80FC701F6011995D3
:106B9000D82F682FC801D4DDEDCFD03221F09189F4
:106BA0008389890F01C080898C0F01C080E0DF914B
:106BB000CF911F910F91FF90EF90DF90CF900895AC
:106BC00049E853E3C0CFCF93DF93FC0124813581A3
:106BD0002617370741F0EC017583648365DF87E88A
:106BE00093E39E8B8D8BDF91CF910895CF93DF93AD
:106BF00000D01F92CDB7DEB76115710581059105F3
:106C000079F09B01AC0169833A834B835C830F94D9
:106C1000E34429813A814B815C810F94574403C03E
:106C200060E070E0CB010F900F900F900F90DF911C
:106C3000CF910895CF92DF92EF92FF920F931F931F
:106C400062177307840795077CF489019A016B0129
:106C50007C01C901B8016C197D098E099F09C6DF45
:106C60006C0D7D1D8E1D9F1D1F910F91FF90EF904C
:106C7000DF90CF9008954F925F926F927F92AF9284
:106C8000BF92CF92DF92EF92FF920F931F93CF9319
:106C9000DF93CDB7DEB729013A019B01AC0124197E
:106CA0003509460957098A899B89AC89BD89BC0188
:106CB000CD016A197B098C099D090F94F343A80142
:106CC000970124193509460957090F945744CA01F9
:106CD000B9016A0D7B1D8C1D9D1DDF91CF911F9108
:106CE0000F91FF90EF90DF90CF90BF90AF907F908B
:106CF0006F905F904F90089580E090E00895089520
:106D0000CF92DF92EF92FF920F931F93CF93DF9377
:106D10006C017A018B01C0E0D0E0CE15DF0589F06F
:106D2000D8016D918D01D601ED91FC910190F0811A
:106D3000E02DC6011995892B11F47E0102C0219620
:106D4000ECCFC701DF91CF911F910F91FF90EF9092
:106D5000DF90CF9008956115710579F0FB010190E6
:106D60000020E9F73197AF01461B570BDC01ED918D
:106D7000FC910280F381E02D199480E090E0089569
:106D8000DC01ED91FC910190F081E02D19944F927E
:106D90005F926F927F92EF92FF920F931F93CF9328
:106DA000DF93CDB7DEB7A1970FB6F894DEBF0FBE65
:106DB000CDBF7C01FA01CB0119A2223008F42AE0F0
:106DC0008E010F5D1F4F422E512C612C712CBF0183
:106DD000A30192010F943544F901CA010150110930
:106DE0006A3014F4605D01C0695CD8016C93232B98
:106DF000242B252B61F7B801C701ADDFA1960FB693
:106E0000F894DEBF0FBECDBFDF91CF911F910F91E0
:106E1000FF90EF907F906F905F904F900895CF928A
:106E2000DF92EF92FF920F931F93CF93DF93EC01CA
:106E30006A017B012115310579F4E881F98101901E
:106E4000F081E02D642FDF91CF911F910F91FF9082
:106E5000EF90DF90CF9019942A303105D9F477FF65
:106E600018C06DE28DDF8C0144275527BA014C19FB
:106E70005D096E097F092AE0CE0189DF800F911F2D
:106E8000DF91CF911F910F91FF90EF90DF90CF9006
:106E900008952AE0B701A601CE01DF91CF911F919D
:106EA0000F91FF90EF90DF90CF9071CF9A01AB01DF
:106EB000770F660B770BB3CFCF93CFB7F894809152
:106EC0001D04811127C0ECECF2E08491E6E8F2E0C9
:106ED0009491E82FF0E0EE0FFF1FEF5EFC4FA591BD
:106EE000B491EC91E92321F461E085E30E94AE2D99
:106EF00061E085E30E94722D8CB580618CBD8CB5FC
:106F000080648CBD61E084E30E94722D61E083E3C4
:106F10000E94722D80911D048F5F80931D04CFBF4E
:106F2000CF910895CF92EF920F93FC0113AE14AE60
:106F300015AE0496C4D80F91EF90CF9008958EBDF2
:106F400000000DB407FEFDCF8EB5089580E090E0FF
:106F5000089508950E94F32BFCDF0F94573FC0E083
:106F6000D0E00F94E23F2097E1F30E940000F9CFB8
:106F7000EFE3F4E083AF64AF08954AE050E0BC0172
:106F80008FE394E093CFEF92FF920F931F93CF93F1
:106F9000DF937A016F3F71058105910509F048F48F
:106FA0008FE394E0EDDE83E494E0C2DB282F30E051
:106FB00014C0C0917A04D0917B044D2F50E0EC2F87
:106FC000F0E08B019C01BF0183E494E04CD6C80F34
:106FD000C0937A04D0937B049C01C901DF91CF91C7
:106FE0001F910F91FF90EF900895EF92FF920F93F2
:106FF0001F93CF93DF938B01CFE3D4E0FBACECACDA
:107000004E2D50E06F2D70E09C0183E494E083D618
:10701000F80EFBAEECAEDF91CF911F910F91FF9078
:10702000EF900895EF92FF920F931F93CF93DF930A
:107030008B01CFE3D4E0FBACECAC4E2D50E06F2DD8
:1070400070E09C0183E494E0B2D6F80EFBAEECAEA7
:10705000DF91CF911F910F91FF90EF9008956FEF07
:107060007FEFC3CF4FEF5FEF8ECF0F931F93CF9381
:10707000DF931F92CDB7DEB7082F83ED96E00E9415
:107080007C79182F863168F483ED96E0E8DF1531BE
:1070900009F43DC060E270E080E090E0E3DF1F5F54
:1070A000F6CFCE0101960E941E7D60E870E09DDF64
:1070B0008981853120F56EE270E080E090E0D2DFDA
:1070C00019811431E1F06EE270E080E090E0CADFF7
:1070D0001331A9F089812EEF3FEF281B310986E09B
:1070E000829FB001839F700D112460587F4F83ED04
:1070F00096E07BDF60E270E080E090E0B3DF8091BB
:107100001E04801721F000931E040E94007D0F9042
:10711000DF91CF911F910F9108954F925F926F92DF
:107120007F928F929F92AF92BF92CF92DF92EF9217
:10713000FF920F931F93CF93DF93CDB7DEB72D97B9
:107140000FB6F894DEBF0FBECDBF8091C90688236D
:1071500009F48AC06091310D7091320D072E000C38
:10716000880B990B0F948D4111E020912D0D3091DA
:107170002E0D40912F0D5091300D0F94EE421816A8
:107180000CF010E060910B0D70910C0D072E000CAF
:10719000880B990B0F948D412091070D3091080DAC
:1071A0004091090D50910A0D0F94EE4218160CF4FF
:1071B000106810933104C0906A02D0906B02E09086
:1071C0006C02F0906D0220E030E0A901C701B60129
:1071D0000F94EB4087FD05C020E030E040E05FE326
:1071E00004C020E030E040E05FEBC701B6010F943F
:1071F00012400F945A41CB010F94E634BC018CE24B
:1072000094E00F945E49C0906E02D0906F02E090BF
:107210007002F090710220E030E0A901C701B601D0
:107220000F94EB4087FD05C020E030E040E05FE3D5
:1072300004C020E030E040E05FEBC701B6010F94EE
:1072400012400F945A41CB010F94E634BC0187E2FF
:1072500094E00F945E4982E792E00F94F739BC0105
:107260008FE194E00F945E490E94BB7B182F81E070
:107270005FD62091310427FF03C048E00CE002C034
:1072800042E102E08091770490E044977CF48091A1
:107290007904841758F027FD37C180E596E17C0119
:1072A00023E060E583E494E00E94DB308091770482
:1072B0008431B8F480917904823098F0112309F474
:1072C00026C18091270D882309F421C180EC95E126
:1072D0007C0102E123E042E068E683E494E00E945E
:1072E000DB30809177048C31D0F59091310480901F
:1072F0002D0D90902E0DA0902F0DB090300DC090C0
:10730000310DD090320D843128F480917904883089
:1073100008F03AC280917704883008F415C2809151
:1073200077048C3108F417C28090070D9090080DF7
:10733000A090090DB0900A0D80910B0D90910C0D4D
:1073400020917704283008F40CC2809177048C31A6
:1073500008F40EC2809177048C3108F40FC280913A
:10736000AD0983FF27C08091DD07882319F1809143
:1073700077048433F8F4809179048A32D8F007E0F6
:1073800028E04AE26AE283E494E08DD905E022E055
:107390004CE262E383E494E086D904E02AE041E32E
:1073A0006AE283E494E02FD94BE262E383E494E061
:1073B0000E949A3080917704853328F48091790473
:1073C000813308F0A7C00E94CD80823048F09091B0
:1073D0007704943328F490917904923308F0A2C092
:1073E000809177048F3208F05EC0809179048832F2
:1073F00008F459C00F94AC3B2B013C018CE3C82E20
:10740000D12CE12CF12CC301B201A70196010F94FC
:107410003544CA01B901A70196010F943544CA0148
:10742000062FD72E5901AE014F5F5F4F7A0150E80A
:10743000451651E5550651E06506710408F48CC007
:10744000B90128E130E040E050E00F9435442901D3
:107450003A01DF920F93C50168E170E00F940E448A
:107460009F938F935F924F9282EB95E19F938F93BF
:10747000FF92EF920F948D490FB6F894DEBF0FBEC6
:10748000CDBF5AE0451651046104710408F08EC066
:1074900098E0892F880F980F892F81956FE2855A80
:1074A00067DDC701DCDD809177048632A0F480912E
:1074B00079048E3180F008E020E84EE160E083E45A
:1074C00094E0F1D880917704863228F48091790491
:1074D0008F3108F06DC080917704823328F4809159
:1074E00079048B3208F014C180917704813408F05C
:1074F00040C280917904873308F43BC26EE380E098
:1075000037DD812FB2DD35C28CE296E1C8CE86EF41
:1075100095E1DECE04E02AE441E366E383E494E00F
:1075200072D851CFF8E48F9FB0011124072E000CC0
:10753000880B990B0F948D412AE037ED43E25CE311
:107540000F9429430F945F41262F02E042E367E343
:1075500083E494E0A8D844CF84E6A816B10498F454
:10756000DF920F933F932F9388EA95E19F938F9338
:10757000FF92EF920F948D490FB6F894DEBF0FBEC5
:10758000CDBF95E086CFDF920F933F932F9380EA94
:1075900095E19F938F93FF92EF920F948D490FB6D1
:1075A000F894DEBF0FBECDBF96E073CF99E071CFE8
:1075B00060E083E494E00E94B13065E283E0D8DCCF
:1075C00068E570E080E090E04DDD65E28BE0D0DCC6
:1075D000112321F08CE294E042DD24C08091E60D7D
:1075E00080FD17C03CE2E32E34E0F32EF7016191F9
:1075F0007F016623B9F06F3234F4062E000C770B4E
:10760000880B990B04C06FE370E080E090E02ADD06
:10761000EDCF8091E50D80FDDDCF6FEF7FEF83E94A
:1076200095E100DD65E288E2A3DC69E570E080E0D9
:1076300090E018DD65E280E39BDC112321F087E216
:1076400094E00DDD26C08091E60D869580FD17C083
:1076500027E2E22E24E0F22EF70161917F016623FA
:10766000C1F06F3234F4062E000C770B880B990BA7
:1076700004C06FE370E080E090E0F4DCEDCF809137
:10768000E50D869580FDDBCF6FEF7FEF83E995E118
:10769000C9DC65E28DE46CDC6AE570E080E090E0D6
:1076A000E1DC65E285E564DC112321F08FE194E003
:1076B000D6DC28C08091E60D8695869580FD17C0A2
:1076C0009FE1E92E94E0F92EF70161917F01662395
:1076D000C9F06F3234F4062E000C770B880B990B2F
:1076E00004C06FE370E080E090E0BCDCEDCF8091FF
:1076F000E50D8695869580FDD9CF6FEF7FEF88E900
:1077000095E190DC61E083E494E00E94B130E3CE47
:1077100083E00ED462E383E02BDC66E070E080E07F
:1077200090E0A0DC81E004D462E38CE021DC809175
:107730006402909165020F94B03491DC65E270E0D0
:1077400080E090E08FDCD0CE80911E0D11112DC015
:107750008111E5CD2AC080917904853108F059C0A6
:10776000E3CD2091FA0C111184C02111EECD81C01E
:1077700080917904853108F0B0C0ECCD8091790416
:10778000853108F0DAC0EBCD90FD03C086E596E1C7
:1077900002C08EE696E17C010CE022E048E068E061
:1077A00083E494E00E94DB30B5CDB601DD0C880B9C
:1077B000990B0F948D4120E030E040E05FE30F949F
:1077C00012400F945A41CB010F94B0347C01FC015C
:1077D00080818032E1F4F7018181803211F401E08F
:1077E00001C002E0902F990F900F892F819567E0DB
:1077F000815FBEDB83E090E0801B91098E0D9F1DB1
:107800002EDC69E070E080E090E02CDC88CD03E0C5
:10781000E9CF20E030E040E05FE3C501B4010F9420
:1078200012400F945A41CB010F94B0347C01FC01FB
:1078300080818032E1F4F7018181803211F401E02E
:1078400001C002E0902F990F900F892F81956CE174
:10785000815F8EDB83E090E0801B91098E0D9F1D80
:10786000FEDB69E070E080E090E0FCDB5DCD03E0F2
:10787000E9CFBC01990F880B990B0F948D4120E043
:1078800030E040E05FE30F9412400F945A41CB0187
:107890000F94B0347C01FC0180818032E1F4F70167
:1078A0008181803211F401E001C002E0902F990F34
:1078B000900F892F819567E0845A5ADB83E090E02E
:1078C000801B91098E0D9F1DCADB69E070E080E08E
:1078D00090E0C8DB3ACD03E0E9CF20E030E040E0C3
:1078E0005FE3C501B4010F9412400F945A41CB01DC
:1078F0000F94B0347C01FC0180818032E1F4F70107
:107900008181803211F401E001C002E0902F990FD3
:10791000900F892F81956CE1845A2ADB83E090E0F7
:10792000801B91098E0D9F1D9ADB69E070E080E05D
:1079300090E098DB0FCD03E0E9CF0091270D002305
:1079400009F40DCD6CE187E613DBF4E60F9FC0016F
:10795000112481589F4F6FEF70E00F942244CB01A8
:107960000F94B0347CDB65E270E080E090E07ADB7D
:10797000F6CC2D960FB6F894DEBF0FBECDBFDF91CB
:10798000CF911F910F91FF90EF90DF90CF90BF901C
:10799000AF909F908F907F906F905F904F900895E1
:1079A0000F931F93CF93DF93CDB7DEB728970FB612
:1079B000F894DEBF0FBECDBF8A0123E0660F771FAC
:1079C0002A95E1F7680F791F48E050E0CE01019653
:1079D0000F94C14829813A81F8018081918128174B
:1079E000390790F08217930760F09C818281981785
:1079F00058F081E090E03B812381231738F080E04C
:107A000005C081E090E002C08FEF9FEF28960FB68F
:107A1000F894DEBF0FBECDBFDF91CF911F910F91C4
:107A20000895EF92FF920F931F93CF93DF93EC0192
:107A30008B017A018A859B858617970729F08881B3
:107A40009981C1D81B870A8788859985019681F01D
:107A50000E811F81B70188819981B2D8080F111D4D
:107A6000888599858017910718F481E090E011C00E
:107A70006E818A81680F97014C81888199810E946B
:107A8000F4342E813F81280F311D3F832E8380E007
:107A900090E0DF91CF911F910F91FF90EF900895AB
:107AA0004F925F926F927F928F929F92AF92BF920E
:107AB000CF92DF92EF92FF920F931F93CF93DF93BA
:107AC000CDB7DEB72D970FB6F894DEBF0FBECDBF92
:107AD0006C012A013B01490158011B861C86CE011D
:107AE00001967C0188E0F70111928A95E9F7DB01A4
:107AF000CA0127E0B695A795979587952A95D1F75E
:107B00009A838983F42FFF77FD878F2F80588B838B
:107B10008C831A8619864F3F51056105710509F05E
:107B200018F460E070E026C0609134047091350470
:107B30008E01075F1F4F970140ED5CE38091320497
:107B4000909133040E94CD7797FDEBCF69857A85BC
:107B500083E0660F771F8A95E1F780913204909158
:107B60003304680F791F48E050E0C7010F94C14803
:107B70006F8178856115710519F44B86B60106C0D1
:107B8000C616D70619F08D8580688B87AE01455FD4
:107B90005F4FC401F50119952D960FB6F894DEBF1D
:107BA0000FBECDBFDF91CF911F910F91FF90EF904E
:107BB000DF90CF90BF90AF909F908F907F906F900D
:107BC0005F904F9008956F927F928F929F92AF92A5
:107BD000BF92CF92DF92EF92FF920F931F93CF93BA
:107BE000DF9300D01F92CDB7DEB76C017B013A0165
:107BF0005901480119821A821B821C82AE014F5F13
:107C00005F4FB301C7010E942D787C0149815A81E1
:107C10006B817C81411551056105710529F0840155
:107C20009501C6013DDFE6CF0F900F900F900F90AA
:107C3000DF91CF911F910F91FF90EF90DF90CF9048
:107C4000BF90AF909F908F907F906F90089521E0AC
:107C500020933604E2E3F4E09183808373836283AC
:107C600080E090E008957F92AF92BF92CF92DF9232
:107C7000EF92FF920F931F93CF93DF93CDB7DEB7B1
:107C80002C970FB6F894DEBF0FBECDBF6C01762ED9
:107C9000F72F842FE52FB901A801D6011496AD90D6
:107CA000BC9015979091360491110AC026EC36E1EC
:107CB000482F672DC6010E942B3580E090E019C047
:107CC000DA82C9827B82FC838D83EE8318861F82D1
:107CD000FA86E9861C861B8601E11DE39E012F5F63
:107CE0003F4FC501DDDEB501C6010E94E3358F813E
:107CF00098852C960FB6F894DEBF0FBECDBFDF91EE
:107D0000CF911F910F91FF90EF90DF90CF90BF9098
:107D1000AF907F900895CF92DF92EF92FF920F93F2
:107D20001F93CF93DF93CDB7DEB72C970FB6F894A0
:107D3000DEBF0FBECDBF7C01C901F701C480D58075
:107D400020913604211108C026EA36E1C7010E94BD
:107D50002B3580E090E01CC0FA82E9826B837C8343
:107D60004D835E8318861F821A8709871C861B86AF
:107D700001E11DE39E012F5F3F4F47EC57E7BC0138
:107D8000C60121DFB601C7010E94E3358F819885C6
:107D90002C960FB6F894DEBF0FBECDBFDF91CF910A
:107DA0001F910F91FF90EF90DF90CF900895CF92A9
:107DB000DF92EF92FF920F931F93CF93DF93CDB794
:107DC000DEB72C970FB6F894DEBF0FBECDBF7C0197
:107DD000C901F701C480D58020913604211108C063
:107DE00026E836E1C7010E942B3580E090E01CC0F8
:107DF000FA82E9826B837C834D835E8318861F82BF
:107E00001A8709871C861B8601E11DE39E012F5FEF
:107E10003F4F4AEC57E7BC01C601D5DEB601C701AA
:107E20000E94E3358F8198852C960FB6F894DEBFBB
:107E30000FBECDBFDF91CF911F910F91FF90EF90BB
:107E4000DF90CF900895CF93DF93EC01262F4CADB8
:107E50006BAD04960E94D6342BAD082E000C990B06
:107E6000820F911D8BAF81E090E0DF91CF9108955B
:107E70000F939CE0899F802D112421E0280F2093EF
:107E80003E04845F80933D0490E002964091770425
:107E900050E08417950714F480E033C0822F90E0FF
:107EA0002091790430E082179307B4F76623A9F094
:107EB00061E083E494E00E94B13040913E044E5F63
:107EC0000BE020E860E083E494E00E94533360E03C
:107ED00083E494E00E94B13005C061E083E494E063
:107EE0000E94B13060913D04809177046817A0F240
:107EF00090913E0480917904891770F280E038D81F
:107F000081E00F910895CF93DF93FC0185ADEF01E0
:107F10002496811105C081E085AFCE010E945130C9
:107F2000CE01DF91CF910C9488306FEF7FEF7AC84C
:107F3000482F50E020913C04022E000C330B4217D6
:107F4000530781F080933C04813031F461EA7FE192
:107F500083E494E00C94E33561EB77E183E494E00F
:107F60000C94E3350895EF92FF920F9383E6E82E89
:107F70008DE1F82E00E428E040E060E083E494E046
:107F80000E94DB306BE273E083E494E00E94E3350F
:107F900020E233E041E169E383E494E00E94F434B9
:107FA0006BE97BE083E494E00E94E33526E233E072
:107FB0004CE16AE383E494E00E94F43466EF7EE0EF
:107FC00083E494E00E94E33523E333E049E26BE38A
:107FD00083E494E00E94F43466EF7EE083E494E06E
:107FE0000E94E3352FE333E04EE36DE383E494E056
:107FF0000E94F43421E433E04EE362E483E494E04D
:108000000E94F43461EB77E183E494E00F91FF90F8
:10801000EF900C94E3358FE394E075DF61E080E04E
:10802000A2DF83E494E00E948C308111F7CF64ECEE
:1080300079E080E090E00C94F898EF92FF920F9333
:108040008EEDE82E8CE1F82E03E127E047E064E2B4
:1080500083E494E00E94DB3083E06ADF21E433E0D4
:108060004BE265E283E494E00E94F4342BE433E0D5
:1080700047E367E083E494E00F91FF90EF900C9466
:10808000F4348FE394E03FDFD8DF83E494E00E9490
:108090008C308111F9CF64EC79E080E090E00C94B1
:1080A000F898B9DFEECF60E070E081EA9FE1CFCDD4
:1080B0001F93CF93DF93C0914404C695C6958FE379
:1080C00094E021DFDC2FDD0F1D2F1C0F83E030DF5C
:1080D0006C2F80E00E94B83783ED96E00E942F3825
:1080E0006D2F80E00E94B83783EF96E11EDF612F8D
:1080F00080E00E94B83786EE96E117DF83E494E0D3
:108100000E948C308111E2CFDF91CF911F910895B1
:108110000895CF93E62F6CE0869F602D112481E0B7
:10812000860F80933E04645F60933D04462F50E0C9
:108130004E5F5F4F2091770430E0421753070CF4F5
:108140004CC090E02091790430E0821793070CF046
:1081500044C0CE2F8EE30E94B83765E470E080E023
:1081600090E00E94323861E36C0F062E000C770B12
:10817000880B990B0E94323860E270E080E090E05A
:108180000E94323860912D0D70912E0D80912F0D2F
:108190009091300D0F945A41CB010F94B0340E944E
:1081A0002F386FE270E080E090E00E9432380E9449
:1081B000BB7B811109C085E0C89FF0011124E65EF8
:1081C000F24F8481811109C08091310D9091320D5F
:1081D0000F94B034CF910C942F38CF910895CF9253
:1081E000DF92EF92FF920F931F93CF93DF931F9233
:1081F0001F92CDB7DEB77B01622F498339DE4981FB
:10820000882309F444C0442311F101151105F9F440
:10821000C7010E949D7925E130E0281B310937FF15
:1082200002C02F5F3F4F3595279530E82158822FA8
:10823000830F87FD0DC060E270E080E090E02A834C
:1082400039830E943238398131502A81F0CF30E8A9
:10825000C32ED12CB601C7010E9412387601E81A4C
:10826000F90A0115110511F41E2D07C0FF24B701ED
:10827000C8010E94F5371E2D181B173040F060E230
:1082800070E080E090E00E943238181BF6CF0F902B
:108290000F90DF91CF911F910F91FF90EF90DF90A2
:1082A000CF9008950F93CF93DF93982F862FEA01F5
:1082B000692FDEDD882331F162E770E0CE010E9494
:1082C0001238C2E7C81BC73040F060E270E080E0BF
:1082D00090E00E943238C81BF6CF60913D048AE7D7
:1082E0000E94B837602F000F770B880B990B0E9404
:1082F000323860E270E080E090E0DF91CF910F9142
:108300000C943238DF91CF910F910895CF92DF9284
:10831000EF92FF920F931F93CF93DF93982F862FA7
:108320006A017901692FA4DD882309F447C0C701D8
:10833000002321F00E949D79182F03C00E947C79B0
:10834000182FC3E1D0E0C11BD1098C2F880FC80FB3
:10835000CC0FD0E0BE01C6010E941238C81B6AE3F0
:1083600070E080E090E00E943238C73040F060E278
:1083700070E080E090E00E943238C81BF6CF8AEFB0
:10838000189F802D112460913D0480580E94B837B9
:10839000C701002349F0DF91CF911F910F91FF900A
:1083A000EF90DF90CF90C1CDDF91CF911F910F91D2
:1083B000FF90EF90DF90CF900C942F38DF91CF910A
:1083C0001F910F91FF90EF90DF90CF900895BF9293
:1083D000CF92DF92EF92FF920F931F93CF93DF9391
:1083E0006C017B010E949D79C82FC7010E947C7996
:1083F00003E110E0081B11098C2F90E0BB24B3941B
:10840000081719071CF0B12CC5E201C0CFE12C2FD1
:1084100030E0A9014E5F5F4F8091770490E04817EC
:10842000590744F0295031098091790490E082176E
:108430009307BCF5D0E0E114F104D9F16AE370E0F0
:1084400080E090E00E943238BB2081F0C45F8091D0
:108450007704C81770F12C2F30E029503109809132
:10846000790490E0821793071CF423C0DD2309F1FF
:10847000802F880F800F6C2F880F0E94B83760E222
:1084800070E080E090E00E943238C701DF91CF9128
:108490001F910F91FF90EF90DF90CF90BF900C94C1
:1084A0002F386C2F80E00E94B837C6013EDDD1E046
:1084B000C2CFDF91CF911F910F91FF90EF90DF908E
:1084C000CF90BF900895CF92DF92EF92FF920F93DB
:1084D0001F93CF93DF931F92CDB7DEB7182F7A018A
:1084E000D22ECA0169830E949D79082F812F880F9F
:1084F000810FC82ECC0C1CE06981169F100D112431
:10850000DD20C1F061E083E494E00E94B130202FCF
:10851000220F200F220F2E5F0BE047EF410F6FEF6E
:108520006C0D83E494E00E94533360E083E494E0B4
:108530000E94B130612F8C2D0E94B837C701F5DC45
:10854000DD2071F061E083E494E00F90DF91CF9142
:108550001F910F91FF90EF90DF90CF900C94B1306E
:108560000F90DF91CF911F910F91FF90EF90DF90CF
:10857000CF900895AF92BF92DF92EF92FF920F9348
:108580001F93CF93DF93EC015B01D42EC901B80197
:10859000A7010E944C7B91E02D2D2927A50164E0C5
:1085A00081E091DFCE010E949D792D2DAE0164E026
:1085B00094E1981B892FDF91CF911F910F91FF902C
:1085C000EF90DF90BF90AF907ECFEF92FF920F932E
:1085D000CF93DF93D82FC62F7901682F8C2F48DCDB
:1085E0008823F1F0002331F062E070E080E090E059
:1085F0000E9432382D2F4C2F64E1C7010E94287A47
:1086000068E770E00E94F537C8E7C81BC73040F044
:1086100060E270E080E090E00E943238C81BF6CF44
:10862000DF91CF910F91FF90EF9008958F929F92DD
:10863000AF92BF92CF92DF92EF92FF920F936B01B6
:108640007C018090380490903904A0903A04B09056
:108650003B04A50194010F94EB40882301F120E035
:1086600030E0A901C701B6010F94EB40882351F017
:10867000A5019401C701B6010F94EB4087FD04C02A
:1086800081E003C080E001C08FEF80933704C09287
:108690003804D0923904E0923A04F0923B0480917D
:1086A0007704813128F480917904833008F048C040
:1086B00080917704853128F480917904843108F021
:1086C0004FC0809177048F3308F057C080917904B0
:1086D0008F3208F452C08091370440E3481B87E38F
:1086E000E82E87E1F82E0DE022E06AE583E494E0CD
:1086F0000E94DB308091370441E3481B9DE1E92E65
:1087000097E1F92E22E065E083E494E00E94DB30FB
:1087100021E5E22E27E1F22E00E123E04FE262E1C3
:1087200083E494E00E94DB3031E8E32E37E1F32E5E
:1087300023E04FE267E683E494E00E94DB301DC053
:108740008091370444E0481B52E0E52E57E1F52EB6
:108750000CE022E062E483E494E00E94DB30A8CFE6
:108760004AE1E42E47E1F42E01E023E044E16CE32A
:1087700083E494E00E94DB30A4CF0F91FF90EF9050
:10878000DF90CF90BF90AF909F908F900895CF9241
:10879000EF920F93CF93DF93CFE3D4E01B821A8243
:1087A00083E693E099838883CC24CA94EE24EA94E8
:1087B00006E427E448E464E172E0CE010E949237C7
:1087C0008FE693E099838883DF91CF910F91EF90AB
:1087D000CF9008959091050194709093030187FDC7
:1087E00076C0A398909105019095947090930301A1
:1087F00090910501947090930301982F990F86FD35
:1088000072C0A398809105018095847080930301C4
:1088100080910501847080930301292F220F96FD1A
:1088200060C0A398809105018095847080930301B6
:1088300080910501847080930301922F990F26FD8A
:108840004EC0A398809105018095847080930301A8
:1088500080910501847080930301292F220F96FDDA
:108860003CC0A3988091050180958470809303019A
:1088700080910501847080930301922F990F26FD4A
:108880002AC0A3988091050180958470809303018C
:1088900080910501847080930301292F220F96FD9A
:1088A00018C0A3988091050180958470809303017E
:1088B0008091050184708093030126FD16C0A39862
:1088C0008091050180958470809303010895A39A97
:1088D00089CFA39AE7CFA39AD5CFA39AC3CFA39A60
:1088E000B1CFA39A9FCFA39A8DCFA39A8091050170
:1088F000809584708093030108952F923F925F9238
:108900007F929F92AF92BF92CF92DF92EF92FF92AF
:108910000F931F93CF93DF937C011B01942E69016A
:108920008AE0481709F47BC0A5E14A134EC0DB0179
:108930001296ED91FC9113971281C681D781A49A6A
:1089400088E28A950000E9F700EE010F80E1582ED9
:10895000510E98E2792E88EF3DDF872D8A95000031
:10896000E9F7103208F046C0812F8077806832DF47
:10897000812F8295807F2EDF872D8A950000E9F771
:1089800080E828DF80E026DF872D8A950000E9F760
:108990008AEF20DF872D8A950000E9F75E01B0E1BC
:1089A000AB0EB11C8881807F15DF89918295807F15
:1089B00011DFCA15DB05B1F7872D8A950000E9F7AD
:1089C0001F5F0F5F1511C7CFA4989601492DB10104
:1089D000C701DF91CF911F910F91FF90EF90DF9032
:1089E000CF90BF90AF909F907F905F903F902F90DF
:1089F0000C941532802F80778068ECDE802F829572
:108A0000807FE8DE872D8A950000E9F780E8E2DEC6
:108A100080E8E0DE872D8A950000E9F7B9CF9C9ABF
:108A2000A4989B9AA3988091040184608093040188
:108A3000809105018095847080930301A49AC8E217
:108A40008C2F8A950000E9F788E790E00E94323188
:108A500088EFC0DE8C2F8A950000E9F780E2BADE4D
:108A600080E0B8DE8C2F8A950000E9F780E0B2DE66
:108A700080E8B0DE8C2F8A950000E9F780E0AADE5E
:108A800080E1A8DE8C2F8A950000E9F78FE090E066
:108A90000E94323180E29EDE80E49CDE8C2F8A953B
:108AA0000000E9F780E296DE80E694DECA950000D9
:108AB000E9F710E0D8E208E2812F807780688ADE4B
:108AC000812F8295807F86DE8D2F8A950000E9F7C1
:108AD00080E880DE80E07EDE8D2F8A950000E9F759
:108AE0008AEF78DE8D2F8A950000E9F7C0E280E0FA
:108AF00071DE80E06FDE9D2F9A950000E9F7C1508E
:108B0000B1F788EF67DE802F8A950000E9F71F5FD5
:108B1000103209F0D1CF80E05DDE80EC5BDE88E2D0
:108B20008A950000E9F7A49850CFCF93DF931F9266
:108B30001F92CDB7DEB789839A830E94B97420E073
:108B400040E060E070E089819A810F900F90DF91A2
:108B5000CF910C945E750F93CF93DF9361E081E02A
:108B60000E946276D091A106C0E0D11117C0809119
:108B7000A006811104C00E94727A811165C08091A3
:108B80002202882309F457C081E09091A006911138
:108B900080E004E024E045EB58E24BC0D130C1F462
:108BA0008091A006813021F40E94727A811154C014
:108BB00080912202882309F43EC081E09091A006B2
:108BC000913009F080E003E02EE34CEA58E231C036
:108BD000D230B9F48091A006823021F40E94727ADA
:108BE000811143C080912202882329F181E0909174
:108BF000A006923009F080E003E02EE343EA58E259
:108C000018C0D330C1F48091A006833021F40E94B3
:108C1000727A811133C080912202882361F081E051
:108C20009091A006933009F080E003E02EE34DE937
:108C300058E26C2F37DBCF5FDF5FC53009F095CF8F
:108C400084E080939F0621C00E948C7580916D0600
:108C5000882309F494CF19C087EF9AE666DF8091E4
:108C60006D06882309F4A4CF10C086E090E75DDF8D
:108C700080916D06882309F4B5CF07C087EC93E790
:108C800054DF80916D06882331F2DF91CF910F91EF
:108C90000895CF92DF92EF92FF920F931F938091EE
:108CA0005E09811103C080EA99E002C08EE599E077
:108CB00029EFC22E28E2D22E7C010CEE18E22CE81D
:108CC00035E740E756E465EE78E28FED98E20E94E2
:108CD0005A771F910F91FF90EF90DF90CF900895FA
:108CE00080EA99E00E943A850E9485750C94738011
:108CF0000E94D68921E030E0811102C020E030E0FE
:108D00003093C8062093C7061092A10681E0809395
:108D10006D0683E0809322020895CF92DF92EF9256
:108D2000FF920F931F93CF93DF930E94DA8A6C0117
:108D300061E081E00E946276C091A106D0E081E00E
:108D4000C81AD108C11117C08091A006811104C0B2
:108D50000E94727A811195C080912202882359F075
:108D600081E09091A006911180E004E024E04AEDBA
:108D700058E26D2F97DA60EA79E087E299E00E9485
:108D8000D3908091A0098F3201F18091AD0983FFCA
:108D90001CC0C130C1F48091A006813021F40E9432
:108DA000727A811176C080912202882361F081E07D
:108DB0009091A006913009F080E000E22EE346EDAC
:108DC00058E26D2F6FDA92E001C091E080912202AB
:108DD000882309F44EC0760111E01C0F8FEFE816CE
:108DE000F80609F446C0C9133FC060E070E0C7014F
:108DF0000E94AF869091AD098091A00694FF1CC09F
:108E00008C134EC00E94727A882309F449C080EA0C
:108E100099E00E9480891092A10682E090E09093F0
:108E2000C8068093C70681E080936D061092CA063B
:108E300083E08093220252C08C1304C00E94727A95
:108E400081113DC080912202882361F081E09091E0
:108E5000A0069C1380E000E02EE437E14AEB58E2E4
:108E60006D2FB3DB912F01C09F5F81E0E81AF108FD
:108E7000B5CFDF5FCF5FD53009F064CF90939F0609
:108E80002DC00E948C7580916D06882309F464CFF3
:108E900025C02EDF80916D06882309F484CF1EC083
:108EA000809122028823F1F281E09091A0069C1328
:108EB00080E001E02EE437E148EC58E2D1CF0E9497
:108EC000B97420E040E060E070E089E496E40E943C
:108ED0005E7580916D06882309F4B4CFDF91CF9140
:108EE0001F910F91FF90EF90DF90CF900895CF9357
:108EF000DF93EC01CB01BA010F948D410F945F41D8
:108F00006883DF91CF910895CF93DF93EC01CB017C
:108F1000BA010F948D412FE632E143E85AE30F94F2
:108F20002943688379838A839B83DF91CF91089556
:108F300067E777E484EA97E40C94A17564E877E442
:108F400081EC97E40C94A1750F948D410F945F41CF
:108F5000862F0D940534CF93DF9300D01F92CDB7A9
:108F6000DEB769837A838B839C8360E2CE010196AE
:108F70000F9429370F900F900F900F90DF91CF91A2
:108F800008950F948D412FE632E143E85AE30F94A0
:108F90002943E1CF2F923F924F925F926F927F923F
:108FA0008F929F92AF92BF92CF92DF92EF92FF92F9
:108FB0000F931F93CF93DF93CDB7DEB729970FB6EB
:108FC000F894DEBF0FBECDBF1C0179876887CA0148
:108FD000B901E982FA820B831C83DE82CD82AF82E3
:108FE00020E030E04AE754E40F9429436B017C0110
:108FF00020E030E040E057EC0F94EE4218162CF0E1
:10900000C12CD12CE12C27ECF22EC701B6010F9414
:109010005A412B013C0120E030E04AE754E46981E9
:109020007A818B819C810F9429434B015C0120E064
:109030003EEF4FEF56E40F94EB4087FD07C0812CC5
:109040009EEF992EAA24AA9496E4B92E20E030E04F
:109050004AE754E4E885F9856081718182819381D2
:109060000F9429436B017C01C301B2010F948D4120
:109070009B01AC01C701B6010F9411400F945F41F1
:1090800069837A838B839C83C501B4010F945A4111
:109090007B018C01E418F50806091709FF81FF938D
:1090A0008D809E808EE9A82E87E4B82EC980DA8054
:1090B000A301920168857985C1010E94E0740F9037
:1090C00029960FB6F894DEBF0FBECDBFDF91CF91CA
:1090D0001F910F91FF90EF90DF90CF90BF90AF90D6
:1090E0009F908F907F906F905F904F903F902F90C8
:1090F00008958F929F92AF92BF92CF92DF92EF929C
:10910000FF920F931F93CF93DF9361E081E00E9462
:109110006276D091A106C0E0D11119C08091A0065D
:10912000811104C00E94727A8111C4C08091220210
:10913000882309F4B6C081E09091A006911180E0E7
:1091400004E024E041E359E26C2FACD8AAC0D1304E
:10915000E1F48091A006813021F40E94727A81119D
:10916000B1C080912202882309F49BC011E0809154
:10917000A006813009F010E08091A20C0F94053414
:1091800000E09C014BE159E289C0D23009F58091A1
:10919000A006823021F40E94727A8111B4C08091BD
:1091A0002202882309F47DC011E08091A00682305C
:1091B00009F010E06091A30C7091A40C8091A50CB3
:1091C0009091A60CC8DE00E09C0147E159E266C020
:1091D000D33009F58091A006833021F40E94727A81
:1091E0008111AAC080912202882309F45AC011E09B
:1091F0008091A006833009F010E06091A70C709177
:10920000A80C8091A90C9091AA0CA5DE00E09C010D
:1092100043E159E243C0D43001F58091A006843087
:1092200021F40E94727A8111A0C0809122028823C9
:10923000C1F111E08091A006843009F010E0609146
:10924000AB0C7091AC0C8091AD0C9091AE0C83DEA8
:1092500000E09C014FE059E221C0D53011F580912A
:10926000A006853021F40E94727A811197C0809106
:1092700022028823B1F011E08091A006853009F028
:1092800010E060912602709127028091280290914F
:10929000290261DE00E09C014BEF58E26C2F812F28
:1092A00035D8CF5FDF5FC53009F036CF86E08093D9
:1092B0009F068CC00E948C7580916D06882309F4EE
:1092C00035CF84C081E00E94677AC090A20CD12C77
:1092D0001F92812C912C48E9A42E47E4B42EE12C56
:1092E000F12C8701EA9420E030E0A90162EA7CE0F9
:1092F00086E299E20E94E0740F9080916D068823C7
:1093000009F42FCF63C081E00E94677AA12CC12CA1
:10931000D12C16E6E12EFE2C0EE111E420E030E027
:10932000A90163EA7CE089E199E234DE80916D066F
:10933000882309F434CF4AC081E00E94677AA12CC7
:10934000C12CD12C16E6E12EFE2C0EE111E420E01A
:1093500030E0A90167EA7CE085E199E21BDE8091BB
:109360006D06882309F43ECF31C081E00E94677A00
:10937000A12CC12CD12C16E6E12EFE2C0EE111E41D
:1093800020E030E0A9016BEA7CE081E199E202DEB5
:1093900080916D06882309F448CF18C081E00E94AF
:1093A000677AA12CC12CD12C16E6E12EFE2C0EE101
:1093B00011E420E030E0A90166E272E085E099E284
:1093C000E9DD80916D06882309F451CFDF91CF91BB
:1093D0001F910F91FF90EF90DF90CF90BF90AF90D3
:1093E0009F908F900895CF93DF93EC01CB01BA014A
:1093F0000F948D412AE037ED43E25CE30F9429435B
:10940000688379838A839B83DF91CF910895CF937B
:10941000DF93EC01CB01BA010F948D41688379830E
:109420008A839B83DF91CF910895CF93DF93EC01E3
:10943000CB01BA010F948D4120E030E048EC51E4BB
:109440000F942943688379838A839B83DF91CF912B
:109450000895CF93DF93EC01CB01BA010F948D41B6
:1094600020E030E048EC52E40F942943688379838C
:109470008A839B83DF91CF910895CF93DF93EC0193
:10948000CB01BA010F948D4120E030E048EC51E46B
:109490000F9429430F945F41688379838A839B8368
:1094A000DF91CF910895CF93DF93EC01CB01BA0107
:1094B0000F948D4120E030E048EC52E40F942943B2
:1094C0000F945F41688379838A839B83DF91CF9177
:1094D0000895CF93DF93EC01CB01BA010F948D4136
:1094E0002AE037ED43E25CE30F94294368837983F4
:1094F0008A839B83DF91CF910895CF93DF93EC0113
:10950000CB01BA010F948D412DEC3CEC4CEC5DE3AA
:109510000F942943688379838A839B83DF91CF915A
:10952000089563EF79E482EE9AE40C94A17567E004
:109530007AE48AE99BE40C94A17569E27AE48CE10F
:109540009BE40C94A17565E17AE48FEF9AE40C94A6
:10955000A1756DE37AE48DED9EE40C94A17563E54D
:109560007AE486E59BE40C94A17569E67AE489E3E4
:109570009BE40C94A1756DE77AE485EC9AE40C9475
:10958000A1750C9447F80C948EF8CF93DF9300D01C
:109590001F92CDB7DEB70F948D412DEC3CEC4CEC17
:1095A0005DE30F94294369837A838B839C83CE0187
:1095B00001960F9447390F900F900F900F90DF9105
:1095C000CF910895CF93DF9300D01F92CDB7DEB730
:1095D0000F948D412AE037ED43E25CE30F94294379
:1095E00069837A838B839C83CE0101960F94EB353C
:1095F0000F900F900F900F90DF91CF910895CF9320
:10960000DF9300D01F92CDB7DEB70F948D4120E0DD
:1096100030E048EC51E40F94294369837A838B83CB
:109620009C83CE0101960F9472380F900F900F908B
:109630000F90DF91CF910895CF93DF9300D01F92C9
:10964000CDB7DEB70F948D4120E030E048EC52E416
:109650000F94294369837A838B839C83CE0101967F
:109660000F9472380F900F900F900F90DF91CF9161
:109670000895CF93DF9300D01F92CDB7DEB70F943C
:109680008D412AE037ED43E25CE30F94294369837F
:109690007A838B839C83CE0101960F94A7380F9019
:1096A0000F900F900F90DF91CF910895CF93DF939C
:1096B00000D01F92CDB7DEB70F948D4120E030E08F
:1096C00048EC52E40F9429430F945F410F948B416F
:1096D00069837A838B839C83CE0101960F947238C1
:1096E0000F900F900F900F90DF91CF910895CF9230
:1096F000DF92EF92FF926B017C0120E030E0A90144
:109700000F94EB4087FD05C020E030E040E05FE3D0
:1097100004C020E030E040E05FEBC701B6010F94E9
:1097200012400F945A41CB01FF90EF90DF90CF9001
:109730000D94B0340F948D41DACFCF93DF9300D0E6
:109740001F92CDB7DEB70F945F410F948B416983B1
:109750007A838B839C83CE0101960F9472380F908D
:109760000F900F900F90DF91CF9108956F927F929D
:109770008F929F92AF92BF92CF92DF92EF92FF9221
:109780000F931F93CF93DF9300D01F92CDB7DEB717
:1097900061E081E00E9462766090A106712C611008
:1097A0001AC08091A006811104C00E94727A8111B2
:1097B00059C180912202882309F44BC181E0909124
:1097C000A006911180E004E024E048E95AE2672D08
:1097D0000E9452413EC181E068122CC08091A006D7
:1097E000813021F40E94727A811144C18091220259
:1097F000882309F42EC111E08091A006813009F080
:1098000010E08091C90E9091CA0EA091CB0EB0913C
:10981000CC0E89839A83AB83BC83CE0101960F94CF
:10982000723800E09C014CE85AE2672D812F0E94BB
:1098300086410FC182E068122CC08091A006823060
:1098400021F40E94727A81114DC1809122028823F5
:1098500009F4FFC011E08091A006823009F010E009
:109860008091CD0E9091CE0EA091CF0EB091D00EE2
:1098700089839A83AB83BC83CE0101960F9472389F
:1098800000E09C0148E75AE2672D812F0E94864143
:10989000E0C083E068122CC08091A006833021F4E0
:1098A0000E94727A811156C180912202882309F4A4
:1098B000D0C011E08091A006833009F010E08091C3
:1098C000D10E9091D20EA091D30EB091D40E898377
:1098D0009A83AB83BC83CE0101960F94723800E06B
:1098E0009C0146E65AE2672D812F0E948641B1C055
:1098F00084E0681227C08091A006843021F40E9481
:10990000727A81115FC180912202882309F4A1C07B
:1099100011E08091A006843009F010E06091950E6E
:109920007091960E8091970E9091980E0F948B41A6
:1099300004DF00E09C0148E55AE2672D812F0E9478
:10994000864187C085E0681227C08091A0068530D7
:1099500021F40E94727A811171C1809122028823C0
:1099600009F477C011E08091A006853009F010E07D
:109970006091990E70919A0E80919B0E90919C0E21
:109980000F948B41DADE00E09C014AE45AE2672D35
:10999000812F0E9486415DC086E0681227C08091B9
:1099A000A006863021F40E94727A811183C18091D1
:1099B0002202882309F44DC011E08091A006863070
:1099C00009F010E060919D0E70919E0E80919F0EA7
:1099D0009091A00E0F948B41B0DE00E09C014CE30F
:1099E0005AE2672D812F0E94864133C087E06812BA
:1099F00030C08091A006873021F40E94727A8111D4
:109A00008EC180912202882321F111E08091A0066D
:109A1000873009F010E06091A10E7091A20E809144
:109A2000A30E9091A40E0F948B410F945F410F945D
:109A30008B4169837A838B839C83CE0101960F943B
:109A4000723800E09C014EE25AE2672D812F0E949D
:109A500086417394639485E07812A1CE88E0809368
:109A60009F0698C10E948C7580916D06882309F429
:109A7000A0CE90C181E00E94677A2AE037ED43E2F0
:109A80005DE36091C90E7091CA0E8091CB0E9091EA
:109A9000CC0E0F94294320E030E040E85FE30F94C0
:109AA00011400F945F411F92812C912C53EAA52EF7
:109AB0005AE4B52E6B0117E7E12E1FE0F12E00E00E
:109AC00010E021E030E040E050E069EC7EE082E927
:109AD0009AE20E94E0740F9080916D06882309F449
:109AE00085CE58C181E00E94677A2AE037ED43E2D3
:109AF0005CE36091CD0E7091CE0E8091CF0E90916F
:109B0000D00E0F94294320E030E040E85FE30F944B
:109B100011400F945F411F92812C912C3DE9A32E9F
:109B20003AE4B32E6B011DEDE12E13E0F12E00E0BF
:109B300010E021E030E040E050E06DEC7EE082E8B3
:109B40009AE20E94E0740F9080916D06882309F4D8
:109B50007CCE20C181E00E94677A2AE037ED43E2A3
:109B60005DE36091D10E7091D20E8091D30E9091F1
:109B7000D40E0F94294320E030E040E85FE30F94D7
:109B800011400F945F411F92812C912C93EAA92ED2
:109B90009AE4B92E6B0117E7E12E1FE0F12E00E0E9
:109BA00010E021E030E040E050E061ED7EE08FE643
:109BB0009AE20E94E0740F9080916D06882309F468
:109BC00073CEE8C081E00E94677A6091950E709133
:109BD000960E8091970E9091980E0F948B412AE0EB
:109BE00037ED43E25DE30F94294320E030E040E8A5
:109BF00050E40F9411400F945F411F92B1EC8B2EF3
:109C0000BAE49B2E19EAA12E1AE4B12E6B0114E7D7
:109C1000E12E1FE0F12E00E010E024E030E040E013
:109C200050E065E97EE08FE59AE20E94E0740F90D3
:109C300080916D06882309F466CEACC081E00E9455
:109C4000677A6091990E70919A0E80919B0E909117
:109C50009C0E0F948B412AE037ED43E25DE30F94B5
:109C6000294320E030E040E850E40F9411400F9485
:109C70005F411F92E1EC8E2EEAE49E2EF9EAAF2EB0
:109C8000FAE4BF2E6B0114E7E12E1FE0F12E00E095
:109C900010E024E030E040E050E069E97EE081E55A
:109CA0009AE20E94E0740F9080916D06882309F477
:109CB00054CE70C081E00E94677A60919D0E7091D1
:109CC0009E0E80919F0E9091A00E0F948B412AE0E2
:109CD00037ED43E25DE30F9429430F945F411F92F8
:109CE00031EC832E3AE4932E49EAA42E4AE4B42EB2
:109CF0006B0118E7E12E1FE0F12E00E010E020E0FC
:109D000030E0A9016DE97EE083E49AE20E94E0740C
:109D10000F9080916D06882309F449CE3BC081E005
:109D20000E94677A6091A10E7091A20E8091A30E9D
:109D30009091A40E0F948B412AE037ED43E25CE34F
:109D40000F94294320E030E040E85FE30F94114096
:109D50000F945F411F9281EC882E8AE4982E9FEA2F
:109D6000A92E9AE4B92E6B011DEDE12E13E0F12E20
:109D700000E010E021E030E040E050E061EA7EE009
:109D800085E39AE20E94E0740F9080916D0688232B
:109D900009F437CE0F900F900F900F90DF91CF9175
:109DA0001F910F91FF90EF90DF90CF90BF90AF90F9
:109DB0009F908F907F906F9008950F948D4120E039
:109DC00030E048EC51E40F942943B7CC0F931F9334
:109DD000CF93DF9361E081E00E946276C091A1069B
:109DE000D0E0C1111AC08091A006811104C00E9468
:109DF000727A8111CCC080912202882309F461C05B
:109E000081E09091A006911180E004E024E04CE60E
:109E100059E26D2F0E94524154C0C130D9F4809153
:109E2000A006813021F40E94727A8111B8C080911D
:109E30002202882309F445C081E09091A006913068
:109E400009F080E003E02EE343E659E26D2F0E9423
:109E5000524137C0C230D1F48091A006823021F443
:109E60000E94727A8111A5C080912202882349F153
:109E700081E09091A006923009F080E003E02EE3AB
:109E800046E559E26D2F0E9452411BC0C330C9F410
:109E90008091A006833021F40E94727A811193C0D0
:109EA00080912202882369F081E09091A00693308E
:109EB00009F080E003E02EE341E559E26D2F0E94B6
:109EC00052410E94477581111DC0C430E9F4809150
:109ED000A006843021F40E94727A81117EC08091A4
:109EE0002202882309F483C081E09091A006943077
:109EF00009F080E003E02EE348E459E26D2F0E9470
:109F0000524175C014E001C015E0C1131BC080911F
:109F1000A0068C1304C00E94727A81116AC08091DD
:109F20002202882371F081E09091A0069C1380E0CA
:109F300003E02EE34FE359E26D2F0E9452411C2FA4
:109F400001C01C2F81E0810FC81318C08091A006AA
:109F50008C1304C00E94727A811155C08091220234
:109F6000882361F081E09091A0069C1380E003E0DB
:109F70002EE346E359E26D2F0E945241DF5FCF5F2F
:109F8000D53009F02ECF1E5F10939F0645C00E946A
:109F90008C7580916D06882309F42DCF3DC08FEC20
:109FA00091E50E94954580916D06882309F43FCF85
:109FB00033C086EB9BE40E94954580916D06882313
:109FC00009F452CF29C087E993E50E949545809115
:109FD0006D06882309F464CF1FC08BEC95E50E94C1
:109FE000954580916D06882309F479CF15C015E059
:109FF000A9CF89E798E40E94954580916D06882352
:10A0000009F48DCF09C08CE990E50E9495458091B7
:10A010006D06882309F4A2CFDF91CF911F910F9194
:10A0200008952F923F924F925F926F927F928F92FC
:10A030009F92AF92BF92CF92DF92EF92FF920F93D7
:10A040001F93CF93DF9300D000D0CDB7DEB71C01B4
:10A050007E836D8329013A01460120E030E040E033
:10A0600057ECB201C3010F94EE4218162CF0412CAC
:10A07000512C612C27EC01C0272DB201862D922F87
:10A080000F945A412B013C0120E03EEF4FEF56E484
:10A09000B701C8010F94EB4087FD06C0B12C9EEFBD
:10A0A000F92E0FEF16E401C0BE2CC301B2010F94CC
:10A0B0008D419B01AC01ED81FE81608171818281C6
:10A0C00093810F9411400F945F4169837A838B834E
:10A0D0009C836B2D7F2DC8010F945A417B018C010D
:10A0E000E418F50806091709AF9287E9A82E8AE453
:10A0F000B82EC980DA80A30192016D817E81C101F1
:10A100000E94E0740F9026960FB6F894DEBF0FBE43
:10A11000CDBFDF91CF911F910F91FF90EF90DF9016
:10A12000CF90BF90AF909F908F907F906F905F90F7
:10A130004F903F902F9008956F927F928F929F92B1
:10A14000AF92BF92CF92DF92EF92FF920F931F9345
:10A15000CF93DF9300D01F92CDB7DEB761E081E0EF
:10A160000E9462766090A106712C61101AC08091E5
:10A17000A006811104C00E94727A811198C080915A
:10A180002202882309F48AC081E09091A0069111EF
:10A1900080E004E024E04AE45BE2672D0E94524143
:10A1A0007DC081E068122CC08091A006813021F42E
:10A1B0000E94727A811183C080912202882309F45F
:10A1C0006DC011E08091A006813009F010E080910F
:10A1D000070E9091080EA091090EB0910A0E898386
:10A1E0009A83AB83BC83CE0101960F94EB3500E0DC
:10A1F0009C0146E35BE2672D812F0E9486414EC0A1
:10A2000082E0681225C08091A006823021F40E946D
:10A21000727A811182C080912202882309F43EC0A3
:10A2200011E08091A006823009F010E060917B0C73
:10A2300070917C0C80917D0C90917E0C58DA00E03E
:10A240009C0142E25BE2672D812F0E94864126C07D
:10A2500083E0681223C08091A006833021F40E941D
:10A26000727A811172C0809122028823B9F011E0C4
:10A270008091A006833009F010E060917F0C70910E
:10A28000800C8091810C9091820C31DA00E09C016D
:10A2900042E15BE2672D812F0E94864173946394B3
:10A2A00085E0781262CF84E080939F0665C00E94AB
:10A2B0008C7580916D06882309F461CF5DC020E024
:10A2C00030E048EC52E46091070E7091080E8091E6
:10A2D000090E90910A0E0F9429430F945F411F922B
:10A2E000812C912C21E9A22E2AE4B22E6B01EE24BE
:10A2F000EA941FE7F12E00E010E020E030E0A90131
:10A3000067E07EE080E49BE20E94E0740F90809121
:10A310006D06882309F450CF2FC081E00E94677A30
:10A32000A12CC12CD12CE12CF12C08E413E420E069
:10A3300030E0A9016BE77CE08CE29BE272DE809169
:10A340006D06882309F467CF17C081E00E94677A01
:10A35000A12CC12CD12CE12CF12C08E413E420E039
:10A3600030E0A9016FE77CE08AE19BE25ADE809150
:10A370006D06882309F477CF0F900F900F900F9000
:10A38000DF91CF911F910F91FF90EF90DF90CF90D1
:10A39000BF90AF909F908F907F906F900895AF92F5
:10A3A000CF92DF92EF92FF920F931F93CF93DF93A1
:10A3B00061E081E00E946276D091A106C0E0D111F7
:10A3C0001AC08091A006811104C00E94727A811186
:10A3D00003C180912202882309F4F5C081E09091A5
:10A3E000A006911180E004E024E040E05BE26C2FE5
:10A3F0000E945241E8C0D13029F58091A0068130F9
:10A4000021F40E94727A8111EFC080912202882388
:10A4100009F4D9C011E08091A006813009F010E064
:10A420006091B90E7091BA0E8091BB0E9091BC0EE6
:10A430005ED900E09C0142EF5AE26C2F812F0E940E
:10A440008641C1C0D23029F58091A006823021F426
:10A450000E94727A8111E2C080912202882309F45D
:10A46000B2C011E08091A006823009F010E0609146
:10A47000BD0E7091BE0E8091BF0E9091C00E37D967
:10A4800000E09C0144EE5AE26C2F812F0E9486412D
:10A490009AC0D33029F58091A006833021F40E9420
:10A4A000727A8111D5C080912202882309F48BC071
:10A4B00011E08091A006833009F010E06091C10E98
:10A4C0007091C20E8091C30E9091C40E10D900E01D
:10A4D0009C0146ED5AE26C2F812F0E94864173C089
:10A4E000D43029F58091A006843021F40E94727A3C
:10A4F0008111C8C080912202882309F464C011E050
:10A500008091A006843009F010E06091C50E709132
:10A51000C60E8091C70E9091C80EE9D800E09C014C
:10A5200048EC5AE26C2F812F0E9486414CC0D530F6
:10A5300029F58091A006853021F40E94727A81115C
:10A54000BBC080912202882309F43DC011E08091B4
:10A55000A006853009F010E06091D50E7091D60EFE
:10A560008091D70E9091D80EC2D800E09C014EEB9E
:10A570005AE26C2F812F0E94864125C0D63019F5F2
:10A580008091A006863021F40E94727A8111ADC0BC
:10A59000809122028823B9F011E08091A0068630D4
:10A5A00009F010E06091D90E7091DA0E8091DB0E07
:10A5B0009091DC0E9CD800E09C014AEA5AE26C2F94
:10A5C000812F0E948641CF5FDF5FC53009F0F7CE53
:10A5D00087E080939F06A1C00E948C7580916D06D4
:10A5E000882309F4F6CE99C081E00E94677AA12CF5
:10A5F000C12CD12CE12C10ECF12E09E714E420E061
:10A6000030E040E85FE369EB7EE089EF9AE209DD44
:10A6100080916D06882309F4F8CE7FC081E00E9406
:10A62000677AA12CC12CD12CE12C10ECF12E09E77A
:10A6300014E420E030E040E85FE36DEB7EE08BEE79
:10A640009AE2EFDC80916D06882309F405CF65C09E
:10A6500081E00E94677AA12CC12CD12CE12C10EC56
:10A66000F12E09E714E420E030E040E85FE361EC1C
:10A670007EE08DED9AE2D5DC80916D06882309F4A9
:10A6800012CF4BC081E00E94677AA12CC12CD12C43
:10A69000E12C10ECF12E09E714E420E030E040E872
:10A6A0005FE365EC7EE08FEC9AE2BBDC80916D06A7
:10A6B000882309F41FCF31C081E00E94677AA12C62
:10A6C000C12CD12CE12C10ECF12E09E714E420E090
:10A6D00030E0A90165ED7EE083EC9AE2A2DC809196
:10A6E0006D06882309F42DCF18C081E00E94677A97
:10A6F000A12CC12CD12CE12C10ECF12E09E714E493
:10A7000020E030E0A90169ED7EE084EB9AE289DC8B
:10A7100080916D06882309F43BCFDF91CF911F9183
:10A720000F91FF90EF90DF90CF90AF9008956F92D0
:10A730007F928F929F92AF92BF92CF92DF92EF92D1
:10A74000FF920F931F93CF93DF9300D01F92CDB74B
:10A75000DEB761E081E00E9462766090A106712C14
:10A7600061101AC08091A006811104C00E94727A03
:10A770008111C2C080912202882309F4B5C081E012
:10A780009091A006911180E004E024E04CE15AE2AF
:10A79000672D0E945241A8C081E0681226C08091B6
:10A7A000A006813021F40E94727A8111ADC080919F
:10A7B0002202882309F498C011E08091A00681301C
:10A7C00009F010E06091650E7091660E8091670E41
:10A7D0009091680E0E94774B00E09C014CE05AE299
:10A7E000672D812F0E9486417FC082E0681226C0BB
:10A7F0008091A006823021F40E94727A81119EC05D
:10A8000080912202882309F46FC011E08091A00694
:10A81000823009F010E06091690E70916A0E8091AB
:10A820006B0E90916C0E0E94774B00E09C014CEFF8
:10A8300059E2672D812F0E94864156C083E068123D
:10A840002CC08091A006833021F40E94727A81117D
:10A850008FC080912202882309F446C011E08091C4
:10A86000A006833009F010E080916D0E90916E0E7D
:10A87000A0916F0EB091700E89839A83AB83BC83D5
:10A88000CE0101960F94A73800E09C014CEE59E2EE
:10A89000672D812F0E94864127C084E0681224C062
:10A8A0008091A006843021F40E94727A811198C0B0
:10A8B000809122028823C1F011E08091A0068430AB
:10A8C00009F010E06091710E7091720E8091730E1C
:10A8D0009091740E0E94774B00E09C014CED59E280
:10A8E000672D812F0E9486417394639485E07812CE
:10A8F00037CF70929F068DC00E948C7580916D0637
:10A90000882309F437CF85C081E00E94677AA12CA3
:10A91000C12CD12CE12C10E8F12E07E714E420E043
:10A9200030E040E85FE365E67EE084E19AE279DBCF
:10A9300080916D06882309F43ACF6BC081E00E94B4
:10A94000677AA12CC12CD12CE12C10E8F12E07E75D
:10A9500014E420E030E040E85FE369E67EE084E074
:10A960009AE25FDB80916D06882309F449CF51C0DC
:10A9700081E00E94677A20E030E048EC52E4609188
:10A980006D0E70916E0E80916F0E9091700E0F94FF
:10A99000294320E030E040E251E40F9411400F944D
:10A9A0005F411F92812C912C95EBA92E9AE4B92E30
:10A9B0006B0115EFE12E1FE7F12E00E010E02AE019
:10A9C00030E040E050E06DE67EE084EF99E20E94E6
:10A9D000E0740F9080916D06882309F43ACF19C076
:10A9E00081E00E94677AA12CC12CD12CE12C10E8C7
:10A9F000F12E07E714E420E030E040E85FE361E790
:10AA00007EE084EE99E20DDB80916D06882309F4E7
:10AA10004FCF0F900F900F900F90DF91CF911F911C
:10AA20000F91FF90EF90DF90CF90BF90AF909F90ED
:10AA30008F907F906F9008952F923F924F925F92E8
:10AA40006F927F928F929F92AF92BF92CF92DF923E
:10AA5000EF92FF920F931F93CF93DF93CDB7DEB7A3
:10AA600029970FB6F894DEBF0FBECDBF1C017987C2
:10AA70006887CA01B901E982FA820B831C83DE82EE
:10AA8000CD82AF8220E030E040E251E40F942943D0
:10AA90006B017C0120E030E040E057EC0F94EE4287
:10AAA00018162CF0C12CD12CE12C27ECF22EC7016A
:10AAB000B6010F945A412B013C0120E030E040E206
:10AAC00051E469817A818B819C810F9429434B01E8
:10AAD0005C0120E03EEF4FEF56E40F94EB4087FD22
:10AAE00007C0812C9EEF992EAA24AA9496E4B92E31
:10AAF00020E030E040E251E4E885F9856081718131
:10AB0000828193810F9429436B017C01C301B201BF
:10AB10000F948D419B01AC01C701B6010F94114008
:10AB20000F945F4169837A838B839C83C501B40151
:10AB30000F945A417B018C01E418F50806091709A6
:10AB4000FF81FF938D809E808BEBA82E8AE4B82E28
:10AB5000C980DA80A301920168857985C1010E94CC
:10AB6000E0740F9029960FB6F894DEBF0FBECDBFEC
:10AB7000DF91CF911F910F91FF90EF90DF90CF90D9
:10AB8000BF90AF909F908F907F906F905F904F900D
:10AB90003F902F9008959F92AF92BF92CF92DF92F5
:10ABA000EF92FF920F931F93CF93DF9300D01F92EA
:10ABB000CDB7DEB761E081E00E9462769090A10699
:10ABC000B12C91101AC08091A006811104C00E947E
:10ABD000727A8111D4C080912202882309F4C7C0FF
:10ABE00081E09091A006911180E004E024E04AEC1D
:10ABF00059E26B2D0E945241BAC081E098122CC0DC
:10AC00008091A006813021F40E94727A8111BFC028
:10AC100080912202882309F4AAC011E08091A00645
:10AC2000813009F010E08091A90E9091AA0EA091B8
:10AC3000AB0EB091AC0E89839A83AB83BC83CE01FB
:10AC400001960F94473900E09C0146EB59E26B2DC9
:10AC5000812F0E9486418BC082E098122CC0809187
:10AC6000A006823021F40E94727A8111ACC08091DA
:10AC70002202882309F47BC011E08091A006823073
:10AC800009F010E08091AD0E9091AE0EA091AF0E44
:10AC9000B091B00E89839A83AB83BC83CE010196B9
:10ACA0000F94473900E09C0142EA59E26B2D812F55
:10ACB0000E9486415CC083E098122CC08091A0065F
:10ACC000833021F40E94727A811199C0809122020E
:10ACD000882309F44CC011E08091A006833009F06C
:10ACE00010E08091B10E9091B20EA091B30EB09190
:10ACF000B40E89839A83AB83BC83CE0101960F94F3
:10AD0000473900E09C014EE859E26B2D812F0E94EB
:10AD100086412DC084E098122AC08091A00684301C
:10AD200021F40E94727A811186C0809122028823C8
:10AD3000F1F011E08091A006843009F010E08091DC
:10AD4000B50E9091B60EA091B70EB091B80E898352
:10AD50009A83AB83BC83CE0101960F94473900E000
:10AD60009C014AE759E26B2D812F0E948641B394E2
:10AD7000939485E0B81225CFB0929F0677C00E94C9
:10AD80008C7580916D06882309F425CF6FC081E012
:10AD90000E94677AA12C63ECC62E6AE4D62EE12CC1
:10ADA0001CE3F12E0CE116E420E030E040EA50E430
:10ADB00069EA7EE080EC99E23FDE80916D068823AF
:10ADC00009F426CF53C081E00E94677AA12C43EC9E
:10ADD000C42E4AE4D42EE12C1CE3F12E0CE116E43F
:10ADE00020E030E040EA50E46DEA7EE08CEA99E24F
:10ADF00023DE80916D06882309F439CF37C081E0C6
:10AE00000E94677AA12C23ECC22E2AE4D22EE12CD8
:10AE10001CE3F12E0CE116E420E030E040EA50E4BF
:10AE200061EB7EE088E999E207DE80916D06882378
:10AE300009F44CCF1BC081E00E94677AA12C83ECFF
:10AE4000C82E8AE4D82EE12C1CE3F12E0CE116E486
:10AE500020E030E040EA50E465EB7EE084E899E2EF
:10AE6000EBDD80916D06882309F45FCF0F900F9082
:10AE70000F900F90DF91CF911F910F91FF90EF9066
:10AE8000DF90CF90BF90AF909F9008950F93CF9396
:10AE9000DF9361E081E00E946276D091A106C0E07C
:10AEA000D1111AC08091A006811104C00E94727A4B
:10AEB00081118BC080912202882309F47EC081E039
:10AEC0009091A006911180E004E024E04BEB5BE25E
:10AED0006C2F0E94524171C0D130D9F48091A006EC
:10AEE000813021F40E94727A811177C08091220210
:10AEF000882309F462C081E09091A006913009F0A6
:10AF000080E003E02EE344EB5BE26C2F0E945241B1
:10AF100054C0D230D9F48091A006823021F40E942E
:10AF2000727A811164C080912202882309F445C09D
:10AF300081E09091A006923009F080E003E02EE3DA
:10AF40004DEA5BE26C2F0E94524137C0D330D1F4FE
:10AF50008091A006833021F40E94727A811151C041
:10AF600080912202882349F181E09091A0069330DC
:10AF700009F080E003E02EE346EA5BE26C2F0E94DA
:10AF800052411BC0D430C9F48091A006843021F412
:10AF90000E94727A81113FC080912202882369F059
:10AFA00081E09091A006943009F080E003E02EE368
:10AFB0004CE95BE26C2F0E945241CF5FDF5FC530EE
:10AFC00009F06ECFC0939F062FC00E948C758091B0
:10AFD0006D06882309F46ECF27C081ED9BE50E94A2
:10AFE000954580916D06882309F480CF1DC086EDBC
:10AFF0009BE50E94954580916D06882309F493CFC7
:10B0000013C08BED9BE50E94954580916D068823CA
:10B0100009F4A6CF09C080EE9BE50E94954580917A
:10B020006D06882309F4B8CFDF91CF910F91089571
:10B03000CF92DF92EF92FF92CF93C82F0E947E2B88
:10B040006B017C0124EA30E74DE75FE36091B806CD
:10B050007091B9068091BA069091BB060F94EB40AF
:10B0600087FD05C04AEF50E060E070E003C040E0BB
:10B0700050E0BA01C40ED51EE61EF71EC092B406FB
:10B08000D092B506E092B606F092B706C0932302BE
:10B09000CF91FF90EF90DF90CF9008952F923F9245
:10B0A0004F925F926F927F928F929F92AF92BF92D8
:10B0B000CF92DF92EF92FF921F93CF93DF93CDB7A2
:10B0C000DEB728970FB6F894DEBF0FBECDBF1C01C8
:10B0D000162F0E94727A882329F01092CF060E94C0
:10B0E0008C75DAC02091C7063091C8063E832D8347
:10B0F000232B09F49DC0E4E01E9FC0011124988712
:10B100008F83FC01E659FD4F80809180A280B3803F
:10B1100020E030E04AE754E4C501B4010F94114047
:10B120002B013C0120E030E04AE754E4C501B401C2
:10B130000F9412406B017C0180915F028823B9F16A
:10B14000113029F198F0123091F54090570250904B
:10B1500058026090590270905A02C0905B02D090E1
:10B160005C02E0905D02F0905E0221C040904702D8
:10B17000509048026090490270904A02C0904B0281
:10B18000D0904C02E0904D02F0904E0210C04090E2
:10B190004F02509050026090510270905202C09045
:10B1A0005302D0905402E0905502F09056022D8147
:10B1B0003E81B901330F880B990B0F948D4120917B
:10B1C000B8063091B9064091BA065091BB060F946B
:10B1D00029439B01AC01C501B4010F941240EF81DA
:10B1E000F885E659FD4F5F01608371838283938305
:10B1F0002D813E8137FF0CC0A30192010F94EB40DB
:10B2000087FF11C0F50140825182628273820BC0B8
:10B21000A70196010F94EE4218162CF4F501C08296
:10B22000D182E282F382812F03DF81E080932202C8
:10B230001092C8061092C70680912202882361F1FD
:10B2400024E0129FF0011124E659FD4F8081918185
:10B25000A281B38189839A83AB83BC832DEC3CECC0
:10B260004CEC5DE36091B8067091B9068091BA0626
:10B270009091BB060F94EE4287FD05C0CE0101966A
:10B280000F94B13605C060E2CE0101960F942937C4
:10B29000BC01C1010E94E74128960FB6F894DEBFB9
:10B2A0000FBECDBFDF91CF911F91FF90EF90DF9048
:10B2B000CF90BF90AF909F908F907F906F905F9056
:10B2C0004F903F902F90089560E080E49CE2E6CE9E
:10B2D00061E089E39CE2E2CE62E082E39CE2DECEC2
:10B2E000CF93DF9300D01F92CDB7DEB70E94727A62
:10B2F000882329F01092CF060E948C7557C0609168
:10B30000C7067091C8066115710569F1072E000C1A
:10B31000880B990B0F948D412091B8063091B90696
:10B320004091BA065091BB060F9429439B01AC0192
:10B330006091760270917702809178029091790203
:10B340000F94124060937602709377028093780294
:10B350009093790283E06CDE81E080932202109268
:10B36000C8061092C706809122028823F9F0209126
:10B370007F05309180054091810550918205609153
:10B3800076027091770280917802909179020F9401
:10B39000114069837A838B839C83CE0101960F943D
:10B3A000B136BC0184EC9BE20E94E7410F900F9004
:10B3B0000F900F90DF91CF91089521E02093CF0659
:10B3C0006093B8067093B9068093BA069093BB0653
:10B3D00020E040E060E070E080917D0590917E0586
:10B3E0000C945E7560E070E080E291E4E6CF60E08E
:10B3F00070E080E89FE3E1CF6DEC7CEC8CEC9DE3AA
:10B40000DCCF6DEC7CEC8CEC9CE3D7CFFF920F9300
:10B410001F93CF93DF93F82E70937E0560937D0585
:10B4200061E081E00E946276D091A106C0E091E0E7
:10B4300081E0F81659F1F81628F082E0F81609F4C0
:10B4400049C06CC0D111D1C0992389F08091A00668
:10B4500018166CF02091C7063091C8062F5F3F4F39
:10B460003093C8062093C7068F5F8093A006809113
:10B470002202882309F42EC100E010E021E041E01F
:10B480006BE27CE28C2F0E94EF4024C1D111ADC051
:10B49000992389F08091A00618166CF02091C706B8
:10B4A0003091C8062F5F3F4F3093C8062093C706E0
:10B4B0008F5F8093A00680912202882309F42AC11D
:10B4C00000E010E021E041E064E27CE28C2F0E9489
:10B4D000EF4020C1D11189C0992389F08091A00645
:10B4E00018166CF02091C7063091C8062F5F3F4FA9
:10B4F0003093C8062093C7068F5F8093A006809183
:10B500002202882309F404C100E010E021E041E0B8
:10B510006DE17CE28C2F0E94EF40FAC040917602F0
:10B5200050917702609178027091790240937F0583
:10B53000509380056093810570938205D11120C0DE
:10B54000992389F08091A00618166CF02091C70607
:10B550003091C8062F5F3F4F3093C8062093C7062F
:10B560008F5F8093A00680912202882349F000E03B
:10B5700010E021E041E063E17CE28C2F0E94EF408B
:10B5800083E0F81232C060912D0D70912E0D8091E4
:10B590002F0D9091300D2091F50C211126C00F94A4
:10B5A0005A41209135023091360262177307ECF44C
:10B5B000D130C9F48091A006813021F40E94727AC2
:10B5C0008111B2C080912202882369F081E09091BC
:10B5D000A006913009F080E004E024E043E05CE262
:10B5E0006C2F0E94524182E096C0D130D9F48091F4
:10B5F000A006813021F40E94727A81119DC0809151
:10B600002202882309F466C081E09091A00691305F
:10B6100009F080E004E024E049EF5BE26C2F0E9437
:10B62000524158C0D230D9F48091A006823021F422
:10B630000E94727A811188C080912202882309F4C5
:10B6400049C081E09091A006923009F080E003E0CB
:10B650002EE34FEE5BE26C2F0E9452413BC0D33091
:10B66000D1F48091A006833021F40E94727A811176
:10B6700075C080912202882369F181E09091A00633
:10B68000933009F080E003E02EE346EE5BE26C2F9E
:10B690000E9452411FC0D430E9F48091A00684304A
:10B6A00021F40E94727A811163C080912202882362
:10B6B00089F081E09091A006943009F080E003E0E9
:10B6C0002EE34BED5BE26C2F0E94524182E0F812B8
:10B6D00021C01EC082E0F8121DC0D530C9F480918F
:10B6E000A006853021F40E94727A81114BC08091AE
:10B6F0002202882369F081E09091A006953009F03C
:10B7000080E003E02EE34EEC5BE26C2F0E9452419E
:10B7100086E001C085E0CF5FDF5F90E0C53009F0D3
:10B7200087CE80939F0637C00E948C7580916D06EE
:10B73000882309F447CF2FC00E948C7580916D0635
:10B74000882309F45CCF27C082EF99E50E949545D4
:10B7500080916D06882309F46FCF1DC087EF99E5AE
:10B760000E94954580916D06882309F482CF13C00D
:10B770008CEF99E50E94954580916D06882309F428
:10B7800094CF09C081E09AE50E94954580916D06AD
:10B79000882309F4ACCFDF91CF911F910F91FF90D7
:10B7A00008954FEF64E679E580E030CE4FEF68E62C
:10B7B00079E581E02BCE4FEF6CE679E582E026CE8D
:10B7C0004FEF60E779E583E021CE0F93CF93DF93CE
:10B7D00061E081E00E946276D091A106C0E0D111C3
:10B7E0001AC08091A006811104C00E94727A811152
:10B7F0008BC080912202882309F47EC081E0909161
:10B80000A006911180E004E024E047E95BE26C2FA0
:10B810000E94524171C0D130D9F48091A00681308C
:10B8200021F40E94727A811177C0809122028823CC
:10B8300009F462C081E09091A006913009F080E0A7
:10B8400003E02EE34DE85BE26C2F0E94524154C0AE
:10B85000D230D9F48091A006823021F40E94727A0D
:10B86000811164C080912202882309F445C081E0DF
:10B870009091A006923009F080E000E22EE34FE7BD
:10B880005BE26C2F0E94524137C0D330D1F48091DB
:10B89000A006833021F40E94727A811151C08091F8
:10B8A0002202882349F181E09091A006933009F0AB
:10B8B00080E000E22EE341E75BE26C2F0E94524100
:10B8C0001BC0D430C9F48091A006843021F40E94BA
:10B8D000727A81113FC080912202882369F081E051
:10B8E0009091A006943009F080E000E22EE34CE550
:10B8F0005BE26C2F0E945241CF5FDF5FC53009F0E1
:10B900006ECFC0939F062FC00E948C7580916D06EC
:10B91000882309F46ECF27C086E497E50E949545F9
:10B9200080916D06882309F480CF1DC08CE89BE2CE
:10B930000E94DE7480916D06882309F493CF13C0B2
:10B940008BE79BE20E94DE7480916D06882309F4E8
:10B95000A6CF09C08DE69BE20E94DE7480916D0641
:10B96000882309F4B8CFDF91CF910F910895CF9339
:10B97000DF93EC01CB01BA010F948D410F945A4132
:10B9800079836883DF91CF91089567EB7CE58EE43E
:10B990009DE50C94A1750F931F93CF93DF9361E006
:10B9A00081E00E946276C091A106D0E081E0C111E1
:10B9B00022C0882389F08091A00618166CF020918F
:10B9C000C7063091C8062F5F3F4F3093C8062093BB
:10B9D000C7068F5F8093A00680912202882309F416
:10B9E00041C000E010E020E041E06AEA7DE28D2FF6
:10B9F0000E94EF4037C0C130D1F48091A006813061
:10BA000021F40E94727A811137C08091220288232A
:10BA100049F181E09091A006913009F080E000E2C8
:10BA20002EE34FE95DE26D2F0E9452411BC0C230F0
:10BA3000C9F48091A006823021F40E94727A8111AB
:10BA400022C080912202882369F081E09091A006B3
:10BA5000923009F080E000E22EE34BE85DE26D2FCA
:10BA60000E945241DF5FCF5F80E0D53009F09FCF69
:10BA700083E080939F060DC0C093830C80916D0678
:10BA8000882319F206C0C093830C80916D06882329
:10BA9000C1F2DF91CF911F910F9108950F948D41C5
:10BAA0000F945A41CB010D94B034EF92FF920F9353
:10BAB0001F93CF93DF93CDB7DEB72B970FB6F894D4
:10BAC000DEBF0FBECDBF7C0140918405842F042EC4
:10BAD000000C990B20918505223051F0233019F08C
:10BAE00029ED3DE20AC047FF06C025EE3DE205C054
:10BAF00027EF3DE202C02EEE3DE29F934F933F932E
:10BB00002F938E010F5F1F4F1F930F930F948D493B
:10BB100040913302509134024F50510997010F90D8
:10BB20000F900F900F900F900F904E155F050CF433
:10BB30009A013093320D2093310D80E00E94E6ACE3
:10BB4000C8010E944C772B960FB6F894DEBF0FBE4B
:10BB5000CDBFDF91CF911F910F91FF90EF9008958E
:10BB6000E091840587E1E802F0011124E75DF24FDE
:10BB7000808591859ACF7F928F929F92AF92BF924C
:10BB8000CF92DF92EF92FF920F931F93CF93DF93A9
:10BB9000782E809385056093840561E081E00E94A2
:10BBA0006276D091A106C0E081E0D1112EC0882339
:10BBB00089F08091A00618166CF02091C70630918C
:10BBC000C8062F5F3F4F3093C8062093C7068F5F8C
:10BBD0008093A00680912202882309F494C022E079
:10BBE000721649F033E0731203C06BEB7DE205C0BF
:10BBF0006BEA7DE202C06BEC7DE200E010E021E048
:10BC000041E08C2F0E94EF407EC0D130D9F480916A
:10BC1000A006813021F40E94727A81117DC080914A
:10BC20002202882309F46FC081E09091A006913030
:10BC300009F080E004E024E046E35EE26C2F0E941D
:10BC4000524161C0D230D9F48091A006823021F4F3
:10BC50000E94727A811168C080912202882309F4BF
:10BC600052C081E09091A006923009F080E000E29D
:10BC70002EE34AE25EE26C2F0E94524144C0D33070
:10BC8000D1F48091A006833021F40E94727A811150
:10BC900056C0809122028823B1F181E09091A006E4
:10BCA000933009F080E000E22EE34EE15EE26C2F7B
:10BCB0000E94524128C0D43031F58091A0068430D2
:10BCC00021F40E94727A811145C08091220288235A
:10BCD000D1F011E08091A006843009F010E02091AD
:10BCE000840537E12303F0011124E75DF24F8085DD
:10BCF00091850F94B03400E09C0140E05EE26C2F2F
:10BD0000812F0E948641CF5FDF5F80E0C53009F060
:10BD10004CCFC0939F065BC00E948C7580916D06CE
:10BD2000882309F47CCF53C080918C0590918D05B8
:10BD3000BCDE80916D06882309F48ECF48C08091C7
:10BD40008E0590918F05B1DE80916D06882309F4F0
:10BD5000A0CF3DC081E00E94677A0091840527E171
:10BD6000020380011124F801E75DF24F60857185BF
:10BD7000072E000C880B990B0F948D4120E030E0CA
:10BD800040EF52E40F9411400F945F41F801EF5CD3
:10BD9000F24F1F9280EB882E8DE5982E95ECA92E00
:10BDA0009CE5B92E6B011AEAE12EF12C00E010E0BF
:10BDB00028E730E040E050E0BF018FE09EE20E94C3
:10BDC000E0740F9080916D06882309F47ECFDF9197
:10BDD000CF911F910F91FF90EF90DF90CF90BF9088
:10BDE000AF909F908F907F90089560E081E0C3CEE8
:10BDF0008F929F92AF92BF92CF92DF92EF92FF927B
:10BE00000F931F93CF93DF934C015B016A0160E0B6
:10BE100085E00E946276D091A106F12C82E0E82EA6
:10BE2000D1111AC080912202882321F1809125022C
:10BE3000823041F0833019F460E67DE205C06EE4A3
:10BE40007DE202C060E77DE200E010E021E041E039
:10BE50008F2D0E94EF400EC0D13061F480912202FC
:10BE6000882341F000E010E020E041E0B4018F2D94
:10BE70000E94EF40A114B10481F0D23081F480918E
:10BE80002202882309F46EC000E010E020E041E0C7
:10BE9000B5018F2D0E94EF4065C0C2E001C0C3E034
:10BEA000C114D10491F0DC130FC0809122028823C9
:10BEB00051F000E010E020E041E0B6018F2D0E943B
:10BEC000EF40CD2F01C0CD2FCF5F21E030E0A11496
:10BED000B10411F420E030E081E090E0C114D1041D
:10BEE00011F480E090E0820F931F029781F0DC1341
:10BEF0000DC080912202882349F000E010E020E08C
:10BF000041E069E87DE28F2D0E94EF40CF5FDC13B6
:10BF100014C080912202882371F000E010E021E03B
:10BF200040E06EE77DE28F2D0E94EF406091830537
:10BF30008F2D0E948940E0922202F394DF5F85E01A
:10BF4000F8126ECFCF5FC0939F06DF91CF911F9104
:10BF50000F91FF90EF90DF90CF90BF90AF909F90A8
:10BF60008F900895C3E0C114D10409F0ADCFADCFD7
:10BF700040E050E060E070E083E49DE239CF4AE3C6
:10BF80005DE26AE27DE281E29DE232CF40E050E094
:10BF900061E17DE288E09DE22BCF40E050E069EF77
:10BFA0007CE28AEE9CE224CF40E050E06BED7CE244
:10BFB0008EEC9CE21DCF42EC5CE261EB7CE281EA1C
:10BFC0009CE216CF40E050E063E97CE28AE89CE224
:10BFD0000FCF40E050E06AE77CE28DE69CE208CFBC
:10BFE00040E050E060E67CE28FE59CE201CF40E07B
:10BFF00050E060E57CE287E49CE2FACE6111609358
:10C00000250240938305082E000C990BAA0BBB0B4D
:10C010008C309105A0F5FC018827EA56FF4F8F4F21
:10C020000D9473448FEB9FE51FC086EC9FE51CC009
:10C0300089EE9FE519C08BED9FE516C082EE9FE566
:10C0400013C087EF9FE510C080EF9FE50DC084ED22
:10C050009FE50AC08DEC9FE507C01092830C8BEC26
:10C060009CE502C088EB9FE5009749F021E0209312
:10C07000CF0620E040E060E070E00C945E750C9428
:10C080008575CF92DF92EF92FF920F931F938AE014
:10C09000C82E8FE2D82EE12CF12C0FEF1EE22CE8F7
:10C0A00035E743E950E86AEF7EE285EF9EE20E94C1
:10C0B0005A771F910F91FF90EF90DF90CF900895E6
:10C0C0009091AD0993FB882780F993FF06C081E02A
:10C0D0009091DD07911101C080E00895EF92FF92E9
:10C0E0000F931F93CF93DF9361E081E00E9462760C
:10C0F000C091A10610E0C11118C08091A006811165
:10C1000004C00E94727A8111C8C1809122028823E2
:10C1100061F081E09091A006911180E004E024E0BC
:10C1200049EE5EE2612F0E9452418091AD0982FB8F
:10C13000002700F982FD07C0D1E0909142179130AD
:10C1400019F0D0E001C0D02F83FBEE24E0F883FF8C
:10C1500003C0B6DFF82E01C0F12CDD2309F458C06E
:10C16000C130D9F48091A006813021F40E94727A06
:10C1700081119BC180912202882309F4A8C181E02A
:10C180009091A006913009F080E000E22EE34DEDA1
:10C190005EE2612F0E9452419AC1C230D9F480916F
:10C1A000A006823021F40E94727A811186C18091AA
:10C1B0002202882309F48BC181E09091A00692307D
:10C1C00009F080E003E02EE342ED5EE2612F0E9481
:10C1D00052417DC1C33009F063C08091A006833015
:10C1E00021F40E94727A811174C180912202882305
:10C1F00009F46DC181E09091A006933009F080E0D0
:10C2000003E02EE34DEC5EE2612F0E9452415FC1DC
:10C2100080914217823029F053DF8823F9F0011111
:10C220001DC0C130E9F48091A006813021F40E9444
:10C23000727A811158C180912202882309F45BC16E
:10C2400081E09091A006913009F080E000E22EE3B9
:10C2500040EC5EE2612F0E9452414DC1D1E001C02D
:10C26000D2E0CD131BC08091A0068C1304C00E94A5
:10C27000727A811142C180912202882371F081E09B
:10C280009091A0069C1380E003E02EE347EB5EE272
:10C29000612F0E945241DC2F01C0DC2FDF5F01C003
:10C2A000D4E0CD131BC08091A0068C1304C00E9463
:10C2B000727A81112CC180912202882371F081E071
:10C2C0009091A0069C1380E003E02EE34BEA5EE22F
:10C2D000612F0E945241DC2F01C0DC2F81E08D0FC5
:10C2E000C81318C08091A0068C1304C00E94727AF3
:10C2F000811117C180912202882361F081E0909121
:10C30000A0069C1380E003E02EE34DE95EE2612F7E
:10C310000E94524182E08D0F4091310D5091320DBB
:10C320009091F50C911107C02091350230913602A1
:10C3300042175307DCF0C81333C08091A0068C135A
:10C3400004C00E94727A8111F6C080912202882373
:10C3500039F181E09091A0069C1380E000E22EE389
:10C3600045E85EE2612F0E9452411AC0C81318C00E
:10C370008091A0068C1304C00E94727A8111E5C0DE
:10C3800080912202882361F081E09091A0069C13A5
:10C3900080E003E02EE345E75EE2612F0E94524118
:10C3A000DD5FCD1318C08091A0068C1304C00E94DD
:10C3B000727A8111D4C080912202882361F081E0D9
:10C3C0009091A0069C1380E003E02EE347E65EE236
:10C3D000612F0E94524191E09D0FEE2009F43BC075
:10C3E000F11053C0C91318C08091A0068C1304C06B
:10C3F0000E94727A8111BDC080912202882361F06F
:10C4000081E09091A0069C1380E000E22EE344E5D9
:10C410005EE2612F0E94524182E08D0FC81318C066
:10C420008091A0068C1304C00E94727A8111ABC067
:10C4300080912202882361F081E09091A0069C13F4
:10C4400080E003E02EE346E45EE2612F0E94524169
:10C4500093E09D0F1AC0C91316C08091A0068C13DB
:10C4600002C00E94727A80912202882361F081E0EA
:10C470009091A0069C1380E000E22EE34BE35EE285
:10C48000612F0E94524192E09D0F1F5FCF5F1530D8
:10C4900009F031CE90939F067FC00E948C758091E9
:10C4A0006D06882309F431CE77C00E94A680809162
:10C4B0006D06882309F45ECE6FC081E490E60E9489
:10C4C000954580916D06882309F471CE65C0D4E04E
:10C4D00005CF8AE294E60E94954580916D068823F7
:10C4E00009F483CE59C00E94B78080916D068823DD
:10C4F00009F4A1CE51C0D2E0D1CE85EE9BE50E94D9
:10C50000954580916D06882309F4B5CE45C081EB31
:10C5100096E60E94954580916D06882309F4CBCE5E
:10C520003BC08DEC93E70E94954580916D06882372
:10C5300009F4E0CE31C085E99EE20E94DE7480916C
:10C540006D06882309F401CF27C085EF9EE50E9480
:10C55000954580916D06882309F412CF1DC085E2B0
:10C5600096E60E94954580916D06882309F423CFB5
:10C5700013C083E69EE20E94DE7480916D068823DC
:10C5800009F43ACF09C08DE896E40E949545809160
:10C590006D06882309F44CCFDF91CF911F910F9145
:10C5A000FF90EF9008956091250D70E080E00C946D
:10C5B000FFA760917E0270917F02072E000C880B0E
:10C5C000990B0F948D412AE037ED43E25CE30F9421
:10C5D000294360937A0270937B0280937C0290934C
:10C5E0007D020895CF93DF93EC01CB01BA010F9444
:10C5F0008D410F945F416883DF91CF91089580E072
:10C600000C94E6AC62EF72E688E093E60C94A175B8
:10C610000F948D410F945F41862F0D943434EF9227
:10C62000FF920F931F93CF93DF9300D01F92CDB74C
:10C63000DEB7082F7B010E94727A882329F01092BE
:10C64000CF060E948C753BC06091C7067091C806EA
:10C650006115710551F01092C8061092C70681E06D
:10C6600080932202802F0E94F0A0809122028823D2
:10C6700031F184E0089F800111240B58114F609123
:10C680006D0C70916E0C072E000C880B990B0F949B
:10C690008D419B01AC01F8016081718182819381A0
:10C6A0000F94294369837A838B839C8360E2CE0154
:10C6B00001960F94C137BC01C7010E94E7410F905A
:10C6C0000F900F900F90DF91CF911F910F91FF90DE
:10C6D000EF90089565E87FE280E0A1CF6AE77FE20E
:10C6E00081E09DCF20E040E060E070E00E945E7558
:10C6F00081E08093CF0610926E0C10926D0C08951D
:10C700008AE693E6EFCF8EE693E6ECCF2F923F9248
:10C710004F925F926F927F928F929F92AF92BF9251
:10C72000CF92DF92EF92FF920F931F93CF93DF93FD
:10C73000CDB7DEB729970FB6F894DEBF0FBECDBFD9
:10C740001C017987688769011A830983EB82BA0122
:10C75000550F880B990B0F948D414B015C0120E024
:10C7600030E040E057EC0F94EE4218162CF0812C8C
:10C77000912CA12C27ECB22EC501B4010F945A4183
:10C780002B013C01B601DD0C880B990B0F948D41F8
:10C790004B015C0120E03EEF4FEF56E40F94EB407D
:10C7A00087FD07C0812C9EEF992EAA24AA9496E4B7
:10C7B000B92EE885F98560817181072E000C880B00
:10C7C000990B0F948D416B017C01C301B2010F9451
:10C7D0008D419B01AC01C701B6010F9411400F942C
:10C7E0005F416C837D838E839F83C501B4010F9469
:10C7F0005A417B018C01E418F50806091709FB81F1
:10C80000FF9389809A8085ECA82E8CE5B82ECC8089
:10C81000DD80A301920168857985C1010E94E074E1
:10C820000F9029960FB6F894DEBF0FBECDBFDF91F3
:10C83000CF911F910F91FF90EF90DF90CF90BF901D
:10C84000AF909F908F907F906F905F904F903F90B0
:10C850002F9008958F929F92AF92BF92CF92DF92C6
:10C86000EF92FF920F931F93CF93DF9361E081E0EC
:10C870000E946276D091A106C0E0D1111AC08091C9
:10C88000A006811104C00E94727A811121C1809199
:10C890002202882309F413C181E09091A00691112E
:10C8A00080E004E024E045E75FE26C2F0E94524103
:10C8B00006C1D13011F58091A006813021F40E948B
:10C8C000727A81110DC180912202882309F4F7C088
:10C8D00011E08091A006813009F010E0809164029F
:10C8E000909165020F94B03400E09C0149E65FE24C
:10C8F0006C2F812F0E948641E2C0D23011F58091C9
:10C90000A006823021F40E94727A8111FBC08091CE
:10C910002202882309F4D3C011E08091A00682305E
:10C9200009F010E08091310D9091320D0F94B034E8
:10C9300000E09C014BE55FE26C2F812F0E94864155
:10C94000BEC0D33011F58091A006833021F40E943F
:10C95000727A8111ECC080912202882309F4AFC061
:10C9600011E08091A006833009F010E080910B0D5A
:10C9700090910C0D0F94B03400E09C0143E55FE210
:10C980006C2F812F0E9486419AC0D43001F580918E
:10C99000A006843021F40E94727A8111DDC080915A
:10C9A0002202882309F48BC011E08091A006843014
:10C9B00009F010E08091250D0F94343400E09C01C3
:10C9C0004BE35FE26C2F812F0E94864178C0D53007
:10C9D00011F58091A006853021F40E94727A8111B0
:10C9E000DEC080912202882309F469C011E08091A1
:10C9F000A006853009F010E080917E0290917F02C0
:10CA00000F94B03400E09C0141E35FE26C2F812F72
:10CA10000E94864154C0D630D9F48091A006863059
:10CA200021F40E94727A8111CCC080912202882365
:10CA300009F445C081E09091A006963009F080E0AD
:10CA400003E02EE346E25FE26C2F0E94524137C0C2
:10CA5000D730D1F48091A006873021F40E94727AF9
:10CA60008111B9C080912202882349F181E090911F
:10CA7000A006973009F080E003E02EE34BE15FE28F
:10CA80006C2F0E9452411BC0D830C9F48091A0067F
:10CA9000883021F40E94727A8111A7C0809122020D
:10CAA000882369F081E09091A006983009F080E039
:10CAB00003E02EE34CE05FE26C2F0E945241CF5F17
:10CAC000DF5FC53009F0D9CE89E080939F0696C01C
:10CAD0000E948C7580916D06882309F4D8CE8EC093
:10CAE000E12C00E010E027EE33E04AE050E064E69D
:10CAF00072E08FE69FE20ADE80916D06882309F4DA
:10CB0000E2CE7CC081E00E94677AE12C0FEF12E652
:10CB100022E231E040E050E061E37DE082E69FE226
:10CB2000F5DD80916D06882309F4F1CE67C081E0C0
:10CB30000E94677AE12C03E31DEA2CE830E040E034
:10CB400050E06BE07DE087E59FE2E0DD80916D06DF
:10CB5000882309F400CF52C081E00E94677AC09018
:10CB6000250DD12C1F9283ED882E82E6982E92E01F
:10CB7000A92E93E6B92EE12CF12C8701EA9420E04E
:10CB800030E0A90165E27DE087E49FE20E94E07465
:10CB90000F9080916D06882309F401CF2FC0E12CFE
:10CBA00009ED12E627EE33E04AE050E06EE772E06E
:10CBB00086E39FE2ABDD80916D06882309F411CFF7
:10CBC0001DC080E893E60E94954580916D068823FC
:10CBD00009F42BCF13C083E893E60E94954580911A
:10CBE0006D06882309F43ECF09C088EC96E70E94C1
:10CBF000954580916D06882309F450CFDF91CF9140
:10CC00001F910F91FF90EF90DF90CF90BF90AF906A
:10CC10009F908F9008950E94727A882321F010923D
:10CC2000CF060E948C750C941D400E94727A882356
:10CC300041F020E040E060E070E08BE096E60E948A
:10CC40005E7561E080E00C94B33F0F93CF93DF9368
:10CC500061E081E00E946276D091A106C0E0D1112E
:10CC600017C08091A006811104C00E94727A8111C0
:10CC70004CC080912202882309F43EC081E090914B
:10CC8000A006911180E004E024E047EA5FE231C0B1
:10CC9000D130B9F48091A006813021F40E94727ADB
:10CCA00081113BC080912202882331F181E0909173
:10CCB000A006913009F080E003E02EE346E95FE250
:10CCC00018C0D530C9F48091A006853021F40E94A7
:10CCD000727A81112CC080912202882369F081E050
:10CCE0009091A006953009F080E003E02EE340E942
:10CCF0005FE26C2F0E945241CF5FDF5FC53009F0C9
:10CD0000AECF86E080939F061AC00E948C758091FA
:10CD10006D06882309F4ADCF12C085E196E60E9426
:10CD2000954580916D06882309F4BCCF08C08BEA35
:10CD300095E40E94954580916D06882361F2DF910C
:10CD4000CF910F91089560E070E080E00E94FFA70E
:10CD500060E070E081E00E94FFA70E9480AD0C942B
:10CD600085758F929F92AF92BF92CF92DF92EF9292
:10CD7000FF920F931F93CF93DF9361E081E00E94B6
:10CD80006276D091A106C0E0D1111AC08091A006B0
:10CD9000811104C00E94727A8111ABC0809122027D
:10CDA000882309F474C081E09091A006911180E07D
:10CDB00004E024E043EE5FE26C2F0E94524167C022
:10CDC000D13011F58091A006813021F40E94727A51
:10CDD000811197C080912202882309F458C011E084
:10CDE0008091A006813009F010E08091310D909182
:10CDF000320D0F94B03400E09C0145ED5FE26C2FE2
:10CE0000812F0E94864143C0D23009F58091A0064F
:10CE1000823021F40E94727A811199C0809122029D
:10CE20008823A9F111E08091A006823009F010E07A
:10CE300080910B0D90910C0D0F94B03400E09C018B
:10CE40004DEC5FE26C2F812F0E94864120C0D330D1
:10CE5000F1F48091A006833021F40E94727A81114E
:10CE60009BC080912202882391F011E08091A0065E
:10CE7000833009F010E08091250D0F94053400E017
:10CE80009C0145EB5FE26C2F812F0E9486418091CF
:10CE9000310D9091320D20910B0D30910C0D232B03
:10CEA00011F4892BE9F0D430C9F48091A0068430C4
:10CEB00021F40E94727A811192C08091220288230B
:10CEC00069F081E09091A006943009F080E000E2E2
:10CED0002EE34CEA5FE26C2F0E94524185E001C0D4
:10CEE00084E0CF5FDF5FC53009F04ECF80939F06AF
:10CEF0007CC00E948C7580916D06882309F44ECF0A
:10CF000074C081E00E94677AC090310DD090320DDC
:10CF10001F926FEF862E62E6962E75ECA72E7CE5AB
:10CF2000B72E12E2E12EFF24F39400E010E020E09F
:10CF300030E0A90161E37DE08CED9FE20E94E074A6
:10CF40000F9080916D06882309F444CF4EC081E094
:10CF50000E94677AC0900B0DD0900C0D1F9233E3A6
:10CF6000832E3DEA932E45ECA42E4CE5B42E1CE80E
:10CF7000E12EF12C00E010E020E030E0A9016BE0B0
:10CF80007DE081ED9FE20E94E0740F9080916D063C
:10CF9000882309F443CF29C081E00E94677AC090BA
:10CFA000250DD12C1F9283ED882E82E6982E98E9CC
:10CFB000A92E97E4B92EE12CF12C8701EA9420E008
:10CFC00030E0A90165E27DE081EC9FE20E94E0741F
:10CFD0000F9080916D06882309F443CF06C0B3DE1D
:10CFE00080916D06882309F468CFDF91CF911F915E
:10CFF0000F91FF90EF90DF90CF90BF90AF909F90F8
:10D000008F90089580E095E2909395058093940524
:10D010008CE491E0909391058093900580EC9EEFD5
:10D0200090939305809392059091990580E2890FE2
:10D03000863740F080EF890F20E431E0309393058C
:10D040002093920510929605809397058FEF809319
:10D05000980508958F929F92BF92CF92DF92EF92A0
:10D06000FF920F931F93CF93DF931F92CDB7DEB73D
:10D07000E1D7882309F4D6C18091C706863214F01F
:10D0800085E202C087FD80E0282F082E000C330BBC
:10D090003093C8062093C706982F990F890F809365
:10D0A00099058091E905882309F4BCC12091920576
:10D0B000309193050091960510919705020F131F6B
:10D0C000E0909405F09095058091900590919105E0
:10D0D000E80EF91E01304FE7140768F031952195ED
:10D0E000310930939305209392056CED70E085E053
:10D0F00090E00F94283BF7FE15C080919005909129
:10D100009105919581959109909391058093900552
:10D1100068E171E085E090E00F94283B81E0809326
:10D12000980517C081E0E81680E4F80694F06BE4F7
:10D1300070E084EF91E00F94283B8091A30581502B
:10D140008093A305882311F05DDF6CC11092E9057F
:10D1500069C12091900530919105C7019A508130A5
:10D16000934108F098C08F2D992787FD9A950A97CB
:10D1700065E070E00F942244812F17FF02C087E022
:10D18000810F482F45954595459581E090E0A0E0B9
:10D19000B0E004C0880F991FAA1FBB1F4A95D2F7A1
:10D1A000FB01EE0FFF1FE656FA4F408151818A01C5
:10D1B00008231923012B09F419C180959095842324
:10D1C00095239183808384E090E0861B970B4091A8
:10D1D000EA055091EB05840F951F9093EB05809322
:10D1E000EA058091A20581508093A205811103C0B8
:10D1F00082E08093E905932F9095991F9927991FB5
:10D2000080919805881F8827881F9817F1F031951D
:10D2100021953109309391052093900520E130E06C
:10D2200040E050E060EF7FEF8FEF9FEF0E941A36F3
:10D230002091920530919305620F731F70939305AF
:10D240006093920560E773E021C080919205909110
:10D2500093059195819591099093930580939205FB
:10D2600020E130E040E050E060EF7FEF8FEF9FEF94
:10D270000E941A362091900530919105620F731F1C
:10D28000709391056093900560E872E085E090E00E
:10D290000F94283BABC0121613060CF0A7C0FDE399
:10D2A000FF1A41E0E41642E0F40608F09FC08091C6
:10D2B0009905181B103108F099C031952195310955
:10D2C000309391052093900560E773E083E090E050
:10D2D0000F94283B8FEF8093980521E012300CF0DB
:10D2E00020E08EEF810F8C30A0F08091920590911C
:10D2F000930541E050E01816190614F040E050E0A4
:10D3000030E04217530709F055C091958195910976
:10D3100027C0143050F520E030E0A90160EC7FEF29
:10D320008FEF9FEF0E941A3620919205309193055E
:10D33000620F731F709393056093920561157E4F82
:10D3400034F480E09EEF9093930580939205809152
:10D350009205909193058130924064F180E092E0D3
:10D36000909393058093920525C01C301CF120E416
:10D3700030E040E050E060E070E0CB010E941A36FF
:10D380002091920530919305620F731F709393055E
:10D390006093920561157E4F34F480E09EEF909388
:10D3A0009305809392058091920590919305813029
:10D3B0009240A4F68091E9058230C1F480E4809324
:10D3C000A2058FEF9FEF90939B0580939A05909312
:10D3D0009D0580939C0590939F0580939E05909357
:10D3E000A1058093A00581E08093E9052091960531
:10D3F000309197058091920590919305820F931F2C
:10D40000909397058093960520919405309195050A
:10D410008091900590919105820F931F90939505AF
:10D420008093940561E083E494E00E94B1308091A0
:10D4300077048E3130F0809177048E3308F456C033
:10D440005AC0809179048A30B0F38AE9E82E85E0E9
:10D45000F82E9AE0892E912CB82C8091770490E0D8
:10D4600094012C5F3F4F281739075CF442E0E40E2B
:10D47000F11C85E0880E911CEEE18E16910461F797
:10D48000DACF80917904881588F330E0C12CD12C53
:10D49000F70180819181A0E0B0E00C2C04C0B6952A
:10D4A000A795979587950A94D2F780FD07C0FFEF5F
:10D4B000CF1ADF0A385F303859F7D8CF00E010E0D4
:10D4C000A801480D591D8091770490E0481759072D
:10D4D0003CF08091790490E0841795070CF055C0DA
:10D4E0000F5F1F4F0430110559F7E1CF8091790488
:10D4F0008C3308F055C08091E9058823B1F0809104
:10D500009505482F582F550F550B9A0133272F5F3C
:10D510003F4F8091770490E0281739073CF08091C5
:10D520007904841708F04DC001C09DD5809177041F
:10D530008B30D0F469E080E00E94B8378091EA0532
:10D540009091EB050E94BD3769E08EE60E94B837E6
:10D550002091A30583E090E0821B91096FEF7FEF9C
:10D560008851904D0E9412380E94727A882391F15E
:10D570000F90DF91CF911F910F91FF90EF90DF906F
:10D58000CF90BF909F908F90ABC527E04B2D400F61
:10D59000632F83E494E039830E94C2323981A0CFA3
:10D5A00020E14DE36091990583E494E00E94C2324A
:10D5B00020E14CE36091990583E494E00E94C2323B
:10D5C0009ACF6091970502E022E083E494E00E9404
:10D5D0000333ACCF0F90DF91CF911F910F91FF904C
:10D5E000EF90DF90CF90BF909F908F9008956AE268
:10D5F00078E682E064D588E38093990583E08093A0
:10D60000A30580E48093A205EAE9F5E01182108287
:10D61000138212821582148217821682F3DC82E151
:10D6200090E09093C8068093C70608958F929F92CA
:10D63000AF92BF92CF92DF92EF92FF92CF93709111
:10D64000BC05A7EBB5E020E030E090E080E0622F81
:10D65000CD902F5F3F4FC110722F8C296295607F54
:10D6600040E050E0D12CE12CF12C46015701042E72
:10D6700004C0B694A794979487940A94D2F780FE36
:10D6800008C0E92FF0E0E855FA4FC62FC42BC0833D
:10D690009F5F4F5F5F4F4530510539F723303105AC
:10D6A000B1F67093BC0540E050E020E090E0A0E0CF
:10D6B000B0E06C017D01042E04C0F694E794D79489
:10D6C000C7940A94D2F7C0FE05C02093BE052AE392
:10D6D00035E007C02E504F5F5F4F4530510549F789
:10D6E000F4CF422F3150A0F0225F6C017D01032E58
:10D6F00004C0F694E794D794C7940A94D2F7C0FE76
:10D70000F0CF4093BD058091BB05823069F403C022
:10D710002093BD05F8CF8091BF05181614F08CEF4B
:10D7200001C084E08093BF05CF91FF90EF90DF9020
:10D73000CF90BF90AF909F908F90089580E090E041
:10D74000FC01EE53FA4F128203968E319105C1F718
:10D7500008951092C1058AE08093C00583E080930C
:10D76000BF058FE08093BB05E7EBF5E08FE1808399
:10D77000818382835BDFE2CF1F93CF93DF93EC0142
:10D78000162FDCDF8091E6058093E30587E3809325
:10D79000E40586E08093E5056AE070E088EE93E0BA
:10D7A0000F94283B9091E70591509093E7059923BA
:10D7B00051F01092E20518831092E6051092C80607
:10D7C0001092C70601C01882DF91CF911F91089572
:10D7D0005F926F927F928F929F92AF92BF92CF9201
:10D7E000DF92EF92FF920F931F93CF93DF9384E02A
:10D7F000809322028091C906882309F467C2809130
:10D80000C7069091C8068E31910514F08DE190E025
:10D8100097FF02C080E090E09093C8068093C7060F
:10D82000880F991F880F991F2091E605422F022E1D
:10D83000000C550B4817590774F42D5FAC01421BBF
:10D84000510927FD5395423051051CF02093E60500
:10D8500002C08093E6052091E605422F022E000CBF
:10D86000550B841795077CF42350422F022E000C91
:10D87000550B481B590B423051051CF02093E6050F
:10D8800002C08093E6058091E905882309F41EC251
:10D890002091A605222349F09091A705920F90931D
:10D8A000A705933F14F41092A605823070F08150C2
:10D8B0008093E905823011F44CDF08C2843609F008
:10D8C00005C281E08093E90501C28091A5058F5FC3
:10D8D0008093A5054091BB0590E0242F30E035955D
:10D8E0002795281739070CF0ACC09091A40581E06A
:10D8F00089278093A4051092A505442309F4A1C0AB
:10D900009091BF058091C105890F2091BE058217B6
:10D9100024F02091BD052817D4F491959093BF056C
:10D920002091C0052B5F2093C0058093C105809195
:10D93000BC053AE08302C0011124820F911D27FD2E
:10D940009A95C99724F064E189EE95E015DF9091EE
:10D95000C1058091BF05890F8093C1058091BB05EA
:10D96000882309F46EC024E130E040E050E060E03C
:10D9700070E0CB010E941A36672B682B692B09F0E7
:10D9800060C0E4ECF5E0C0E0D0E08081811153C0DC
:10D99000CE01880F991FC80FD91FCE53DA4F209799
:10D9A00009F44FC02091BB0530E02F5F3F4F032E9D
:10D9B000000C440B550B60E070E0CB010E941A365E
:10D9C000FB01E855FA4F4081242F30E0B4E0359553
:10D9D0002795BA95E1F7F901E358FC4F808190E073
:10D9E0004F705091C1056EE0469F500D1124452F98
:10D9F000FC01E658FC4F5081450FFC01E958FC4FF3
:10DA000090819695842F890F88838091C0058250DC
:10DA10002F5F3F4F9AE0299F800D1124898322E0D8
:10DA200030E040E050E060E070E0CB010E941A3648
:10DA30006E5F6A8306C021963396CA30D10509F01D
:10DA4000A4CF9091E205992341F08091E105890FDF
:10DA50008093E10587FD1092E2058091E20588231D
:10DA600009F4A2C02091E105E091C0052E170CF445
:10DA70009BC0022E000C330B0E2E000CFF0BCF01AF
:10DA80004D96821793070CF48FC0E090E005CE2DE1
:10DA90000E2C000CDD0B1091C105CE01811B9109EC
:10DAA00017FD93956EE070E00F942244F62E6530DA
:10DAB00008F07AC02E1B3F0BC90102966AE070E0A5
:10DAC0000F942244062F633008F06EC0812C912CF5
:10DAD000540183940F2C04C0880C991CAA1CBB1CF5
:10DAE0000A94D2F7A62F660FBB0BBD0169547A4F7B
:10DAF000FB019081892F882109F456C0FD01E3586C
:10DB0000FC4FE0814E2F50E0812FFEE0FF9E800D04
:10DB100011249A0126583C4FF901F080F80EEF14B9
:10DB20000CF442C0FA01E958FC4F1081412F50E03B
:10DB30004F0D511DF7FC5A95C417D507ACF510923F
:10DB4000E205282D20952923FB01208323E030E0E6
:10DB50002A1B3B0B8091EA059091EB05280F391F9A
:10DB60003093EB052093EA056AE070E088E290E0EC
:10DB70000F94283B2091C005FAE00F9F200D11243F
:10DB8000912F96958F2D890F85508093E3052093D3
:10DB9000E40584E08093E5058091BB058150809386
:10DBA000BB05882321F042DDC4ECD5E011C084E13F
:10DBB0008093E905C3DDF8CFFE018291890F808350
:10DBC000803454F01882239625E0C23ED207E1F05B
:10DBD00098819923C1F3F0CF8733ACF3FE013297DC
:10DBE00020818091E605281774F3022E000C330B78
:10DBF000082E000C990B0A968217930724F368E706
:10DC000089EE95E0B9DDDFCF8091A605811124C0B2
:10DC100024EF31E040E050E060E070E0CB010E9492
:10DC20001A36672B682B692BB9F422E030E040E00C
:10DC300050E060E070E0CB010E941A36672B682B41
:10DC4000692B09F091C18FEF8093A605813009F40B
:10DC50008DC18FE78093A7058091E2058823B1F1FC
:10DC60008091A605882391F18091E105873074F5B4
:10DC70002091E0058091A705281744F1022E000CA1
:10DC8000330B082E000C990B0C9682179307F4F0B7
:10DC90001092A6051092E2058091EA059091EB059D
:10DCA0000A969093EB058093EA056AE070E088E2BB
:10DCB00090E00F94283B8091A7058F5F8093E30548
:10DCC00081E08093E40584E08093E5058091D106AE
:10DCD00082FF04C08091BA05815001C08AE0809320
:10DCE000BA050E94727A8823C1F08091E9058111FA
:10DCF00003C01092BA0511C0813079F48091E20519
:10DD000081110BC08091E6058B5F8093E00584E371
:10DD10008093E1058CEF8093E2058091BA05811133
:10DD200001C0DED161E083E494E00E94B130C09193
:10DD3000C0054C2F0C2E000C550B8091BC059A0190
:10DD40006AE08602200D311D112422503109809194
:10DD5000770490E0821793072CF08091A60581113B
:10DD600065C069C08091790490E084179507ACF391
:10DD70007DE7672E73E0772EE7EB8E2EE5E09E2E93
:10DD8000FEE15F2E5C0EF301C1903F012C2F0C2EA3
:10DD9000000C330BA901495F5F4F8091770490E03D
:10DDA000481759073CF4C65FFFEF8F1A9F0AC51149
:10DDB000EACFD3CF8091790490E0821793079CF348
:10DDC000D091C10516E41D0FA12CB12CD12CCC0C87
:10DDD000DD1CF401808190E0A0E0B0E00A2C04C0DA
:10DDE000B695A795979587950A94D2F780FF17C0A7
:10DDF0008091A4057601E80EF11CC70164E0880F4C
:10DE0000991F6A95E1F79C01255E3F4C790108E076
:10DE100022E04C2F6D2F83E494E00E94DB30D25F30
:10DE20003FEFA31AB30AD113D4CFBDCF80917704AB
:10DE3000883008F49DC08091E905882369F09091AD
:10DE400077049F3348F490917904973328F0823017
:10DE500008F49CC081FD9AC08091E2058823B1F04E
:10DE60004091E105242F042E000C330BB9016D5FA6
:10DE70007F4F8091770490E0681779073CF080919C
:10DE8000790490E0821793070CF08EC0C0E0D0E0D8
:10DE9000FE01EE53FA4F8281882399F04181842F4D
:10DEA000042E000C990B2091770430E08217930721
:10DEB00044F002972091790430E0281739070CF0DC
:10DEC0007BC02396CE31D10519F78091E5058823D3
:10DED000B1F04091E405242F042E000C330BB9015E
:10DEE0006A5F7F4F8091770490E0681779073CF074
:10DEF0008091790490E0821793070CF065C08091BF
:10DF0000E905811101C0AFD0809177048A3008F013
:10DF10006DC069E080E00E94B8378091EA05909179
:10DF2000EB050E94BD378091E705882309F45EC0A8
:10DF3000C1E040E1C42ED12C8091E7058C1708F494
:10DF400055C0B6016C1B7109660F660F660F56E06F
:10DF5000E52E50E3F52E05E021E041E083E494E076
:10DF60000E94DB30CF5FE8CF81E06ECE83EF72CED0
:10DF70002EEEE22E2FE2F22E05E022E042E060914A
:10DF8000A70583E494E00E94DB3055CF9BE0E92EA7
:10DF900090E3F92E08E022E047E36091E60583E490
:10DFA00094E00E94DB3058CF24E06091E00583E4E8
:10DFB00094E00E94E2326ACF425023E0608183E421
:10DFC00094E00E94E2327DCF88EFE82E8FE2F82EB7
:10DFD00007E022E06091E30583E494E00E94DB30F7
:10DFE0008091E50581508093E50589CFDF91CF9140
:10DFF0001F910F91FF90EF90DF90CF90BF90AF9067
:10E000009F908F907F906F905F90089568EE7BE671
:10E0100084E155D083E08093E7058AE08093BA05D8
:10E020001092E20596DB1092E6051092C806109257
:10E03000C70608958091C906882319F082E080936D
:10E04000E80584E0809322028091E905882349F065
:10E050009091E8058FEF890F8093E80581E019160C
:10E060000CF080E008950F9380917704853228F5B5
:10E07000809179048B3108F160E083E494E00E94A0
:10E08000B13009E028E34BE164E283E494E00E94CC
:10E09000533361E083E494E00E94B1300E94BB7B83
:10E0A000882359F063E285E20E94B8376FEF7FEF73
:10E0B0008BE790E30F910C9412380F910895FB01B8
:10E0C0001092EB051092EA058093E90520E040E00C
:10E0D00060E070E0CF01F2D481E08093CF06089534
:10E0E0001092CF0619C58091EC059091EE05891329
:10E0F0000DC08091ED059091EF05891714F02FEF79
:10E1000001C021E0820F8093ED0508C0891714F04B
:10E110002FEF01C021E0820F8093EC05891319C015
:10E120002091500621502093500630E0832F90E03C
:10E13000DC01AA0FBB1FA451BA4F880F991FFC0125
:10E14000E251FA4F808191818D939C933F5F231719
:10E1500068F70895EF92FF921F93CF93DF9310918A
:10E16000500620915706E22E022E000CFF08309137
:10E170005806C32F032E000CDD0BEFEEF5E040E058
:10E18000411709F446C0CF010397DC019C91BF0100
:10E1900061507109DB018C9198131DC0692F092E04
:10E1A000000C770B61507109C617D70711F03913AE
:10E1B0002DC09081BF0162507109DB018C91582FF5
:10E1C00098170CF4592F25170CF189170CF4892F87
:10E1D0008217E4F020C0BF0162507109DB015C913D
:10E1E000652F052E000C770B61507109E616F706B6
:10E1F00011F025130BC0582F98170CF4592F351711
:10E200002CF089170CF4892F83172CF44F5F32966A
:10E21000B7CF80E001C081E0DF91CF911F91FF90E7
:10E22000EF90089528E130E040E050E060E070E0D9
:10E23000CB010E941A36609358062AE030E040E095
:10E2400050E060E070E0CB010E941A366093570600
:10E2500081DF8111E7CF089590915906811102C0A5
:10E260008FEF01C081E0980F937090935906E09171
:10E270005006EF5FE0935006F0E0EE0FFF1FE45111
:10E28000FA4F8091540680838091520681830895CD
:10E29000CF9380E091E0909354068093530680E002
:10E2A00095E0909352068093510610925906109271
:10E2B0005006ECEEF5E01082C5E0C18381E0CCDFD2
:10E2C000C09356061092C8061092C70610925506C3
:10E2D000CF910895EF92FF920F931F93CF93DF9307
:10E2E00080915006843008F4B1C090E0FC01EE0F3C
:10E2F000FF1FE651FA4F2081EC01CC0FDD1FC45106
:10E30000DA4F68810297261719F0F12C31966BC00D
:10E31000E12C219631964E2D50E0481759070CF00C
:10E3200095C0BA01660F771F8B0104511A4FD801AF
:10E33000FC90DB01A251BA4F3C91F316E9F0432F58
:10E34000F3160CF44F2D24179CF13F150CF43F2DC0
:10E35000321774F1DB01A451BA4F11965C9141E080
:10E36000308153170CF040E031E0688165170CF400
:10E3700030E04317E9F06CC02F111AC0688140816A
:10E3800011965C91D80111963C91A42F64170CF45E
:10E39000A62F732F35170CF4752F7A174CF04617EC
:10E3A0000CF4462F53170CF4352F43170CF050C0C4
:10E3B000E394B1CFEA01CC0FDD1F8E0104511A4F57
:10E3C000D80111967C91DE01A251BA4F11963C9171
:10E3D0001197731709F14081532F73170CF4572FBE
:10E3E00045173CF4F3944F2D50E04817590714F3A8
:10E3F0002DC037170CF4372F3417A4F3C451DA4F5C
:10E40000588141E052170CF040E031E065170CF400
:10E4100030E0431739F31CC030813713E3CF4C9100
:10E42000D8013C91762F26170CF4722F532F3417F6
:10E430000CF4542F5717B4F2562F62170CF4522FC6
:10E4400043170CF4342F53176CF202C080E001C064
:10E4500081E0DF91CF911F910F91FF90EF90089590
:10E46000CF92DF92EF92FF920F931F93CF93DF93A0
:10E470001F92CDB7DEB7DEDD882309F480C080911E
:10E48000530690915406392F4091510650915206EF
:10E4900020915906213061F02CF4211116C0CA01D7
:10E4A000C3970AC0223031F0233079F4C39709C0F2
:10E4B000C39607C0CA01C396909352068093510633
:10E4C00004C0909354068093530610915406009113
:10E4D0005206311303C0051709F451C0183110F466
:10E4E0000A3048F01092E90568E270E080E991E0B6
:10E4F0000F94283B44C0E0915006F0E0EE0FFF1F60
:10E50000E451FA4F108301838091C706909155061C
:10E51000282F291B39F08093550681E012160CF044
:10E5200080E09ADE80915606882321F08150809306
:10E53000560601C0D8DDCEDE8111D4CF80915806B9
:10E5400018131DC080915706081319C06CED70E0B8
:10E5500085E090E00F94283B68E171E085E090E071
:10E560000F94283B8091EA059091EB0501969093DA
:10E57000EB058093EA0582E08093560653DE61E066
:10E5800083E494E00E94B13080917704893050F4A4
:10E5900067E080E00E94B8378091EA059091EB0532
:10E5A0000E94BD3706E32CE749E062E083E494E093
:10E5B0000E940333F12C8091500620917704F816C5
:10E5C00008F071C0EF2DF0E0AF01440F551FDA01E4
:10E5D000A451BA4F9C91FA01E251FA4F80819813ED
:10E5E00045C091811196EC901E2DE9160CF4192F5F
:10E5F00085E01802B0011124625F7F4F30E062179E
:10E6000073070CF44EC09E150CF4E92E9E2DE5E028
:10E610009E0290011124265F3F4F8091790490E083
:10E6200028173907F4F58E2D880F880F8E0D7BE0A3
:10E63000780FCA0184519A4F6C011E1594F1272F4F
:10E64000072E000C330BA9014D5F5F4F80917704BB
:10E6500090E0481759073CF08091790490E08217C8
:10E6600093070CF04CC0E3947B5FE7CF11963C918D
:10E67000432F440F440F340F4BE0D42ED30E4D2DB7
:10E680000D2C000C550BBA016D5F7F4F30E0621707
:10E6900073073CF02091790430E0241735070CF023
:10E6A0003FC0F39488CF40915706842F880F880F7E
:10E6B000480F455F642F042E000C770BFB01339647
:10E6C000822F90E0E817F9073CF08091790490E000
:10E6D000861797070CF043C08091E905811101C0AE
:10E6E000C2DC00D7882309F448C00F90DF91CF9196
:10E6F0001F910F91FF90EF90DF90CF90F1CCF6013A
:10E700006081862F880F880F680F6C5F04E024E01B
:10E71000472F83E494E079830E9453337981A3CF18
:10E72000E82E98170CF4E92EC82E89170CF4C92E80
:10E730001E2D110F110F1E0D50E01C5FCE140CF496
:10E74000B0CF612F650F04E024E04D2D83E494E009
:10E7500059830E945333E39459815B5FEFCF6091FB
:10E760005806862F880F880F680F6C5F04E024E03E
:10E7700083E494E00E940333AFCF0F90DF91CF91F9
:10E780001F910F91FF90EF90DF90CF90089560E37D
:10E7900072E781E094DC7CDD45CD0F931F93CF932E
:10E7A000DF9361E081E08ED2D091A106C0E0D1116B
:10E7B00016C08091A006811103C094D681119AC021
:10E7C00080912202882309F43CC081E09091A00648
:10E7D000911180E004E024E044ED50E32FC0D130FB
:10E7E000B1F48091A006813019F47CD6811189C0E2
:10E7F00080912202882329F181E09091A006913036
:10E8000009F080E003E02EE342EC50E317C0D23081
:10E81000C1F48091A006823019F464D681117BC0C6
:10E8200080912202882369F081E09091A0069230C5
:10E8300009F080E003E02EE343EB50E36C2F0E94ED
:10E84000524125D1182FD330D1F48091A0068330C6
:10E8500019F448D6811169C080912202882309F4F5
:10E8600076C081E09091A006933009F080E000E24C
:10E870002EE344EA50E36C2F0E94524168C081119C
:10E8800068C0D430B1F48091A006843019F42AD63F
:10E89000811152C080912202882319F181E0909168
:10E8A000A006943009F080E000E22EE346E950E350
:10E8B00015C0D530B1F48091A006853009F443C06D
:10E8C00080912202882369F081E09091A006953022
:10E8D00009F080E000E22EE345E850E36C2F0E944F
:10E8E000524186E0CF5FDF5FC53009F060CF809393
:10E8F0009F063AC011D180916D06882309F460CF3C
:10E9000033C086EE9EE40E94954580916D06882373
:10E9100009F46ECF29C088EC96E70E949545809156
:10E920006D06882309F47CCF1FC0BED280916D068E
:10E93000882309F491CF18C0BAD280916D0688233C
:10E9400009F4A8CF11C0CED5811105C0B9CF1123CC
:10E9500041F284E0C7CF0E946ACE81E005D2809167
:10E960006D06882309F4ACCFDF91CF911F910F91F1
:10E970000895E0916E06E63000F581E08E0F8093F9
:10E980006E068091C7069091C806A0E0B0E0309175
:10E99000A10620919F0648E0E49FF0011124E1596F
:10E9A000F94F4091C2065091C30651834083828340
:10E9B0009383A483B5833683278308950D94D42845
:10E9C0002F923F924F925F926F927F928F929F927F
:10E9D000AF92BF92CF92DF92EF92FF920F931F936D
:10E9E000CF93DF9300D000D0CDB7DEB71C012B83CF
:10E9F0003C834D835E8369837A83BBDF83E08093AE
:10EA0000220230926C0620926B0669817A817093A3
:10EA10006A06609369062B813C814D815E8120935B
:10EA20006506309366064093670650936806E09249
:10EA30006106F09262060093630610936406D0921A
:10EA4000C806C092C706B092C306A092C2069092B2
:10EA5000600680925F068C8D80935E0626960FB6C8
:10EA6000F894DEBF0FBECDBFDF91CF911F910F9104
:10EA7000FF90EF90DF90CF90BF90AF909F908F90DE
:10EA80007F906F905F904F903F902F90089580916E
:10EA9000E30E9091E00E891B8F7071F49091AD0997
:10EAA00092FB882780F992FD08C081E0909142177F
:10EAB000913019F080E0089581E00895E091C20658
:10EAC000F091C306E817F907F9F09093C306809315
:10EAD000C2067093C8066093C7064093A1062093B0
:10EAE0009F06825D994721F41092CF0610926E0620
:10EAF0000E94884082E08093220281E080936D062C
:10EB00001092CA0610925A06089520E040E060E094
:10EB100070E082ED99E7D2CFE0916E06EE2381F0AE
:10EB2000E150E0936E0688E0E89FF0011124E1597E
:10EB3000F94F2781468160E070E080819181BECFEE
:10EB4000E4CFCF93DF93FC01EB018091C706909156
:10EB5000C80697FF04C01092C8061092C7064091DD
:10EB6000610650916206609163067091640680911F
:10EB7000C7069091C806092E000CAA0BBB0B4817BC
:10EB800059076A077B0724F45093C8064093C706C9
:10EB9000809122028823D1F02091C7063091C806C7
:10EBA0008091650690916606A0916706B09168060F
:10EBB000BC01CD01620F731F811D911D1995BC0110
:10EBC00080916B0690916C060E94E7418091BC0693
:10EBD000811108C080915E06882381F18091220214
:10EBE000882361F18091690690916A06009791F0FF
:10EBF0002091C7063091C80640916506509166067F
:10EC00006091670670916806420F531F611D711D68
:10EC1000FE011995E0915F06F0916006309741F092
:10EC200080915E06811103C08091BC068111199507
:10EC300059D4882319F0DF91CF916ECFDF91CF9116
:10EC400008950F931F93CF93DF938091220288231F
:10EC500059F060915B0670915C0600E010E020E0E6
:10EC600041E081E00E94EF4080915D0681111CC06F
:10EC700081E080935D06C091C206D091C30620E07A
:10EC800040E060E070E081E296E718DF0E94FCE877
:10EC900010925D0620E040E060E070E0CE01DF9180
:10ECA000CF911F910F910ACFDF91CF911F910F91BB
:10ECB0000895009711F488EE90E390935C0680939A
:10ECC0005B06BFCF282F1092C1068091C706909196
:10ECD000C8068130904820F01092C8061092C706EE
:10ECE0008091C906882331F08091C7068093A006E1
:10ECF00010926D0680919F061816BCF4082E000C29
:10ED0000990B821B91092091A006022E000C330B57
:10ED10002817390754F097FF02C080E090E08093F5
:10ED2000A0069093C8068093C7068091A00666232C
:10ED3000C1F09091A106891714F48093A106209147
:10ED4000A106022E000C330B2C5F3F4F482F082EDC
:10ED5000000C550B2417350734F484508093A1061A
:10ED600008958093A1060895882361F063E972E015
:10ED700084E690E00F94283B6AEB72E084E690E032
:10ED80000D94283B68EB71E084E190E00D94283B02
:10ED9000CF92DF92EF92FF92CF93DF93A3D388239A
:10EDA00059F00E945CCA1092CF06DF91CF91FF907C
:10EDB000EF90DF90CF90B0CE81E08093CF06C091EE
:10EDC000C706D091C806209709F442C01092C80621
:10EDD0001092C706BE010D2E000C880B990B0F94E4
:10EDE0008D4120917D0E30917E0E40917F0E50918D
:10EDF000800E0F9429432091BE0D3091BF0D40919C
:10EE0000C00D5091C10D0F9412406B017C0120E0A8
:10EE100030E040E050EC0F94EE4287FD19C020E056
:10EE200030E040EA50E4C701B6010F94EB401816F9
:10EE30007CF0BE0182E00E94F0A0C092BE0DD09294
:10EE4000BF0DE092C00DF092C10D82E080932202CE
:10EE5000809122028823C9F08EEB9DE00F944D35FE
:10EE6000BC0189ED90E30E94E7416091BE0D709175
:10EE7000BF0D8091C00D9091C10DDF91CF91FF909A
:10EE8000EF90DF90CF900C941643DF91CF91FF90DD
:10EE9000EF90DF90CF90089521E020935D060F94CE
:10EEA000D92810925D0608950E9497CA5DCF0E94EE
:10EEB0000ED95ACF4F925F926F927F928F929F920C
:10EEC000AF92BF92CF92DF92EF92FF920F931F9378
:10EED000CF93DF931F921F92CDB7DEB72C014A016B
:10EEE00039015801870176012091C7063091C80683
:10EEF0002115310559F081E0121613060CF080E05F
:10EF000080935A061092C8061092C70669837A83C6
:10EF1000E9D2D82E69817A81811104C080912202C0
:10EF2000882311F1950140915A06C2010E94BA420C
:10EF3000DD20D1F080915A06882311F0F40101C040
:10EF4000F3010F900F90DF91CF911F910F91FF90E0
:10EF5000EF90DF90CF90BF90AF909F908F907F9079
:10EF60006F905F904F9019940F900F90DF91CF9119
:10EF70001F910F91FF90EF90DF90CF90BF90AF90D7
:10EF80009F908F907F906F905F904F900895FC01BD
:10EF900080810895FC01849108954F925F926F9251
:10EFA0007F928F929F92AF92BF92CF92DF92EF9219
:10EFB000FF920F931F93CF93DF936C017B015A0154
:10EFC0002901672B31F088248394912CC0E0D0E094
:10EFD00019C0F8011182108227C03701680C791C12
:10EFE00076946794E3012197A201BE01C601F50161
:10EFF00019951816190654F0892BC9F04301FFEF33
:10F000008F1A9F0AE814F90440F702C07E01FACF74
:10F01000CE15DF0530F4CE0102968816990620F051
:10F020002196F801D183C0838FEF9FEF05C0F801CF
:10F03000D183C08380E090E0DF91CF911F910F9149
:10F04000FF90EF90DF90CF90BF90AF909F908F9008
:10F050007F906F905F904F9008958F929F92AF92A4
:10F06000BF92CF92DF92EF92FF920F931F93CF93B5
:10F07000DF93EC016B017A01FB01199587FD06C056
:10F08000082F10E020E030E0219620C1982F907EDC
:10F09000903CC1F4082F0F7110E020E030E04801EF
:10F0A000590186E0880C991CAA1CBB1C8A95D1F7D3
:10F0B000CE010196F60119958F7395018401082BF5
:10F0C000229604C1982F907F903E19F58F70882E5C
:10F0D000912CA12CB12C16E0880C991CAA1CBB1CED
:10F0E0001A95D1F7CE010196F60119958F73882AEA
:10F0F00006E0880C991CAA1CBB1C0A95D1F7CE010E
:10F100000296F60119958F7395018401082B2396B9
:10F11000DDC0982F987F903F81F58770882E912CC5
:10F12000A12CB12CF6E0880C991CAA1CBB1CFA95EA
:10F13000D1F7CE010196F60119958F73882AA6E0C2
:10F14000880C991CAA1CBB1CAA95D1F7CE0102966B
:10F15000F60119958F73882AB6E0880C991CAA1CB1
:10F16000BB1CBA95D1F7CE010396F60119958F73A2
:10F1700095018401082B2496A9C0982F9C7F983F65
:10F18000E9F58370882E912CA12CB12C56E0880CC7
:10F19000991CAA1CBB1C5A95D1F7CE010196F60109
:10F1A00019958F73882A66E0880C991CAA1CBB1CD1
:10F1B0006A95D1F7CE010296F60119958F73882AC8
:10F1C00076E0880C991CAA1CBB1C7A95D1F7CE015D
:10F1D0000396F60119958F73882AE6E0880C991C2E
:10F1E000AA1CBB1CEA95D1F7CE010496F60119952D
:10F1F0008F7395018401082B259668C0982F9E7FF8
:10F200009C3F09F04AC08170882E912CA12CB12C12
:10F2100086E0880C991CAA1CBB1C8A95D1F7CE01EC
:10F220000196F60119958F73882A96E0880C991C2F
:10F23000AA1CBB1C9A95D1F7CE010296F60119952E
:10F240008F73882A26E0880C991CAA1CBB1C2A955F
:10F25000D1F7CE010396F60119958F73882A36E00F
:10F26000880C991CAA1CBB1C3A95D1F7CE010496B8
:10F27000F60119958F73882A46E0880C991CAA1C00
:10F28000BB1C4A95D1F7CE010596F60119958F73EF
:10F2900095018401082B269619C0982F907C9038F0
:10F2A00049F4082F007C003871F42196CE01F60154
:10F2B0001995F7CF082F0E7F0D3F28F02196CE012C
:10F2C000F6011995F7CF00E010E09801E114F10480
:10F2D00029F0F7010083118322833383CE01DF916C
:10F2E000CF911F910F91FF90EF90DF90CF90BF9043
:10F2F000AF909F908F9008951F93CF93DF9300D08E
:10F300001F92CDB7DEB710E0AE014F5F5F4F67ECE5
:10F3100077E7A3DE49815A816B817C81452B462B9F
:10F32000472B11F01F5FF0CF812F0F900F900F90A0
:10F330000F90DF91CF911F9108951F93CF93DF938B
:10F3400000D01F92CDB7DEB710E0AE014F5F5F4F28
:10F350006AEC77E782DE49815A816B817C81452B9B
:10F36000462B472B11F01F5FF0CF812F0F900F908E
:10F370000F900F90DF91CF911F910895FC01A08114
:10F38000B1811C92A281B3818C918F5F8C9302809A
:10F39000F381E02D80816CE0689F600D112480E096
:10F3A0000C94B8371092C1068091BC061092BC062E
:10F3B000882349F020E040E060E070E08EE690E6CF
:10F3C0007DDB0C94534020916402309165024091A2
:10F3D000C7065091C806C901840F951F2436310510
:10F3E00051F44730510514F0069720C04A3F5F4F53
:10F3F00064F506961BC02436310524F48536910544
:10F4000024F504C08436910524F41FC08A30910588
:10F410003CF0883E43E094072CF087EE93E002C076
:10F420008AE090E02817390731F40DC08A30910541
:10F4300084F78AE090E090936502809364021092D2
:10F44000C8061092C7060C948D3884E690E0E1CF90
:10F45000CF93DF931F92CDB7DEB780915E09811104
:10F4600003C080EA99E02FC0211103C08EE599E026
:10F470002AC08DE0815048F0440F411DE82FF0E094
:10F48000E056F64F90814927F5CF8091B306841757
:10F49000A9F04093B3068EE599E069832DDF90E0F3
:10F4A0006981861B910997FF02C080E090E08093FC
:10F4B000C4061092C50688E0809324028091C50698
:10F4C00090E0825A964F0F90DF91CF9108958093EC
:10F4D000C1061092BD061092BE061092BF06109291
:10F4E000C00608958091BC061092BC0608957F92D4
:10F4F0008F929F92AF92BF92CF92DF92EF92FF9244
:10F500000F931F93CF93DF93CDB7DEB728970FB636
:10F51000F894DEBF0FBECDBF7C014B016A015901DB
:10F52000FB0180816CE0689F600D1124F7018081F0
:10F53000982F990F890F880F0E94B837C114D104F2
:10F5400009F496C0FE82ED8298868F82011103C075
:10F550001C2D0D2D74C09D2C0C2D1D2DD12C8824FF
:10F560008394AE014F5F5F4FB5018C2D992D75DDF2
:10F57000C82E992E89819A81AB81BC81772473949E
:10F580000097A105B105C9F0712C80329105A10544
:10F59000B10581F0AC01BD014D52510961097109FC
:10F5A000423051056105710540F08B97A105B10509
:10F5B00089F503C0DD2009F455C0F70120818D2DA8
:10F5C00090E0820F911D46972CF0253018F0CE0167
:10F5D0000596D4DE372D3825D30EF70180818D0DA9
:10F5E0008083DD2089F0DA94AE014F5F5F4FB50173
:10F5F000C80133DD8C0169817A818B819C814FEF59
:10F600005FEF0E94C337EDCF711032C00C2D192D62
:10F61000D12CA7CFD3940115110509F0A2CF0C2D41
:10F62000192D9FCF4FEF5FEF0E94C337F701208165
:10F630002F5F2083253118F0CE0105969FDEAE01A5
:10F640004F5F5F4FB501812F902F07DD182F092FD6
:10F6500069817A818B819C81611571058105910594
:10F6600009F706C00115110589F20F5F1F4FD3CFAF
:10F6700028960FB6F894DEBF0FBECDBFDF91CF91B5
:10F680001F910F91FF90EF90DF90CF90BF90AF90C0
:10F690009F908F907F900895AF92BF92CF92DF920C
:10F6A000EF92FF920F931F93CF93DF931F921F92BE
:10F6B000CDB7DEB75C016B017A013FDE182FE11494
:10F6C000F10419F0C70139DE01C080E01A82198205
:10F6D000C114D104C1F4412F50E090E09A01280FE9
:10F6E000391F263131057CF425E130E0241B350B30
:10F6F000281B390B37FF02C02F5F3F4F35952795E9
:10F700002A8381E0898301E02AEC37E7A501BE0165
:10F710006F5F7F4FCE010296EADEC114D10489F0FB
:10F720008A81882321F01A8289818F5F898300E092
:10F7300027EC37E7A601BE016F5F7F4FCE0102962F
:10F74000D6DEE114F10451F000E02AEC37E7A7011E
:10F75000BE016F5F7F4FCE010296C9DE0F900F9002
:10F76000DF91CF911F910F91FF90EF90DF90CF909D
:10F77000BF90AF900895CF92DF92EF92FF920F93D8
:10F780001F930E947E2B0091AF061091B00620912E
:10F79000B1063091B2066B017C01C01AD10AE20AAF
:10F7A000F30AF7FC13C02091AE0620952093AE0615
:10F7B000DC01CB018A549C4FAF4FBF4F8093AF0603
:10F7C0009093B006A093B106B093B20681E09091F9
:10F7D000AE06911101C080E01F910F91FF90EF9054
:10F7E000DF90CF900895CF9393E090932202811100
:10F7F0001092D1060E947E2BDC01CB018C509E4FD3
:10F80000AF4FBF4F8093CB069093CC06A093CD060D
:10F81000B093CE0668E873E182E090E00F94283B55
:10F82000C6E0C15049F00F94C73A62E070E080E052
:10F8300090E00E94AF2BF5CFCF910895AF92BF9289
:10F84000CF92DF92EF920F931F93CF93DF9300D06D
:10F850001F92CDB7DEB7809123028F3F09F444C0D9
:10F860000E947E2B0091B4061091B5062091B60639
:10F870003091B706DC01CB01801B910BA20BB30BBF
:10F88000B7FD32C09091E00E8091E30E8F5F8F70D4
:10F89000981751F1E091230284E0E802F00111246D
:10F8A000E058FC4F20E030E040E752E46081718195
:10F8B000828193810F94F24069837A838B839C8346
:10F8C000A12CB12C6501E12C8E010F5F1F4F26E7A3
:10F8D00032E042E752E06EE672E08AE692E00E9491
:10F8E00062F68FEF809323020F900F900F900F908E
:10F8F000DF91CF911F910F91EF90DF90CF90BF904C
:10F90000AF9008950F931F930E947E2B0091CB061A
:10F910001091CC062091CD063091CE06DC01CB01B2
:10F92000801B910BA20BB30BB7FD0FC0809103019D
:10F9300085FB992790F981E089279091030196FF33
:10F940008260629B84608093D1068091D106817031
:10F950009091D10691FD82609091A206891741F1A4
:10F960008130A9F028F0823041F0833059F01EC078
:10F97000913089F09230A9F019C0992361F0933049
:10F9800081F014C0913069F0923081F404C0992361
:10F9900041F0933059F49091C6069F5F9093C6064C
:10F9A00005C09091C60691509093C6068093A2061A
:10F9B0001F910F910895CF93DF930E945340E4E08D
:10F9C000F1E080818F7D8083C5E0D1E088818095E2
:10F9D0008072A3E0B1E08C9380818F7B80838881EB
:10F9E000809580748C936A98729A54985C9A82E09D
:10F9F0008093D00687DF1092C606DF91CF910895DD
:10FA0000CF93C091170783ED96E076DCC81790F48A
:10FA1000809117078F5F21E0280FE82FF0E0ED526B
:10FA2000F94F9081907C903811F4822FF4CF80931D
:10FA3000170702C010921707CF9108950F931F93D5
:10FA4000CF93DF938C01C0911707D0E0CD52D94FEF
:10FA5000CE0152DCF8018083CE01DF91CF911F915E
:10FA60000F91089581E09091D306911101C080E03B
:10FA70000895CF93DF9320911607211120C0FC0138
:10FA800001900020E9F73197EF01C81BD90BC3346F
:10FA9000D10534F031972081207C2038D9F3F4CF80
:10FAA000BC01DD27AE0183ED96E00F947349CD5282
:10FAB000D94F18821092170783E080932202DF91BA
:10FAC000CF910895CF93DF93CDB7DEB78E8190911C
:10FAD0001607891790F0809316079E01275F3F4F06
:10FAE0004F81588562E470E083ED96E00F94BC4945
:10FAF0001092170783E080932202DF91CF9108953F
:10FB00000F931F93CF93DF938C0167FF03C0109275
:10FB1000160760E08091160790E0262F062E000C55
:10FB2000330B281739071CF160931607C8010F948F
:10FB3000D548F801E80FF91FEF01C01BD10BC33402
:10FB4000D10534F031978491807C8038D9F3F4CF9B
:10FB5000DD27AE01B80183ED96E00F94F648CD5253
:10FB6000D94F18821092170783E080932202DF9109
:10FB7000CF911F910F9108954F925F926F927F9254
:10FB80008F929F92AF92BF92CF92DF92EF92FF92AD
:10FB90000F931F930E947E2B6B017C014FDEB2DE20
:10FBA0008091D10682FF15C08091AD06811113C0EE
:10FBB00091E09093AD0620914D17211103C08091E3
:10FBC0005D0689278093BC0610924D1781E00BDEFD
:10FBD00002C01092AD0689B184FB992790F981E0AB
:10FBE00089271091D006811749F18093D006882388
:10FBF00009F4CAC164EF71E080E090E00E94F898D7
:10FC00000E94008A123009F0BAC10E94D78A0E946D
:10FC1000534083E0809322020E947E2B6B017C0183
:10FC2000DC01CB018C599F4FAF4FBF4F8093A9068A
:10FC30009093AA06A093AB06B093AC068091A90658
:10FC40009091AA06A091AB06B091AC06A7019601CF
:10FC5000281B390B4A0B5B0B57FF05C08091CA0666
:10FC6000882309F41BC2D701C6018C599F4FAF4F9F
:10FC7000BF4F8093A9069093AA06A093AB06B093BA
:10FC8000AC066091C606062E000C770B77FF03C00A
:10FC9000719561957109062E000C770B880B990BF5
:10FCA0000F948D412B013C0120E030E040E050E416
:10FCB0000F94EE4287FF05C08091BC0681117DC084
:10FCC0008DC08091C106882309F456C08090BD067E
:10FCD0009090BE06A090BF06B090C006811491041B
:10FCE000A104B104E1F120E030E040E05FE3C301B2
:10FCF000B2010F9429432B013C01C701B6016819D9
:10FD000079098A099B090F948B419B01AC01C301BE
:10FD1000B2010F94F24020E030E04AE754E40F943F
:10FD200029434B015C0120E030E040EA52E40F94AB
:10FD3000EE4287FF0FC020E030E040EF51E4C50104
:10FD4000B4010F94EE4287FD0AC02AE030E040E0A3
:10FD500050E009C024E630E040E050E004C021E07B
:10FD600030E040E050E0C092BD06D092BE06E09286
:10FD7000BF06F092C00604C021E030E040E050E051
:10FD8000A091C6060091C7061091C8060A2E000C65
:10FD9000BB0B0F94944422E030E040E050E00F941D
:10FDA0005744DA01C901800F911FA11DB11D909325
:10FDB000C8068093C7061092C606D701C6018856AA
:10FDC000954CAF4FBF4F8093A5069093A606A09386
:10FDD000A706B093A80681E0809322022091C20674
:10FDE0003091C30649E7223D340741F48091240253
:10FDF000882309F4D2C08150809324022D583644C0
:10FE000051F580912402882321F0815080932402AF
:10FE100022C084E0809324028091C5068F5F809386
:10FE2000C5069091C406981728F41092C5068CE078
:10FE30008093240281E080932202D701C601885674
:10FE4000954CAF4FBF4F8093A5069093A606A09305
:10FE5000A706B093A80680916F0081FB222720F9A6
:10FE600081FF05C080916F008D7F80936F0080912E
:10FE7000F30D9091F40DA091F50DB091F60D2223A4
:10FE800029F020916F00226020936F003AE0B69530
:10FE9000A795979587953A95D1F7009721E0A20706
:10FEA000B10520F08FEF9FEFA0E0B0E09695879529
:10FEB00020912202211105C03091CA063111EAC0F9
:10FEC00051C0009741F04091A3065091A4064817F5
:10FED000590708F047C08091CA06811117C0223027
:10FEE00008F06BC080917C04811107C081E0809391
:10FEF0007C0483E494E00E94513083E494E00E9407
:10FF0000883081E08093C9068093CA0683E00E940E
:10FF1000983F61E083E494E00E94B130E091C20632
:10FF2000F091C30619951092C9068091CA068111F5
:10FF300050C01092BC060E947E2BDC01CB018C19B4
:10FF40009D09AE09BF090091A3061091A40620E007
:10FF500030E0081719072A073B0720F49093A406FE
:10FF60008093A3068091C2069091C306825D994753
:10FF700009F481C08091CF0681117DC050C060E03E
:10FF800082E691E3BDDD43CEE6D5123009F43FCEE3
:10FF900060E085E591E3B4DD3ACE8CE08093240205
:10FFA0008091A3069091A40601979093A406809354
:10FFB000A30681E08093220221CF243030F0243048
:10FFC00009F090CF109222028DCF81E0809322021F
:10FFD00089CF83E494E00E948C3091E0811101C0CC
:10FFE00090E09093CA06992309F4A3CF0E947E2B38
:10FFF000DC01CB018C199D09AE09BF09C090A30695
:020000021000EC
:10000000D090A406E12CF12CC816D906EA06FB060E
:1000100008F044C09093A4068093A3063FC080914B
:10002000A5069091A606A091A706B091A806C81AA9
:10003000D90AEA0AFB0AF7FE0E9485758091CA0672
:1000400081112CC080912202813091F0833031F5F2
:100050001F910F91FF90EF90DF90CF90BF90AF90E6
:100060009F908F907F906F905F904F900C948840FE
:100070001092220213C048E9C40E4AE3D41EE11CC8
:10008000F11CC092A506D092A606E092A706F092B7
:10009000A806D4CF009709F439CF15CF1F910F913F
:1000A000FF90EF90DF90CF90BF90AF909F908F9098
:1000B0007F906F905F904F90089561E021DD0C94E8
:1000C0008575CF93DF931F921F92CDB7DEB78983DB
:1000D0009A8371DC89819A81F0DF0F900F90DF9114
:1000E000CF910C9458408091AD0982FD05C080915C
:1000F0004217823061F410C080915E09811103C003
:1001000080EA99E002C08EE599E061E0B2CC8130EE
:1001100031F087E291E305C088E491E302C08CE30B
:1001200091E36FEFEDCC10924D1710928502809104
:10013000AD0980628093AD090E94BDA70F94673B13
:1001400060E089E191E3DCDC0C9485758DE091E35E
:100150000E94597660E080E091E3D2DC40E061E00B
:1001600080E00E94FE5F86EF90E30D94D428BBDF11
:1001700010924D17109285020E946060882321F032
:100180008091AD0982FF04C00E94B5A70D94E03BA9
:1001900082EF90E30F94D428F7CF8091AD0982FFCE
:1001A0002AC00E946060882319F1809168079091AD
:1001B0006907A0916A07B0916B070097A105B10587
:1001C000B9F0BC01CD016D597F4F8F4F9F4F24E691
:1001D00030E040E050E00F94354460916407709146
:1001E000650780916607909167070F94354401C0B9
:1001F00020E02093D2068091D206089582ED99E7FF
:100200009093C3068093C206089561E0FC0180814B
:100210000E94AE2D8FEF0C942EA0CF93DF93EC01B4
:100220008A810E94F09F60E08881DF91CF910C94D9
:10023000AE2D8F929F92AF92BF92EF92FF920F934B
:100240001F93CF93DF93EC018B017A010E947E2BE9
:100250004B015C012CE2820E21E0921EA11CB11C1C
:100260000E9408A08B838F3F61F40E947E2BDC01EB
:10027000CB0188199909AA09BB09B7FDF1CF81E122
:100280000DC08E3F51F4B701C8010E940FA00E941B
:1002900008A00E9408A011E003C08FE0898310E04D
:1002A000CE01B3DF812FDF91CF911F910F91FF908E
:1002B000EF90BF90AF909F908F900895CF92DF9274
:1002C000EF92FF926A017B010E947E2BC60ED71E21
:1002D000E81EF91E0E9408A08F3F61F00E947E2B4D
:1002E000DC01CB018C199D09AE09BF09B7FDF2CF26
:1002F00080E001C081E0FF90EF90DF90CF90089503
:10030000EF92FF921F93CF93DF9300D01F92CDB750
:10031000DEB77C01162F29833A834B835C837DDF14
:1003200048E552E060E070E0C701C8DF812F8064DB
:100330000E942EA08C810E942EA08B810E942EA054
:100340008A810E942EA089810E942EA0112311F083
:1003500087E801C085E90E942EA01C3011F40E949C
:1003600008A010E00E9408A0F701838387FF04C063
:100370001F3F11F01F5FF6CF0F900F900F900F905F
:10038000DF91CF911F91FF90EF9008958F929F92F0
:10039000AF92BF92CF92DF92EF92FF920F931F9393
:1003A000CF93DF93EC01162F1C82198248830E94A1
:1003B0007E2B6B017C0120EDC20E27E0D21EE11CDA
:1003C000F11CA89561E088810E94AE2D61E08881D2
:1003D0000E94722D0E9401A085E08A830E94F09FF6
:1003E0000AE08FEF0E942EA00150D9F7A89520E0D7
:1003F00030E0A90160E0CE0183DF8B83813061F0C2
:100400000E947E2BDC01CB018C199D09AE09BF092E
:10041000B7FDEDCF81E055C0A8952AEA31E040E074
:1004200050E068E0CE016CDF853011F481E009C056
:1004300004E00E9408A08B830150D9F78A3A51F456
:1004400082E08C83A8958C81823081F0812C912C64
:10045000540111C00E947E2BDC01CB018C199D0937
:10046000AE09BF09B7FDD9CF82E02BC0812C912CFA
:10047000A12C80E4B82E20E030E0A90167E3CE0192
:100480003FDFA501940169E2CE013ADF8B83882327
:1004900061F00E947E2BDC01CB018C199D09AE0915
:1004A000BF09B7FDE8CF8AE00CC08C818230D1F45F
:1004B00020E030E0A9016AE3CE0122DF882329F0A1
:1004C00088E08983CE01A1DE16C00E9408A0807C4E
:1004D000803C11F483E08C830E9408A00E9408A055
:1004E0000E9408A0CE0191DE173018F41A8381E033
:1004F00003C088E1898380E0DF91CF911F910F9144
:10050000FF90EF90DF90CF90BF90AF909F908F9033
:1005100008950F931F93CF93DF93EC0189018C8192
:10052000833039F089E0440F551F661F771F8A9585
:10053000D1F79A01AB0161E1CE01E2DE811109C080
:1005400040E052E0B801CE01DF91CF911F910F91B1
:1005500070CE84E08983CE0158DE80E0DF91CF91B8
:100560001F910F910895CF93DF93EC01862FBA016D
:100570000E9433A08FEF0E942EA08FEF0E942EA02A
:100580000E9408A08B83982F9F71953031F083E1F2
:100590008983CE013ADE80E001C081E0DF91CF9116
:1005A00008950F931F93CF93DF93EC0189018C8102
:1005B000833039F089E0440F551F661F771F8A95F5
:1005C000D1F79A01AB0168E1CE019ADE81111EC01C
:1005D000A8016EEFCE01C7DF8823E1F048E552E0C5
:1005E00060E070E0CE016ADE882371F020E030E048
:1005F000A9016DE0CE0184DE81110AC00E9408A02D
:10060000811106C011E007C087E103C086E001C088
:1006100086E1898310E0CE01F8DD812FDF91CF9153
:100620001F910F910895CF93DF931F92CDB7DEB73F
:1006300020914F1730915017CE01019621153105A9
:1006400019F0821B930B02C0855597410F90DF91E3
:10065000CF910895FC01238121110C9441940895B8
:1006600088E197E0F7CF83E397E0F4CF80914E07DE
:10067000811107C00E940ED9882319F081E0809370
:100680004E0708958091AD09847F8B7F8093AD09DB
:100690001092640710926507109266071092670720
:1006A000109268071092690710926A0710926B0700
:1006B0001092D907109218088EE091E0E9E1F8E075
:1006C000DF019C011D9221503040E1F78FEF8093B4
:1006D0005D090895FC0120E03EE2DB014C914032CF
:1006E00041F0283011F430833196DB014C91408386
:1006F00031962F5F6F5F7F4F2B3079F7108208950F
:100700002F923F924F925F926F927F928F929F9221
:10071000AF92BF92CF92DF92EF92FF920F931F930F
:10072000CF93DF93CDB7DEB7C356D1090FB6F89498
:10073000DEBF0FBECDBF8C015B014A014DB65EB678
:10074000312C7E0187E5E80EF11C9BE1292E4EE558
:1007500059E0BE016F5F7F4FC5010E94B19218162C
:100760000CF005C18C85282F2871203109F074C048
:10077000909163079150923008F46EC06DB67EB6CA
:10078000BE016F5F7F4FC701A5DF0115110521F085
:10079000F8018081811173C021E081E090E0F701D0
:1007A00001900020E9F73197EE19FF09E80FF91FD2
:1007B00032968DB79EB78E1B9F0B0FB6F8949EBFD7
:1007C0000FBE8DBFEDB7FEB731966F01211102C08C
:1007D000B80102C060E973E0C6010F945E49B70139
:1007E000C6010F94484960E973E0C6010F94484977
:1007F0001CAE1FAE21E0A701B501CE01CC960E9430
:100800003D9681110DC080916307811109C00E943E
:100810002A9983E693E30E941C99C7010E94C69E11
:10082000FE01FC96DE019196822D01900D928A9533
:10083000E1F740E050E0BE016F5D7F4FC60160DF31
:10084000CE01819607DFCE01CC9604DF0FB6F89477
:100850007EBE0FBE6DBE7BCF9981992309F487C000
:10086000953E09F474CF9E3209F471CF90915E09E0
:100870009E3209F46CCF8A7009F069CF0AC0F80182
:1008800001900020E9F73197CF01801B910B20E008
:1008900086CF81E0203109F080E09091AD0980FBA6
:1008A00094F99093AD09811108C08985873409F0C6
:1008B0004ECF8A858E3709F44ACF80916307813005
:1008C00021F068F08230B9F142CF809161079091B8
:1008D00062070196909362078093610738CFBE014B
:1008E0006F5F7F4F80EA99E0F5DE0115110511F089
:1008F000680105C080EAC82E89E0D82E08C0F6013C
:1009000081916F018823B1F30E946F9EF8CFF601A9
:1009100081916F01882319F00E946F9EF8CF80E2C9
:100920000E946F9E6D8D7E8D8F8D98A14AE050E064
:100930000E947C9F0CCFBE016F5F7F4F80EA99E0E1
:10094000C9DE8114910441F060EA79E0C4010F949A
:100950003549892B51F40BC0832D90E020915F071E
:10096000309160078217930711F03394F0CE0FB6E1
:10097000F8945EBE0FBE4DBECD59DF4F0FB6F89452
:10098000DEBF0FBECDBFDF91CF911F910F91FF90C2
:10099000EF90DF90CF90BF90AF909F908F907F901F
:1009A0006F905F904F903F902F900895CF93DF937B
:1009B000CDB7DEB76B970FB6F894DEBF0FBECDBFD5
:1009C0001092630740E050E0BA0182E499E00E948F
:1009D00060938BE1E2E4F9E0DE01119601900D9263
:1009E0008A95E1F740E050E0BE016F5F7F4F80E005
:1009F00090E086DECE0101962DDE6B960FB6F89460
:100A0000DEBF0FBECDBFDF91CF9108950F931F932F
:100A1000CF93DF93CDB7DEB72D970FB6F894DEBF37
:100A20000FBECDBF8091DD07882391F0BE016F5FBF
:100A30007F4F8AED97E00E94D3908E010F5F1F4F8A
:100A4000F80181918F01882339F00E946F9EF8CFC1
:100A500089E593E30E941C998AE00E946F9E2D967F
:100A60000FB6F894DEBF0FBECDBFDF91CF911F91BF
:100A70000F910895CF92DF92EF92FF920F931F9301
:100A8000CF93DF93CDB7DEB7EDB6FEB6DC010D90A8
:100A90000020E9F79D01281B390B2C5F3F4F4DB714
:100AA0005EB7421B530B0FB6F8945EBF0FBE4DBF2F
:100AB0000DB71EB70F5F1F4F9F938F9383E193E393
:100AC0009F938F931F930F930F948D49680154E068
:100AD000C50ED11C0F900F900F900F900F900F909C
:100AE000F6018081882349F0082E000C990B0F94A1
:100AF000B948F60181936F01F3CFC8010F94D9284B
:100B00008FE093E30F94E7280FB6F894FEBE0FBE74
:100B1000EDBEDF91CF911F910F91FF90EF90DF908D
:100B2000CF9008958091AD0983FF03C084608093C6
:100B3000AD09089510927A0C8091AD098F7D8B7F5D
:100B40008093AD090E946060882321F08AED97E0D0
:100B50000C9441940895EEDF8091AD09877F8093D6
:100B6000AD0908950F931F93CF93DF938B01EA0193
:100B7000DB016D917C910E94D390D801ED91FC91A5
:100B80009081888191110EC08936B0F48FE2808304
:100B9000F8018081918101969183808388818F5FA4
:100BA00088830AC0893680F73196D801ED93FC938B
:100BB00088818F5F8883E1CFDF91CF911F910F9163
:100BC00008950F931F93CF93DF9300D0CDB7DEB777
:100BD0009C012F5F3F4F3B832A832FE2FC01208340
:100BE00081E0898310E00BE180911808181770F4F8
:100BF000019FC0011124AE014F5F5F4FBE016E5FC8
:100C00007F4F875E974FAEDF1F5FEECF89818B35B9
:100C100070F4AE014F5F5F4FBE016E5F7F4F8AED94
:100C200097E0A0DF8A819B8101979B838A83EA8179
:100C3000FB8110820F900F900F90DF91CF911F9149
:100C40000F9108958091AD0982FF1FC087ED91E358
:100C50000E941C99609164077091650780916607F6
:100C6000909167074AE050E00E94719F8FE20E94D6
:100C70006F9E609168077091690780916A079091F3
:100C80006B074AE050E00C947C9F86EC91E30C9457
:100C90001C99EF92FF920F931F93CF93DF938C01D8
:100CA000FC0101900020E9F73197EF01C81BD90B37
:100CB0001092DA076EE470E00F9453497C010097BC
:100CC00029F4FE013197E00FF11F0EC060E270E0E1
:100CD0000F9453498C010F5F1F4F6AE270E0C70108
:100CE0000F945349FC0131978DE081838AE0828320
:100CF0001382B8018AED97E00E94D0988091DA07BC
:100D0000882361F00E942D998FEA91E3DF91CF91C2
:100D10001F910F91FF90EF900C941C99DF91CF9150
:100D20001F910F91FF90EF9008958AED97E00E9438
:100D3000F6938AED97E00E9441948091AD098D7FF2
:100D40008E7F8093AD091092640710926507109210
:100D500066071092670781E080936B0C08950F93EC
:100D60001F93CF93DF93CDB7DEB76B970FB6F89491
:100D7000DEBF0FBECDBF8B0122E0209363079093AF
:100D8000600780935F0740E050E0BA0187E299E096
:100D90000E9460938BE1E7E2F9E0DE011196019099
:100DA0000D928A95E1F7A801BE016F5F7F4F80E049
:100DB00090E0A6DCCE0101964DDC6B960FB6F89460
:100DC000DEBF0FBECDBFDF91CF911F910F91089570
:100DD000CF93DF93CDB7DEB76B970FB6F894DEBF36
:100DE0000FBECDBF81E0809363071092620710921F
:100DF000610740E050E0BA0187E299E00E94609309
:100E00008BE1E7E2F9E0DE01119601900D928A95FF
:100E1000E1F740E050E0BE016F5F7F4F80E090E07F
:100E20006FDCCE01019616DC80916107909162071C
:100E30006B960FB6F894DEBF0FBECDBFDF91CF919A
:100E400008952F923F924F925F926F927F928F926E
:100E50009F92AF92BF92CF92DF92EF92FF920F9349
:100E60001F93CF93DF9300D01F92CDB7DEB77C01E5
:100E70008B01342E2DB73EB73C832B8380915707CF
:100E800081110BC0109233071092360781E08093D6
:100E9000570783E393E80E94A63780914F0781119B
:100EA0000BC01092180710921B0781E080934F0728
:100EB00080E393E80E94A637F80180818F3251F4D5
:100EC00082E499E0F70191838083109218080F5F04
:100ED0001F4F05C087E299E0F70191838083F701F6
:100EE0000190F081E02DFA83E98323E3A22E27E02D
:100EF000B22E3BE1232E0115110509F47FC04DB63A
:100F00005EB66FE270E0C8010F9453493C010817C8
:100F1000190708F073C06C01C01AD10ADD24C6019C
:100F200001962DB73EB7281B390B0FB6F8943EBF7C
:100F30000FBE2DBF8DB79EB701964C01A601B8011B
:100F40000F947349F401EC0DFD1D1082332019F04C
:100F5000C4010E94C69EF7016081718121E0A40155
:100F6000C5010E943D96811111C0B40182E991E34F
:100F70000E9430998FE891E30E941C990FB6F89473
:100F80005EBE0FBE4DBE80E090E039C0F7018081AB
:100F9000918129813A818217930711F00E9441942F
:100FA000F701B182A082A0911808AA3078F481E0FC
:100FB0008A0F809318082A9ED0011124A75EB74F8C
:100FC000F501822D01900D928A95E1F7F70180815C
:100FD00091818353974029F498E1A92E97E0B92E87
:100FE00004C083E3A82E87E0B82E83010F5F1F4F54
:100FF0000FB6F8945EBE0FBE4DBE7DCFC8012B81EB
:101000003C810FB6F8943EBF0FBE2DBF0F900F90DE
:101010000F900F90DF91CF911F910F91FF90EF9064
:10102000DF90CF90BF90AF909F908F907F906F9008
:101030005F904F903F902F9008950F931F93CF9301
:10104000DF931F921F92CDB7DEB72091AD0923FF2A
:1010500028C0BC0140E0CE010196F3DE8C01009770
:1010600001F1BC0189819A810E941797B8018823F8
:1010700081F084E092E30E9430998AE00E946F9EA2
:101080001092640710926507109266071092670726
:1010900008C08CEE91E30E94309989EE91E30E94A2
:1010A0001C990F900F90DF91CF911F910F91089590
:1010B000EF92FF920F931F93CF93DF9300D0CDB7A2
:1010C000DEB72091AD0923FF09C1F42EE62E8C0175
:1010D0000E946060882309F451C0FF2009F45BC0BE
:1010E0008091D907882359F00E942D998AEC92E3C8
:1010F0000E941C9980E090E00F94573EEFC08CE670
:1011000097E05FDDE091D90784E0E89FF0011124CA
:10111000EB52F84F8091640790916507A0916607A4
:10112000B091670780839183A283B3830E942A9939
:10113000B80181EB92E30E9430998091D90799E63A
:10114000899FB00111246459784F86EA92E30E9486
:1011500030994091640750916507609166077091DE
:10116000670780EA92E30E9491998AE00E946F9E4D
:101170008091D9078F5F8093D90725C0FF2039F070
:101180000E942A9980E992E30E941C991CC0109247
:10119000D90722E001C021E02B830E942A998BE825
:1011A00092E30E941C992B81213009F494C08FE7AF
:1011B00092E30E941C99B80187E792E30E9430995C
:1011C0008AE00E946F9EB6DC40E0B801CE01019635
:1011D00038DE8C01009709F481C069817A81EE20A4
:1011E00009F44FC021E0AC018AED97E00E943D96E2
:1011F000882309F43EC08091EB079091EC07A09101
:10120000ED07B091EE078093680790936907A0936C
:101210006A07B0936B0710926407109265071092EB
:10122000660710926707B80189E692E30E94309939
:10123000409168075091690760916A0770916B0748
:1012400081E692E30E9491998AE00E946F9E82E576
:1012500092E30E941C99B80180E090E080DD8091CB
:101260005E09811102C0C80102C08EE599E060E00C
:101270002FC0B8018EE392E30E9430998BE392E392
:101280000FC026E5AC018AED97E00E943D968111E2
:101290000AC0B80187E292E30E94309984E292E3A7
:1012A0000E941C991BC08091AD0981608093AD099B
:1012B000B80180E090E053DD10926B0CB80182E140
:1012C00092E30E9430998AE00E946F9E60E0C8011C
:1012D0000E94397D03C085E892E36BCF0F900F9099
:1012E0000F90DF91CF911F910F91FF90EF90089594
:1012F0002091AD0922602093AD0940E060E0D8CE96
:101300000F931F93CF93DF93CDB7DEB76B970FB6D5
:10131000F894DEBF0FBECDBF8C0119821C82809174
:101320002A09811103C062E479E002C067E279E032
:1013300021E0A801CE0101960E943D968823F1F09C
:101340008BE1FE013196A7E2B9E001900D928A95FA
:10135000E1F7A0911808AA30D8F481E08A0F8093B1
:1013600018088BE18A9FD0011124A75EB74FE7E2EE
:10137000F9E001900D928A95E1F70AC00E942A993E
:10138000B80189E791E30E9430998AE00E946F9E3C
:10139000CE0101965FD96B960FB6F894DEBF0FBEF3
:1013A000CDBFDF91CF911F910F91089580911808C3
:1013B0008823C9F0815080931808882359F090E061
:1013C00001972BE1289FF001299FF00D1124E75E82
:1013D000F74F02C0E2E4F9E08BE1A7E2B9E0019047
:1013E0000D928A95E1F78091180808958BE1E2E467
:1013F000F9E0A7E2B9E001900D928A95E1F708952E
:101400008091AD09877F8093AD098091450988233C
:1014100021F082E499E00E94419445E360E083E199
:1014200098E00E94C681811105C00E942A998BE430
:1014300093E314C041E063E178E085EF97E08AD45C
:1014400081110FC040E063E178E085EF97E082D43E
:10145000811107C00E942D9987E393E30E941C9994
:1014600018C065EF77E082E499E0F9D6811105C0F4
:101470000E942D9986E293E3F1CF8091AD098860B7
:101480008093AD090E942A998AE193E30E941C99F6
:10149000EDD8ACDF83E0809322020895AF92BF9233
:1014A000CF92DF92EF92FF921F93CF93DF93CDB74E
:1014B000DEB7A8970FB6F894DEBF0FBECDBF809100
:1014C0005D0987FD64C08091AD0982FD60C083FD28
:1014D00002C096DF01C0CAD88091AD0983FF54C015
:1014E00080915D09082E000C990BC0969F938F93F5
:1014F00086EA91E39F938F936E0181E2C80ED11C1F
:10150000DF92CF920F948D4940E050E0BA0182E41F
:1015100099E00E9460930F900F900F900F900F90A2
:101520000F90FE0131967F0140E050E0B70182E468
:1015300099E00E94B19218163CF5F7010190002045
:10154000E9F731971E2F1E19115068F05701A10EAF
:10155000B11C17FDBA94F501808190E00F94B94851
:10156000F5018083F1CF8A858E37F1F245E050E0B6
:10157000B601C7010F946549892BB1F6C6017ADA25
:1015800080915D098F5F01C08FEF80935D09A89600
:101590000FB6F894DEBF0FBECDBFDF91CF911F9184
:1015A000FF90EF90DF90CF90BF90AF900895109292
:1015B0005D091CCF0DCC0E94FCE88AED97E00E94EB
:1015C00041948091D907882329F181508093D907CC
:1015D00029E6829FC001112441E061E08459984FBF
:1015E00067DDE091D90784E0E89FF0011124EB5218
:1015F000F84F408151816281738140936407509319
:10160000650760936607709367078AED97E00E940D
:10161000609388CA8FDA0E94D6E80F94673B0F94D4
:10162000AC3B6D3371058105910518F480E791E3BA
:1016300002C085E791E30F94E72884E68093D20601
:1016400008951092420910924509109227091092AC
:101650002A0980E090E0FC01E75EF74F10821382D8
:101660004B968E3021E09207B1F789E18093140800
:101670001092170810920C081092DA071092DD07EA
:101680000895CF93DF938AED97E00E942A83C7E203
:10169000D9E06B97CE010E942A8388E0C931D80730
:1016A000C1F787E299E00E942A8382E499E0DF9102
:1016B000CF910C942A83CF938091B2098823B9F1FA
:1016C0004091B50B5091B60B6091B70B7091B80B70
:1016D00025EB39E08091B3099091B4090E94D18241
:1016E000C82F811102C0C0E023C04091AE095091C3
:1016F000AF096091B0097091B109411551056105BB
:10170000710591F025EB39E08091B3099091B4090E
:101710000E94D182882339F31092AE091092AF094A
:101720001092B0091092B1091092B20901C0C1E043
:101730008C2FCF910895CF92DF92EF92FF92CF93AB
:101740006B017C01C42F8091B50B9091B60BA091D9
:10175000B70BB091B80B8C159D05AE05BF05C9F050
:10176000AADF811102C080E018C025EB39E0B70183
:10177000A6018091B3099091B4090E9489828823BF
:1017800091F3C092B50BD092B60BE092B70BF092EA
:10179000B80B81E0C1118093B209CF91FF90EF9017
:1017A000DF90CF900895CF92DF92EF92FF920F9348
:1017B0001F93CF93DF93FC0181859285A385B48528
:1017C0000196A11DB11D84179507A607B70710F450
:1017D00080E060C08789803149F4BB27A72F962F0E
:1017E000852FC388D488E588F6880FC0803281F7BA
:1017F00083899489A589B6896A017B01C7E0F6943B
:10180000E794D794C794CA95D1F78C0D9D1DAE1D52
:10181000BF1DE9016A017B018F014091B50B509119
:10182000B60B6091B70B7091B80B84179507A6079C
:10183000B70731F040E0BC01CD017DDF882341F2E4
:10184000F8018789803179F4B701A6015527662709
:101850007727440F551FFA01EB54F64F8081918191
:10186000A0E0B0E012C0B701A6014F775527662768
:101870007727440F551F440F551FFA01EB54F64FBD
:1018800080819181A281B381BF7088839983AA836B
:10189000BB8381E0DF91CF911F910F91FF90EF907B
:1018A000DF90CF9008954F925F926F927F92AF92A8
:1018B000BF92CF92DF92EF92FF920F931F93CF933D
:1018C000DF9300D01F92CDB7DEB78C0149835A83D6
:1018D0006B837C835901C12CD12C7601412C82E091
:1018E000582E612C712C49815A816B817C819E011B
:1018F0002F5F3F4FC80157DF882341F1D301C20159
:10190000F801058404C0880F991FAA1FBB1F0A9401
:10191000D2F7C80ED91EEA1EFB1E49815A816B817F
:101920007C818789803139F481E0483F5F4F6105D0
:10193000710538F4D8CF81E0483F5F4F6F4F7F404B
:1019400090F2F501C082D182E282F3820F900F9073
:101950000F900F90DF91CF911F910F91FF90EF901B
:10196000DF90CF90BF90AF907F906F905F904F903F
:1019700008954F925F926F927F928F929F92AF9253
:10198000BF92CF92DF92EF92FF920F931F93CF936C
:10199000DF93EC016A017B012801390142305105D6
:1019A0006105710510F480E064C089859A85AB8576
:1019B000BC850196A11DB11D84179507A607B70721
:1019C00090F38F89803149F48D2C9E2CAF2CBB2451
:1019D0008B899C89AD89BE890FC0803221F78B88A5
:1019E0009C88AD88BE88DB01CA0157E0B695A795F3
:1019F000979587955A95D1F7880E991EAA1EBB1EFA
:101A000041E0C501B40197DE882369F29F899031D6
:101A100061F4DD24EE24FF249601220F331FF90127
:101A2000EB54F64F5182408211C0E894C7F8DD2490
:101A3000EE24FF249601220F331F220F331FF901DA
:101A4000EB54F64F40825182628273829A899230BF
:101A500080F04D815E816F817885840E951EA61E73
:101A6000B71E8092AE099092AF09A092B009B092D1
:101A7000B109DF91CF911F910F91FF90EF90DF900F
:101A8000CF90BF90AF909F908F907F906F905F901E
:101A90004F9008952F923F924F925F926F927F9254
:101AA0008F929F92AF92BF92CF92DF92EF92FF926E
:101AB0000F931F93CF93DF93CDB7DEB72F970FB65A
:101AC000F894DEBF0FBECDBF1C014D835E836F83D4
:101AD00078873B872A87FC0181859285A385B48519
:101AE0008C019D010F5F1F4F2F4F3F4F0C871D87AC
:101AF0002E873F87AA85BB85CD90DD90ED90FC9029
:101B0000C114D104E104F10431F0BFEFCB1ADB0AB8
:101B1000EB0AFB0A10C0F101C080D180E280F380A3
:101B2000F1E0F9870D811E812F8138850130110583
:101B30002105310509F0198646015701412C512C28
:101B40003201F10181859285A385B4854816590635
:101B50006A067B0608F04EC00C851D852E853F85E4
:101B6000081519052A053B0550F482E0882E912CB2
:101B7000A12CB12C92E0C92ED12CE12CF12C9E018C
:101B80002F5F3F4FB501A401C1010DDE882391F104
:101B900049815A816B817C81D501C4010196A11DC7
:101BA000B11D452B462B472B19F06C017D010FC051
:101BB000AC01BD014C195D096E097F090D811E81C3
:101BC0002F813885401751076207730741F01FEFD7
:101BD000411A510A610A710A4C015D01B2CF0FEF3F
:101BE0001FEF2FEF3FE0B501A401C101C2DE8D83DD
:101BF000811113C01D823DC02401350121E0421A2C
:101C000051086108710895018401B301A201C10165
